:020000040800F2
:1000000000000120E5260008C11A0008C31A0008F4
:10001000C51A0008C71A0008C91A00080000000025
:10002000000000000000000000000000CB1A0008E3
:10003000CD1A000800000000CF1A0008D11A0008ED
:100040002D2700082D2700082D270008D91A0008A1
:100050002D270008E91A0008EB1A0008F51A000815
:100060002D2700082D270008FF1A00082D2700085B
:100070002D2700082D2700082D270008091B000840
:100080002D2700082D2700082D2700082D27000800
:10009000191B00082D2700082D2700082D27000810
:1000A0002D2700082D2700082D2700082D270008E0
:1000B0002D2700082D270008291B00082D270008E0
:1000C0002D2700082D2700082D2700082D270008C0
:1000D0002D270008391B00082D270008491B0008A0
:1000E0002D270008591B00082D2700082D27000880
:1000F0002D2700082D2700082D2700082D27000890
:100100002D2700082D2700082D2700082D2700087F
:100110002D2700082D2700082D2700082D2700086F
:100120002D2700082D2700082D2700082D2700085F
:1001300000000000000000000000000000000000BF
:1001400000000000000000000000000000000000AF
:10015000000000000000000000000000000000009F
:10016000000000000000000000000000000000008F
:10017000000000000000000000000000000000007F
:10018000000000000000000000000000000000006F
:10019000000000000000000000000000000000005F
:1001A000000000000000000000000000000000004F
:1001B000000000000000000000000000000000003F
:1001C000000000000000000000000000000000002F
:1001D000000000000000000000000000000000001F
:0401E0005FF8E0F1F3
:1001E8004FF0FF0C1CEAD0521EBF1CEAD15392EA12
:1001F8000C0F93EA0C0F6FD01A4480EA010C4002EE
:1002080018BF5FEA41211ED04FF0006343EA501047
:1002180043EA5111A0FB01310CF00040B1F5000F89
:100228003EBF490041EAD3715B0040EA010062F138
:100238007F02FD2A1DD8B3F1004F40EBC25008BF22
:1002480020F00100704790F0000F0CF0004C08BF40
:1002580049024CEA502040EA51207F3AC2BFD2F10D
:10026800FF0340EAC250704740F400004FF000031B
:10027800013A5DDC12F1190FDCBF00F00040704755
:10028800C2F10002410021FA02F1C2F1200200FA93
:1002980002FC5FEA310040F1000053EA4C0308BF5A
:1002A80020EADC70704792F0000F00F0004C02BFAB
:1002B800400010F4000F013AF9D040EA0C0093F026
:1002C800000F01F0004C02BF490011F4000F013B80
:1002D800F9D041EA0C018FE70CEAD15392EA0C0FEE
:1002E80018BF93EA0C0F0AD030F0004C18BF31F059
:1002F800004CD8D180EA010000F00040704790F02F
:10030800000F17BF90F0004F084691F0000F91F0D2
:10031800004F14D092EA0C0F01D142020FD193EA98
:100328000C0F03D14B0218BF084608D180EA010020
:1003380000F0004040F0FE4040F40000704740F0FC
:10034800FE4040F44000704781F0004102E000BFE9
:1003580083F0004330B54FEA41044FEA430594EA7D
:10036800050F08BF90EA020F1FBF54EA000C55EAB8
:10037800020C7FEA645C7FEA655C00F0E2804FEA89
:100388005454D4EB5555B8BF6D420CDD2C4480EA6B
:10039800020281EA030382EA000083EA010180EA9B
:1003A800020281EA0303362D88BF30BD11F0004FE9
:1003B8004FEA01314FF4801C4CEA113102D040421F
:1003C80061EB410113F0004F4FEA03334CEA13335A
:1003D80002D0524263EB430394EA050F00F0A78072
:1003E800A4F10104D5F1200E0DDB02FA0EFC22FA6D
:1003F80005F2801841F1000103FA0EF2801843FA61
:1004080005F359410EE0A5F120050EF1200E012A51
:1004180003FA0EFC28BF4CF0020C43FA05F3C0188F
:1004280051EBE37101F0004507D54FF0000EDCF108
:10043800000C7EEB00006EEB0101B1F5801F1BD3B1
:10044800B1F5001F0CD349085FEA30004FEA3C0CB5
:1004580004F101044FEA445212F5800F80F09A80AB
:10046800BCF1004F08BF5FEA500C50F1000041EBAF
:10047800045141EA050130BD5FEA4C0C404141EBB3
:100488000101013C28BFB1F5801FE9D291F0000FAE
:1004980004BF01460020B1FA81F308BF2033A3F15D
:1004A8000B03B3F120020CDA0C3208DD02F1140C54
:1004B800C2F10C0201FA0CF021FA02F10CE002F18F
:1004C8001402D8BFC2F1200C01FA02F120FA0CFC88
:1004D800DCBF41EA0C019040E41AA2BF01EB0451D1
:1004E800294330BD6FEA04041F3C1CDA0C340EDCCF
:1004F80004F11404C4F1200220FA04F001FA02F312
:1005080040EA030021FA04F345EA030130BDC4F1CF
:100518000C04C4F1200220FA02F001FA04F340EAC4
:100528000300294630BD21FA04F0294630BD94F075
:10053800000F83F4801306BF81F480110134013D5C
:100548004EE77FEA645C18BF7FEA655C29D094EACD
:10055800050F08BF90EA020F05D054EA000C04BF4B
:100568001946104630BD91EA030F1EBF0021002036
:1005780030BD5FEA545C05D14000494128BF41F0D5
:10058800004130BD14F580043CBF01F5801130BD39
:1005980001F0004545F0FE4141F470014FF00000C4
:1005A80030BD7FEA645C1ABF194610467FEA655C75
:1005B8001CBF0B46024650EA013406BF52EA033517
:1005C80091EA030F41F4002130BD00BF90F0000F05
:1005D80004BF0021704730B54FF4806404F1320441
:1005E8004FF000054FF0000150E700BF90F0000FFA
:1005F80004BF0021704730B54FF4806404F1320421
:1006080010F0004548BF40424FF000013EE700BFF0
:1006180042004FEAE2014FEA31014FEA02701FBF80
:1006280012F07F4393F07F4F81F06051704732F0B2
:100638007F4208BF704793F07F4F04BF41F4002109
:10064800704730B54FF4607401F0004521F0004167
:100658001CE700BF50EA010208BF704730B54FF0F1
:1006680000050AE050EA010208BF704730B511F0F2
:10067800004502D5404261EB41014FF4806404F12A
:1006880032045FEA915C3FF4D8AE4FF003025FEAB0
:10069800DC0C18BF03325FEADC0C18BF033202EB34
:1006A800DC02C2F1200300FA03FC20FA02F001FA8E
:1006B80003FE40EA0E0021FA02F11444BDE600BF31
:1006C8004FF0FF3C06E000BF4FF0010C02E000BF16
:1006D8004FF0010C4DF804CD4FEA410C7FEA6C5CF9
:1006E8004FEA430C18BF7FEA6C5C1BD001B050EA9C
:1006F800410C0CBF52EA430C91EA030F02BF90EA87
:10070800020F0020704710F1000F91EA030F58BF45
:10071800994208BF90422CBFD8176FEAE37040F0A7
:10072800010070474FEA410C7FEA6C5C02D150EA45
:10073800013C07D14FEA430C7FEA6C5CD6D152EA00
:10074800033CD3D05DF8040B704700BF84461046C5
:1007580062468C461946634600E000BF01B5FFF7C4
:10076800B7FF002848BF10F1000F01BD4DF808ED94
:10077800FFF7F4FF0CBF012000205DF808FB00BF65
:100788004DF808EDFFF7EAFF34BF012000205DF8BF
:1007980008FB00BF4DF808EDFFF7E0FF94BF01200C
:1007A80000205DF808FB00BF4DF808EDFFF7CEFF0D
:1007B80094BF012000205DF808FB00BF4DF808ED4C
:1007C800FFF7C4FF34BF012000205DF808FB00BF1D
:1007D8004FEA410C7FEA6C5C02D150EA013C0AD135
:1007E8004FEA430C7FEA6C5C02D152EA033C02D127
:1007F8004FF0000070474FF0010070474FEA410288
:1008080012F5001215D211D56FF47873B3EB62525A
:1008180012D94FEAC12343F0004343EA505311F081
:10082800004F23FA02F018BF404270474FF0000013
:10083800704750EA013005D111F0004008BF6FF051
:10084800004070474FF00000704700BF4FEA410278
:10085800B2F1E04324BFB3F5001CDCF1FE5C0DD916
:1008680001F0004C4FEAC0024CEA5070B2F1004F60
:1008780040EB830008BF20F00100704711F0804F63
:1008880021D113F13872BCBF01F00040704741F428
:1008980080114FEA5252C2F11802C2F1200C10FA2C
:1008A8000CF320FA02F018BF40F001004FEAC12310
:1008B8004FEAD32303FA0CFC40EA0C0023FA02F3B4
:1008C8004FEA4303CCE77FEA625307D150EA01338A
:1008D8001EBF4FF0FE4040F44000704701F000405A
:1008E80040F0FE4040F40000704700BF80F0004038
:1008F80002E000BF81F0004142001FBF5FEA4103F0
:1009080092EA030F7FEA226C7FEA236C6AD04FEAEF
:100918001262D2EB1363C1BFD21841404840414034
:10092800B8BF5B42192B88BF704710F0004F40F4E6
:10093800000020F07F4018BF404211F0004F41F402
:10094800000121F07F4118BF494292EA030F3FD0CE
:10095800A2F1010241FA03FC10EB0C00C3F12003E1
:1009680001FA03F100F0004302D5494260EB400070
:10097800B0F5000F13D3B0F1807F06D340084FEADB
:10098800310102F10102FE2A51D2B1F1004F40EBD0
:10099800C25008BF20F0010040EA03007047490038
:1009A80040EB0000013A28BFB0F5000FEDD2B0FAD5
:1009B80080FCACF1080CB2EB0C0200FA0CF0AABFF8
:1009C80000EBC25052421843BCBFD0401843704796
:1009D80092F0000F81F4000106BF80F4000001329C
:1009E800013BB5E74FEA41037FEA226C18BF7FEA73
:1009F800236C21D092EA030F04D092F0000F08BFB5
:100A08000846704790EA010F1CBF0020704712F09B
:100A18007F4F04D1400028BF40F00040704712F1DA
:100A280000723CBF00F50000704700F0004343F03F
:100A3800FE4040F4000070477FEA226216BF084675
:100A48007FEA23630146420206BF5FEA412390EA38
:100A5800010F40F4800070474FF0000304E000BF2E
:100A680010F0004348BF40425FEA000C08BF7047DF
:100A780043F0964301464FF000001CE050EA0102A3
:100A880008BF70474FF000030AE000BF50EA0102B8
:100A980008BF704711F0004302D5404261EB4101A5
:100AA8005FEA010C02BF84460146002043F0B643CA
:100AB80008BFA3F18053A3F50003BCFA8CF2083AEF
:100AC800A3EBC25310DB01FA02FC634400FA02FCF8
:100AD800C2F12002BCF1004F20FA02F243EB0200FF
:100AE80008BF20F00100704702F1200201FA02FC61
:100AF800C2F1200250EA4C0021FA02F243EB020054
:100B080008BF20EADC70704780EA010C1CF0030F74
:100B180037D110F0030C20F0030021F0030150F846
:100B2800042B08BF51F8043B0ED08CF0030C6FF077
:100B38007F434FEACC0C23FA0CFC51F8043B42EA01
:100B48000C0243EA0C0300BFA2F1013C9A4201BF28
:100B58002CEA020C1CF0803F50F8042B51F8043B9F
:100B6800F2D04FEA02604FEA1222012828BFB0EB08
:100B7800036F08BF1B0AF4D003F0FF03000EC01A6E
:100B8800704710F0030F0AD010F8012B11F8013B41
:100B9800012A28BF9A42F4D0A2EB030070474DF80F
:100BA800045D50F8042B01F0030521F0030151F80E
:100BB800043B022D26D04DD822F07F45B5EB132FEC
:100BC800A2F1013C2CEA020C0DD11CF0803C08BFBC
:100BD80051F8043B0AD185EA0205B5EB036F0CD145
:100BE80050F8042BE8E74FEA13235BE03CF07F4C16
:100BF80054D10B784FEA126554E04FEA126503F0BE
:100C0800FF034FE04FEA0245A2F1013C4FEA1545C8
:100C18002CEA020CB5EB134F18D11CF0803C08BF2E
:100C280051F8043B07D185EA0205B5EB034F09D11A
:100C380050F8042BE6E75FEA0C4C2FD10B884FEAFB
:100C480012452FE04FEA03434FEA12454FEA134398
:100C580028E000BF02F0FF05B5EB136FA2F1013CDD
:100C68002CEA020C0DD11CF0803C08BF51F8043B63
:100C78000AD185EA0205B5EB032F0AD150F8042BF7
:100C8800E8E74FEA13630DE012F0FF0F06D051F8C2
:100C9800043B4FEA122523F07F4303E04FF00000A6
:100CA80020BC704705F0FF0203F0FF00012828BFB1
:100CB800904204BF2D0A1B0AF4D0A2EB000020BC0E
:100CC800704700BF844641EA000313F0030349D18B
:100CD800403A23D30B6803604B6843608B6883609A
:100CE800CB68C3600B6903614B6943618B6983619E
:100CF800CB69C3610B6A03624B6A43628B6A836286
:100D0800CB6AC3620B6B03634B6B43638B6B83636D
:100D1800CB6BC36340304031403ADBD230320BD327
:100D28000B6803604B6843608B688360CB68C36063
:100D380010301031103AF3D20C3205D351F8043B7D
:100D480040F8043B043AF9D2043208D0D2071CBF59
:100D580011F8013B00F8013B01D30B880380604682
:100D6800704700BF082A13D38B07B1D010F00303D4
:100D7800AED0C3F10403D21ADB071CBF11F8013B44
:100D880000F8013BA4D331F8023B20F8023B9FE76F
:100D9800043AD9D3013A11F8013B00F8013BF9D2E2
:100DA8000B7803704B7843708B788370604670477C
:100DB80070B54FF0FF0C4CF4E06C1CEA11541DBFE9
:100DC8001CEA135594EA0C0F95EA0C0F00F0DEF8B4
:100DD8002C4481EA030621EA4C5123EA4C5350EA99
:100DE800013518BF52EA033541F4801143F48013EA
:100DF80038D0A0FB02CE4FF00005E1FB02E506F07B
:100E08000042E0FB03E54FF00006E1FB03569CF0CF
:100E1800000F18BF4EF0010EA4F1FF04B6F5007FD5
:100E280064F5407404D25FEA4E0E6D4146EB060647
:100E380042EAC62141EA55514FEAC52040EA5E50D0
:100E48004FEACE2EB4F1FD0C88BFBCF5E06F1ED87A
:100E5800BEF1004F08BF5FEA500E50F1000041EBB1
:100E6800045170BD06F0004646EA010140EA02005E
:100E780081EA0301B4EB5C04C2BFD4EB0C0541EA80
:100E8800045170BD41F480114FF0000E013C00F395
:100E9800AB8014F1360FDEBF002001F0004170BDB9
:100EA800C4F10004203C35DA0C341BDC04F11404D2
:100EB800C4F1200500FA05F320FA04F001FA05F25E
:100EC80040EA020001F0004221F0004110EBD3702B
:100ED80021FA04F642EB06015EEA430E08BF20EA57
:100EE800D37070BDC4F10C04C4F1200500FA04F3FA
:100EF80020FA05F001FA04F240EA020001F000418C
:100F080010EBD37041F100015EEA430E08BF20EAFE
:100F1800D37070BDC4F1200500FA05F24EEA020E46
:100F280020FA04F301FA05F243EA020321FA04F075
:100F380001F0004121FA04F220EA020000EBD3702C
:100F48005EEA430E08BF20EAD37070BD94F0000F2C
:100F58000FD101F00046400041EB010111F4801F60
:100F680008BF013CF7D041EA060195F0000F18BF11
:100F7800704703F00046520043EB030313F4801F4D
:100F880008BF013DF7D043EA0603704794EA0C0F07
:100F98000CEA135518BF95EA0C0F0CD050EA41061D
:100FA80018BF52EA4306D1D181EA030101F000419A
:100FB8004FF0000070BD50EA410606BF10461946C2
:100FC80052EA430619D094EA0C0F02D150EA0136CE
:100FD80013D195EA0C0F05D152EA03361CBF10460F
:100FE80019460AD181EA030101F0004141F0FE41AE
:100FF80041F470014FF0000070BD41F0FE4141F432
:10100800780170BD70B54FF0FF0C4CF4E06C1CEA31
:1010180011541DBF1CEA135594EA0C0F95EA0C0FE6
:1010280000F0A7F8A4EB050481EA030E52EA0335A1
:101038004FEA013100F088804FEA03334FF08055C2
:1010480045EA131343EA12634FEA022245EA1115EF
:1010580045EA10654FEA00260EF000419D4208BFA0
:10106800964244F1FD0404F5407402D25B084FEA4D
:101078003202B61A65EB03055B084FEA32024FF4F9
:1010880080104FF4002CB6EB020E75EB030E22BF56
:10109800B61A754640EA0C005B084FEA3202B6EB16
:1010A800020E75EB030E22BFB61A754640EA5C00C5
:1010B8005B084FEA3202B6EB020E75EB030E22BF55
:1010C800B61A754640EA9C005B084FEA3202B6EB56
:1010D800020E75EB030E22BFB61A754640EADC0015
:1010E80055EA060E18D04FEA051545EA16754FEA77
:1010F80006164FEAC30343EA52734FEAC2025FEA95
:101108001C1CC0D111F4801F0BD141EA00014FF023
:1011180000004FF0004CB6E711F4801F04BF0143F4
:101128000020B4F1FD0C88BFBCF5E06F3FF6AFAE10
:10113800B5EB030C04BFB6EB020C5FEA500C50F1A0
:10114800000041EB045170BD0EF0004E4EEA113123
:1011580014EB5C04C2BFD4EB0C0541EA045170BD2A
:1011680041F480114FF0000E013C90E645EA060E6E
:101178008DE60CEA135594EA0C0F08BF95EA0C0F9C
:101188003FF43BAF94EA0C0F0AD150EA01347FF4E4
:1011980034AF95EA0C0F7FF425AF104619462CE7BB
:1011A80095EA0C0F06D152EA03353FF4FDAE10461E
:1011B800194622E750EA410618BF52EA43067FF46F
:1011C800C5AE50EA41047FF40DAF52EA43057FF4FF
:1011D800EBAE12E74A0011D212F5001211D20DD56A
:1011E8006FF47873B3EB62520ED44FEAC12343F025
:1011F800004343EA505323FA02F070474FF00000CF
:10120800704750EA013002D14FF0FF3070474FF07D
:101218000000704753B94AB9002908BF00281CBF0D
:101228004FF0FF314FF0FF3000F00CB8ADF1080C73
:101238006DE904CE18F020FDDDF804E0DDE90223B5
:1012480004B07047704700BF0348044B834202D084
:10125800034B03B118477047EC070020EC07002048
:10126800000000000548064B1B1AD90F01EBA3012B
:10127800491002D0034B03B118477047EC07002010
:10128800EC0700200000000010B5064C237843B995
:10129800FFF7DAFF044B13B10448AFF300800123D2
:1012A800237010BDEC07002000000000349F0108E7
:1012B80008B5054B1BB105490548AFF30080BDE8EB
:1012C8000840FFF7CFBF00BF00000000F007002074
:1012D800349F010800B583B00A4B5A6942F00102F5
:1012E8005A615B6903F001030193019B00221146D7
:1012F8000F2002F097FF0F2002F0A4FF03B05DF863
:1013080004FB00BF0010024030B587B000230293F1
:10131800039304930593134B1B680BB107B030BDBF
:10132800104B01221A60104B5A6942F480725A61BC
:101338005B6903F480730193019B4FF680730293FA
:10134800022503950324059402A9084803F086FAA8
:101358004CF6B37302930395059402A9044803F06D
:101368007DFADBE708080020001002400018014061
:101378000014014010B588B0002201920292039235
:10138800049205920692079216484FF02043036094
:1013980003F5827343608260C2600261102141617B
:1013A8008261C261026242624FF480538362C26208
:1013B8000263426382630F2301930293FF24039421
:1013C800049305911123069301A906F056F830B944
:1013D800054AD36943F48063D36108B010BD00F0B7
:1013E800FFF8F5E70C0800200000014008B5FFF7FA
:1013F8008BFF08BD2DE9F0478AB0002406940794B6
:1014080008940994474B9A6942F010029A619A69C4
:1014180002F010020192019A9A6942F004029A615C
:101428009A6902F004020292029A9A6942F008024A
:101438009A619A6902F008020392039A9A6942F043
:1014480040029A619A6902F040020492049A9A69E9
:1014580042F020029A619B6903F020030593059BE3
:10146800DFF8C49001222021484603F01AFBDFF878
:10147800BC8001220421404603F013FB2C4F224676
:101488004FF40041384603F00CFB01260696DFF8BE
:10149800A4A0CDF81CA00225089506A9384603F09B
:1014A800DDF912230693CDF81CA0089606A9384644
:1014B80003F0D4F92023069307960894099506A902
:1014C800484603F0CBF90423069307960894099538
:1014D80006A9404603F0C2F94FF400430693079665
:1014E8000894099506A9384603F0B8F92246294612
:1014F800062002F097FE062002F0A4FE22462946A6
:10150800072002F08FFE072002F09CFE22462946A3
:101518000A2002F087FE0A2002F094FE0AB0BDE815
:10152800F08700BF0010024000100140000C01408D
:10153800000801400000111038B502680C4B9A42AF
:1015480000D038BD0B4C204602F09AFA78252A467E
:10155800002120460DF09AFE2A462146064806F04C
:1015680087FE064B1A68136823F004031360E8E744
:10157800003801405C080020A40A0020180A002056
:1015880010B50446002200F10C0105F099F9134B3F
:10159800DB78E27B934204D1104B5978637B994204
:1015A80015D00221204605F073FA627B03212046FC
:1015B80005F06EFAA27B0421204605F069FAE27B69
:1015C800064BDA70627B5A70A27B9A7010BD034B8F
:1015D8009978A37B9942E4D1F8E700BF540800202A
:1015E80072B6FEE700B597B0282200210CA80DF0CE
:1015F8004DFE00230793089309930A930B930193D5
:101608000293039304930593069309230C934FF4D1
:1016180080330D9301221092129202221392149396
:101628004FF4E01315930CA804F09EFAD8B90F23D1
:10163800079302210891002309934FF480620A92CC
:101648000B9307A804F0C2FC78B9112301934FF457
:10165800007302930023069301A804F093FD30B9A8
:1016680017B05DF804FBFFF7BBFFFFF7B9FFFFF703
:10167800B7FF000008B502F057FDFFF7B3FF184C9D
:10168800204600F035F8FFF7B5FEFFF723FEFFF719
:1016980071FE00F09BFA00F0F1FA00F031F900F069
:1016A80007FB08F07DF90BF013FC00F091F800F04F
:1016B8007BF900F08FFE78220A49204606F0D8FD13
:1016C800094B1A68136823F00403136007480DF0E8
:1016D800EDFB02F0ADFA02F009FC02F059FBFCE761
:1016E800A40A00205C080020180A0020509F010866
:1016F80008B5054B1860054B1868002302221946E7
:1017080080680DF0DBFB08BDD8080020C00600206B
:10171800022801D80120704708B50EF0D5F8092332
:101728000360002008BD000010B5013801280AD860
:1017380014464FF0FF3392B20748006806F02CFABF
:1017480040B9204610BD0EF0BFF8092303604FF0E2
:10175800FF30F7E70520F5E7D8080020022801D870
:101768000020704708B50EF0AFF8092303604FF06A
:10177800FF3008BD08B50EF0A7F8092303604FF045
:10178800FF3008BD08B548B94FF0FF3301220848BB
:10179800006806F060FA40B9012008BD0EF094F820
:1017A800092303604FF0FF30F7E70520F5E700BF96
:1017B800D808002008B5022804D84FF400534B601D
:1017C800002008BD0EF080F809230360F8E7000048
:1017D80010B582B00023ADF804308DF806300093C0
:1017E8002D482E4B03604FF0FF3343604FF4807356
:1017F800836005F0D1F878BB27480268136843F086
:1018080001031360012105F04BF941F2342398429A
:1018180025D000228DF804208DF805208DF80620AB
:1018280001A91D4804F0FBFE78BB01238DF80030A8
:101838008DF801308DF8023000228DF803206946BA
:10184800154804F0D3FF18BB41F234220121124895
:1018580005F01EF902B010BDFFF7C2FECCE70E4C32
:101868000221204605F01CF9E0730321204605F00B
:1018780017F960730421204605F012F9A0730022BD
:1018880001A9204604F02CFFE4E7FFF7A9FECCE706
:10189800FFF7A6FED8E700BFDC08002000280040BC
:1018A8000268144B9A4200D0704700B583B004F028
:1018B8003FF9114BDA6942F00062DA61DB6903F043
:1018C80000630193019B0D4B0122C3F83C240022C5
:1018D8000321084602F0A6FC032002F0B3FC002214
:1018E8000321292002F09EFC292002F0ABFC03B062
:1018F8005DF804FB0028004000100240000042424E
:10190800054B064A1A6000225A609A60DA601A612A
:101918005A6104229A617047F00800200080014053
:1019280030B589B0002304930593069307930268A2
:101938001A4B9A4201D009B030BD03F510435A69D9
:1019480042F480625A615A6902F480620192019AF3
:101958009A6942F010029A619A6902F010020292A2
:10196800029A9A6942F020029A619B6903F0200367
:101978000393039B4FF4885304930225059503248E
:10198800079404A9064802F069FF04230493059507
:10199800079404A9034802F061FFCCE700800140E6
:1019A800001001400014014008B50E480E4B0360BA
:1019B8004FF48273436000238360C3600361436113
:1019C8004FF4007282610822C2610362436283623B
:1019D8000A23C36205F0F6FC00B908BDFFF700FE54
:1019E800FBE700BF740900200030014010B586B045
:1019F800002302930393049305930268164B9A42BB
:101A080001D006B010BD03F560439A6942F48052D4
:101A18009A619A6902F480520092009A9A6942F097
:101A280004029A619B6903F004030193019BA023BC
:101A380002930223039303230593084C02A920462B
:101A480002F00CFF4023029300230393049302A99E
:101A5800204602F003FFD4E70030014000080140AF
:101A680000B583B0124B9A6942F001029A619A69F3
:101A780002F001020092009ADA6942F08052DA61BB
:101A8800DB6903F080530193019B00221146052076
:101A980002F0C8FB052002F0D5FB064A536823F084
:101AA800E06343F00073536003B05DF804FB00BFCC
:101AB8000010024000000140FEE7FEE7FEE7FEE7F7
:101AC800FEE770477047704708B502F03FFB08BD56
:101AD80008B5024804F0B9FF08BD00BFDC080020C3
:101AE800704708B5012002F0E3FF08BD08B50220E1
:101AF80002F0DEFF08BD08B5102002F0D9FF08BDCE
:101B080008B5024802F034FD08BD00BF180A0020DD
:101B180008B5024803F0CEFD08BD00BFE41B002055
:101B280008B5024805F00DFD08BD00BFD00900202A
:101B380008B5024806F0ACF908BD00BFA40A0020A9
:101B480008B5024806F0A4F908BD00BF5C0A0020E9
:101B580008B5024804F0E8FE08BD00BFDC08002014
:101B68000120704708B50DF0AFFE162303604FF053
:101B7800FF3008BD08B54FF0FF31FFF7F3FFFEE770
:101B880010B503460C4A0D490D48006840B10C4891
:101B980000680344521A934206D8094A136010BDDC
:101BA8000748084C0460F2E70DF08EFE0C23036032
:101BB8004FF0FF30F3E700BF0000012000040000F1
:101BC800CC090020E82100207047000000B587B04C
:101BD80000230293039304930593009301931548FC
:101BE800154A026047224260836040F2E732C260D1
:101BF8000361836105F0AEFD90B94FF48053029301
:101C080002A90C4805F0DEFD68B900230093019392
:101C18006946084805F056FE40B907B05DF804FB70
:101C2800FFF7DEFCE9E7FFF7DBFCEEE7FFF7D8FCA0
:101C3800F3E700BFD00900200008004002680E4BFF
:101C48009A4200D0704700B583B003F50233DA69D1
:101C580042F00402DA61DB6903F004030193019B9B
:101C6800002201211E2002F0DDFA1E2002F0EAFA0D
:101C780003B05DF804FB00BF0008004008B50A483F
:101C88000A4B03604FF4E133436000238360C36071
:101C980003610C2242618361C36105F04DFF00B905
:101CA80008BDFFF79DFCFBE7A40A002000380140AF
:101CB80008B50A480A4B03604FF4E1334360002338
:101CC8008360C36003610C2242618361C36105F0D4
:101CD80033FF00B908BDFFF783FCFBE75C0A00206F
:101CE8000048004070B588B000230493059306931C
:101CF80007930368404A934204D0404A934248D02D
:101D080008B070BD04463E4B9A6942F480429A611D
:101D18009A6902F480420092009A9A6942F0040299
:101D28009A619B6903F004030193019B4FF40073CC
:101D380004930223059303230793324E04A93046E4
:101D480002F08CFD4FF480630493002505950695F9
:101D580004A9304602F082FD2B482C4B03604560F5
:101D680085608023C360056145618561C56102F0B6
:101D7800A1FA58B9244BE3635C62002202212520B2
:101D880002F050FA252002F05DFAB9E7FFF728FCC7
:101D9800F0E71B4BDA6942F48022DA61DA6902F46F
:101DA80080220292029A9A6942F008029A619B691B
:101DB80003F008030393039B4FF480630493022307
:101DC800059303250795124E04A9304602F046FDF7
:101DD8004FF40063049300240594069404A9304644
:101DE80002F03CFD22462946272002F01BFA272054
:101DF80002F028FA84E700BF00380140004800409C
:101E08000010024000080140180A00205800024053
:101E1800000C0140034B044A1A60044B023A1A6052
:101E2800704700BF0010002000000260FC0F002077
:101E38000B4B2A225A812B229A812C221A810022AA
:101E48009A71F0221A804FF4A0725A80054B1B68D1
:101E580036221A80044B1B6808221A80704700BF7C
:101E6800EC0F0020FC0F00200010002070B5174E6A
:101E78003468174DB5F80AC0A4F800C0154C4FEAED
:101E8800102CD4F800E0AEF800C0C0B2D4F800C0FE
:101E9800ACF8000020684FEA122CA0F800C02068B7
:101EA800D2B202803268A88910802268080A10809D
:101EB8002268C9B211802268190A11802268DBB22F
:101EC800138033682A891A8070BD00BFFC0F002078
:101ED800EC0F00200010002010B504460A4B1A88A9
:101EE8005B88013B013A9BB292B200210846FFF79A
:101EF800BDFF002303E0054A126814800133B3F5DF
:101F0800963FF8D310BD00BFEC0F00200010002052
:101F18000020704700207047002070472DE9F843E3
:101F28008046894616461F46BDF82050BDF8244015
:101F38001EE0194A12681580013B002B08DB41FAA4
:101F480003F212F0010FF4D0134A12681480F3E779
:101F580002301F2806DC335C3218517841EA03212D
:101F68000F23EAE708F110082036B8F1E00F11DC7A
:101F78003B46013FBFB26BB11FFA88F01FFA89F1E7
:101F880001F10F0300F10F029BB292B2FFF76EFF4F
:101F98000020DEE7BDE8F883001000202DE9F843B3
:101FA8008046894616461F46BDF82050BDF8244095
:101FB8001AE0174A12681580013B002B08DB41FA2A
:101FC80003F212F0010FF4D0114A12681480F3E7FB
:101FD8000130472802DC315C0723EEE708F11808D6
:101FE8004836B8F1D80F11DC3B46013FBFB26BB1A0
:101FF8001FFA88F01FFA89F101F1170300F117029F
:102008009BB292B2FFF732FF0020E2E7BDE8F88307
:10201800001000202DE9F8438046894616461F46E1
:10202800BDF82050BDF824401AE0174A1268158000
:10203800013B002B08DB41FA03F212F0010FF4D048
:10204800114A12681480F3E701307F2802DC315C02
:102058000723EEE708F120088036B8F1D00F11DC2D
:102068003B46013FBFB26BB11FFA88F01FFA89F1F6
:1020780001F11F0300F11F029BB292B2FFF7F6FEB7
:102088000020E2E7BDE8F883001000202DE9F047C2
:1020980007468A4690461D46BDF8206010460DF05A
:1020A80057FC5FFA80F900242DE0B8B21FFA8AF1D4
:1020B800CB1D421D9BB292B2FFF7D8FE18F8040060
:1020C8002038C000002111E0144B1B681D800CF162
:1020D800FF3CBCF1010F08DD42FA0CF313F0010FCD
:1020E800F2D00E4B1B681E80F1E70131072905DC91
:1020F80043180B4AD25C4FF0070CEAE70637E92F82
:102108000ADC0134E4B24C4506D218F90430002B3D
:10211800CBDA0134E4B2F1E7BDE8F0870010002023
:102128001CD601082DE9F04F83B007468A46904631
:102138001C46BDF8305010460DF00AFC5FFA80F9D5
:10214800002633E0B8B21FFA8AF101F10F03C21D6D
:102158009BB292B2FFF78AFE18F8060020380001F9
:10216800002116E0234B1B681C800CF1010C1FFAA0
:102178008CFCBCF1070F0AD8CCF1070342FA03F331
:1021880013F0010FEED01B4B1B681D80EDE70131EA
:1021980089B20F2905D84318174AD25C4FF0000CB2
:1021A800E7E708370136F6B2E82F20DC4E451ED2A5
:1021B80008EB060118F90630002BC3DA14220F4881
:1021C800FFF7A6FE834610B90236F6B2ECE7019592
:1021D8000094C0F34F13094A51463846FFF79EFE54
:1021E80007EB5B0706EB1B1B5FFA8BF6DCE703B01C
:1021F800BDE8F08F001000202CD00108EC0A002068
:102208002DE9F04F85B08046039191461C46BDF8F4
:10221800385010460DF09CFB5FFA80FB002637E033
:102228001FFA88F0BDF80C1001F1170300F10B023A
:102238009BB292B2FFF71AFE19F80630203B03EB67
:102248004303284F07EB0317002011E0264A1268C2
:102258001480013B9BB2032B08D941FA03F212F018
:10226800010FF3D0204A12681580F2E7023080B2DD
:102278002F2806D83B5C3A18517841EA03210F23EE
:10228800E9E708F10C080136F6B2B8F1E40F26DCEC
:102298005E4524D209EB060119F90630002BBFDA96
:1022A80014221248FFF736FE074610B90236F6B276
:1022B800EBE70F4BA3FB003A01950094CAF30F1309
:1022C8000A4A03994046FFF769FE0A4BA3FB073702
:1022D80008EB570806EBDA0A5FFA8AF6D5E705B085
:1022E800BDE8F08F8CBE010800100020EC0A002029
:1022F800398EE338ABAAAAAA2DE9F04F83B08046FD
:102308008B4617461C46BDF8305010460DF020FB92
:102318005FFA80F9002634E01FFA88F01FFA8BF183
:1023280001F11F0300F10F029BB292B2FFF79EFD6D
:10233800BB5D203B244A02EB831C00200FE0234AAC
:1023480012681480013B002B08DB41FA03F212F0FB
:10235800010FF4D01D4A12681580F3E702303F28B8
:1023680008DC1CF800300CEB0002517841EA03212C
:102378000F23E8E708F110080136F6B2B8F1E40FC8
:102388001EDC4E451CD2B919BB57002BC4DA1422E7
:102398000F48FFF7C1FD824610B90236F6B2EDE7E5
:1023A80001950094C0F3CF13094A59464046FFF7F8
:1023B80031FE08EB9A0806EB9A1A5FFA8AF6DDE70F
:1023C80003B0BDE8F08F00BF0CA701080010002083
:1023D800EC0A00202DE9F04F83B0FFF71BFDA64D56
:1023E8002B68CF221A80A54B1A68002414801A681B
:1023F800C9211180196830220A802968ED200880D7
:102408001968642008801968032008801968122058
:1024180008801968812008802968E82008801968E0
:1024280085200880196810270F8019687A2008808D
:102438002968CB20088019683920088019682C2061
:10244800088019680C8019683420088019680220EF
:1024580008802968F720088019684FF02009A1F83A
:1024680000902968EA20088019680C8019680C8097
:102478002968C020088019681B2008802968C120A5
:10248800088019680C802968C520088019680A80A6
:1024980019680A802A68C72111801A68B721118033
:1024A8002A684FF03608A2F800801A6808261680B5
:1024B8002A683A2111801A68552111802A68B121A9
:1024C80011801A6814801A681A2111802A68B621A6
:1024D80011801A680A2111801A68A22010802A68BF
:1024E800F22010801A6814802A68262010801A6842
:1024F8004FF0010EA2F800E02A68E020108018686A
:102508000F22028018684FF02A0AA0F800A0186865
:102518004FF0280CA0F800C01868068018684FF023
:102528000E0CA0F800C01868068018684FF0540C0C
:10253800A0F800C018684FF0A90CA0F800C01868EF
:102548004FF0430CA0F800C01868018019680A8091
:1025580019680C8019680C8019680C8019680C803F
:102568002968E120088019680C80196815200880FE
:1025780019681720088019680720088019684FF023
:10258800110BA1F800B019680620088019684FF0EF
:102598002B0CA1F800C019685620088019683C2047
:1025A800088019680520088019680F8019680A8052
:1025B80018683F21018018680180186802802A681D
:1025C800A2F800C01A6814801A6814801A68A2F861
:1025D80000E01A6811802A68A2F800A01A6814801E
:1025E8001A6814801A6814801B68EF221A802B68F6
:1025F800A3F800B0782001F0BBFD2B6829221A80CF
:10260800FFF716FC1E4AD36843F40043D3604FF427
:102618007840FFF761FCC82001F0AAFD4FF4FC6088
:10262800FFF75AFCC82001F0A3FD1F20FFF754FC58
:10263800C82001F09DFD4FF6FF70FFF74DFCC82044
:1026480001F096FD4FF4784500954FF6FF730D4A5B
:1026580021462046FFF766FDDFF82CA000954FF6CF
:10266800FF7352462146A020FFF710FD4FF6FF7575
:1026780000952346524609E0FC0F00200010002078
:1026880000080140649F01087C9F01083146A02092
:10269800FFF7FCFC4FF4FC6300932B460C4A3946C9
:1026A8002046FFF73FFD1F2300932B46094A494662
:1026B8002046FFF7A5FD4BF6404300932B46064AFC
:1026C80041462046FFF718FE03B0BDE8F08F00BF73
:1026D8008C9F0108A49F0108BC9F0108FFF774FAAA
:1026E8000B480C490C4A002302E0D458C450043368
:1026F800C4188C42F9D3094A094C002301E013603D
:102708000432A242FBD30DF0E5F8FEF7B3FF7047A1
:1027180000000020EC070020A4480208EC07002075
:10272800E8210020FEE7000020B3844621B3884258
:1027380024D000B50DE086460B78124AD25C02F030
:102748000302012A10D09E4510D1C8B10CF1010C2A
:1027580001319CF800000B4B1B5C03F00303012BB9
:10276800E9D100F1200EE7E72033ECE7AEEB0300F8
:102778005DF804FB01207047012070470020704776
:102788000020F5E761DA01082E2070472DE9F84F9F
:1027980082468B4614461D4621F00049164623F012
:1027A80000473B464946FEF709F808B156464F46EA
:1027B80022462B4650465946FDF7CAFD044621F0ED
:1027C80000450022084B30463946FEF7F1FA02462A
:1027D8000B46012620462946FDF7DCFF00B90026F6
:1027E8003046BDE8F88F00BF0000B03C84460022A8
:1027F80010460BE0A1F14103DBB2052B12D80B18F0
:10280800A3F13700022A00D800010132032A12D8A6
:102818001CF80210A1F13003DBB2092BEAD80844F6
:102828003038EFE7A1F16103DBB2052B04D80B18B0
:10283800A3F15700E6E7704700207047F8B50B1A78
:10284800052B61DD06460F4615460230FFF7CEFF21
:102858000446A0F55C43B3F5806F57D3A0F5584301
:10286800B3F5806F1CD2B31DFF1A052F50DDB37965
:102878005C2B4FD1F379752B4ED106F10800FFF789
:10288800B5FFA0F55C43B3F5806F47D2254B03EA4B
:102898008423C0F30900034303F580340C2002E0CD
:1028A8007F280CD90620B4F5006F0ED3B4F5803F0D
:1028B8000ED3B4F5881F33D2F027042602E0062091
:1028C80000270126731EDBB20EE0C0270226F9E7B7
:1028D800E0270326F6E704F03F012A6841F080016B
:1028E800D154A409013BDBB2002BF4D1012E06D947
:1028F8002B6827431F702B6833442B6005E02B6837
:1029080004F07F041C70F6E70020F8BD0020FCE707
:102918000020FAE70020F8E70020F6E70020F4E7B7
:102928000020F2E700FC0F002DE9F04182B080465C
:102938000E460F688B685D1C3D4400220192F81812
:10294800FB5C222B43D12C46944600E00134E11B6A
:10295800726891420BD22378222B08D05C2BF5D1D8
:102968000134E31B934232D20CF1010CEEE79142A1
:102978002DD22378222B2AD1201AA0EB0C00336900
:1029880001309847074610B3019030E0631B002BD5
:102998001ADD6B78752B17D85C2B11D35C3B192B80
:1029A80012D8DFE803F04C11111111111D1111118A
:1029B8003011111111111111371111113E11455317
:1029C800222B3CD02F2B3AD0736938469847002DDC
:1029D80054D03368ED1AB560002002B0BDE8F0812C
:1029E800019B5A1C019208221A7002231D44A54219
:1029F80035D22B785C2BC9D0019B5A1C019215F853
:102A0800012B1A70F3E7019B5A1C01920C221A70D1
:102A18000223EBE7019B5A1C01920A221A70022337
:102A2800E4E7019B5A1C01920D221A700223DDE78C
:102A3800019B5A1C019209221A700223D6E7019BB6
:102A48005A1C01926A781A700223CFE701AA21461C
:102A58002846FFF7F3FE03460028C7D1B4E7019BD9
:102A680000221A701023C8F80C30C8F810703368A8
:102A7800E41AB4600134B4600120AEE70020ACE78A
:102A88000246D0B110B40468ACB183684068834290
:102A980002D30AE0013393609368984202D9E15C5B
:102AA8002029F7D99368984202D0104610BC704785
:102AB800013B9360F9E72246F7E7704701604860F9
:102AC8007047A1B138B504460D4690B1814212D085
:102AD80083683BB1586880B1FFF7F0FFA3685D6079
:102AE800012038BD816049600B600120F9E70020B2
:102AF80070470020F5E70020F3E70120F1E7704771
:102B080050B138B50546006828B1AC6820440CF0CF
:102B18001FFF0444AC6038BD704770B5064670B1FD
:102B28000D460CF015FF441C2B68204698470546B7
:102B380018B122463146FEF7C5F8284670BD05464D
:102B4800FBE768B32DE9F0410D4614461E460746DB
:102B580041B34AB3904229D0069BBBB10846FFF760
:102B6800CEFF8046E56845F40075E36813F4007FFE
:102B780003D1206A08B173689847C4F82080E560DB
:102B880021463846FFF79DFFBDE8F08131462846CB
:102B9800FFF7C3FF804658B1E56825F40075E4E700
:102BA800002070470020EFE70020EDE70020EBE76A
:102BB8000698E9E770B50546002846D0066836B39A
:102BC800436813B18268934241D9002941DBAA685E
:102BD800114401318B420AD22B69002B3BD1B1F150
:102BE800804F08D3002904DB6FF0004404E016444A
:102BF8000DE000260BE04C002B6A8BB121463046D5
:102C08009847064628B16C602E60AB681E44304673
:102C180070BDEB692868984700236B602B60F6E766
:102C2800AB6920469847064640B1AA680132296830
:102C3800FEF748F8EB6928689847E4E7EB692868E5
:102C4800984700236B602B60E1E70646DFE7002624
:102C5800DDE70026DBE70026D9E710B50368282062
:102C68009847044618B1282200210CF00FFB204693
:102C780010BD000038B5044678B1006878B1A56881
:102C88007DB92B1D6268934207D203220649284466
:102C98000CF04CFB08B90335A560204638BD044646
:102CA800FBE70024F9E700BFD49F010800000000FB
:102CB8002DE9F04393B005460C4600231193FFF726
:102CC80063FD002C65D02368002B64D0002330E01E
:102CD800652A28D048336B44002203F8442C0DF1B0
:102CE800040911A948460BF085FF06460F46DDF892
:102CF8004480C84551D0C5E9066729A3D3E9002314
:102D0800FDF752FD002833D06FF000436B610823B4
:102D1800EB60A36801AAA8EB02084344A360012062
:102D280013B0BDE8F08303F14801694401F8442C6D
:102D380001333E2BCED8A2681A4461688A42C9D2B0
:102D480021688A5C452AC3D82B2AC3D3A2F12B0653
:102D5800F6B20121B140144E0E40002EE3D111F01D
:102D6800080FB7D003F148026A4402F8440CDFE7C1
:102D780000220E4B30463946FDF70CFD18B14FF0D6
:102D880000436B61C3E730463946FDF737FD68619C
:102D9800BDE70020C4E70020C2E70020C0E700BF6D
:102DA8000000C0FFFFFFDF41E57F00040000E0C135
:102DB800002900F09480F8B50546084615B12A4662
:102DC800002614E00321FFF7F5FE002800F08980B3
:102DD800464A118892780180827001207EE05C2B3F
:102DE80003D01F2B02D8053600E0013601321378D4
:102DF80063B1222BF3D8082BF3D3A3F10804E4B270
:102E08003B49E14011F0010FEFD1EAE7521B941959
:102E1800E11CFFF7CFFE0746002864D026B106461E
:102E2800222306F8013B30E0222600F8016B2246F7
:102E38002946FDF747FF631CFE54023400233B5527
:102E480001204BE030465C2300F8013B2A78222A17
:102E580015D8082A36D3A2F108031A2B32D8DFE88E
:102E680003F0222E2831252B3131313131313131E6
:102E78003131313131313131313131311F005C2A59
:102E880020D15C2373700135461C2B78FBB11F2BB6
:102E9800D8D9222BD6D05C2BD4D033703046F2E769
:102EA80022237370EFE762237370ECE76623737075
:102EB800E9E76E237370E6E772237370E3E7742320
:102EC8007370E0E70B490CF0CBF8701DDBE7631C6F
:102ED8002222FA54023400233B550120F8BD002079
:102EE80070470020FAE70020F8E700BFD89F0108E4
:102EF80037000004DC9F010808B50069FFF758FF98
:102F080008BD00002DE9F0478AB082460C46D0E99A
:102F18000667002303930493059306930793089386
:102F2800ADF82430FFF730FC00220023CDE9002360
:102F3800002C76D0054632463B4630463946FDF7EA
:102F480047FC88B927F000494FF0FF32374B30462D
:102F58004946FDF73DFCB8B94FF0FF32334B3046D8
:102F68004946FDF717FC78B9314B93E80300039005
:102F78008DF810104FF004084646B8F1190F32D9F1
:102F880000200AB0BDE8F087DAF814804046FDF763
:102F98002DFB32463B46FDF7E9FB30B14246254959
:102FA80003A80CF05DF88046E6E732463B46224926
:102FB80003A80CF055F880466A46204903A80CF08F
:102FC80071F8012807D132463B46DDE90001FFF7D9
:102FD800DDFB0028D0D132463B46194903A80CF046
:102FE8003FF88046C8E708F101012046FFF7E2FDF7
:102FF8000146C0B1002302E02E22CA5401339E428A
:1030080008D903F128026A4412F81C2CAA42F3D00A
:10301800CA54F3E70022CA54A3681E44A6600120DC
:10302800AFE70020ADE70020ABE700BFFFFFEF7F71
:10303800E49F0108EC9F0108F09F0108F89F010830
:10304800FC9F010870B500286CD00D460646002983
:103058006AD0047B202C16DC002C67D0631E1F2B43
:1030680066D8DFE803F0364265286565654F656513
:10307800656565656553656565656565656565650A
:10308800656565656557402C48D0802C11D100696D
:10309800002856D00CF05CFC441C21462846FFF75B
:1030A80089FD00284FD022463169FDF70BFE012427
:1030B8003FE000243DE005212846FFF77BFD03465D
:1030C800002838D0214A1068186012791A71012432
:1030D8002FE006212846FFF76DFD034668B31C4A1A
:1030E8001068186092889A8023E005212846FFF727
:1030F80061FD034618B3174A1068186012791A71EF
:10310800012416E0FFF7FEFE044612E0FFF7F4FE86
:1031180004460EE000F06EF804460AE000F0BEF83F
:10312800044606E0002404E0002402E0002400E055
:103138000024204670BD0024FBE70024F9E70024A2
:10314800F7E70024F5E70024F3E700BFE49F010850
:1031580004A001080CA0010870B58AB006460D4607
:1031680014462422002101A80CF090F823684FF49B
:1031780080709847034601904FF48072029206953A
:1031880094E807000AAD05E9070023B101A9304614
:10319800FFF758FF40B9019D1DB16368284698475D
:1031A800002528460AB070BD01A8FFF7A9FCA3684E
:1031B8004BB1039901310198984705460028EAD098
:1031C80000230193EDE723680398013098470546EB
:1031D8000028E0D0039A0132029B9A4228BF1A467F
:1031E8000199FDF76FFD039B0022EA54636801987B
:1031F8009847D6E770B58568002946D00C46012166
:103208002046FFF7D7FC002842D05B220270A36853
:103218000133A360E3680133E36007E0012616E0A9
:1032280000221A70A3683344A3602D68FDB12146BB
:103238002846FFF707FF034640B32046FFF760FC28
:103248002B68002BF1D06369002BE7D00226711C94
:103258002046FFF7AFFCE8B103462C2103F8011B19
:1032680061690029DCD0831C20214170D8E7022144
:103278002046FFF79FFC78B15D2202700022427061
:10328800E368013BE360012300E00023184670BDBA
:103298000023FBE70023F9E70023F7E770B585680B
:1032A800002900F0A3800C464B69A3B10226711CCB
:1032B8002046FFF77FFC002800F09B807B230370EB
:1032C800E3680133E36063690BB10A234370A368C1
:1032D8003344A36022E00126E9E7E1682046FFF7CE
:1032E80069FC0346002800F08680002203E00921DB
:1032F80003F8011B0132E1689142F8D8A368194428
:10330800A16010E001261CE0002637E0002339E028
:1033180000221A70A3683344A3602D68002D44D09E
:103328006369002BD9D12146286AFFF741FD03467E
:1033380000285CD02046FFF7E3FB6369002BE1D04F
:10334800022631462046FFF735FC002855D03A22A0
:10335800027062690AB109224270A3683344A3600B
:1033680021462846FFF76EFE034600283FD0204638
:10337800FFF7C6FB6369002BC6D001262B68002B1C
:10338800C4D001231E44711C2046FFF713FC0346DA
:10339800A8B32A6812B12C2203F8012B6269002A0B
:1033A800B6D00A2203F8012BB2E763698BB1E16852
:1033B80001312046FFF7FEFB034610B362699AB954
:1033C8007D221A7000225A70E368013BE3600123F2
:1033D8000DE00221EDE7092203F8012B0131E26833
:1033E800013A8A42F7D8EBE70021F8E700231846AC
:1033F80070BD0023FBE70023F9E70023F7E700236C
:10340800F5E70023F3E738B50446C8B10D46C9B15E
:1034180084680AB90AE024687CB1216A69B128463F
:10342800FDF772FB0028F6D107E024682CB1216A69
:103438002846FFF779F90028F7D12CB1236A2BB178
:10344800204638BD0C46FBE70024F9E70024F7E7DF
:1034580038B5044616E0E36813F4807F04D1206988
:1034680010B10F4B5B689847E36813F4007F04D1F1
:10347800206A10B10A4B5B689847094B5B68204685
:1034880098472C4654B12568E36813F4807FE2D14D
:10349800A0680028DFD0FFF7DBFFDCE738BD00BFFE
:1034A80004000020CB68B3F57A7F80F08B802DE98B
:1034B800F04106460C460133CB60002900F08480B9
:1034C8008B684A68934280F081800A68D25C7B2AC4
:1034D80002D00020BDE8F08101338B600846FFF779
:1034E800CFFAA3686268934203D22268D35C7D2B2B
:1034F80059D0A3686268934204D2013BA3600025B7
:103508002F4634E0013BA3600020E3E70746A368A9
:103518000133A3602046FFF7B3FA21462846FFF798
:1035280003FA002839D02046FFF7AAFA2B692B6244
:1035380000232B61A368626893422ED22268D25C72
:103548003A2A2AD10133A3602046FFF799FA214687
:10355800284600F03FF800B32046FFF791FAA36829
:103568006268934211D22268D35C2C2B0DD1A846F5
:1035780004F11000FFF771FB054670B1002FC5D0AC
:10358800C8F80000C0F80480C1E7A36862689342E5
:1035980003D22268D35C7D2B07D0CFB13846FFF722
:1035A80057FF002096E700252F46E368013BE360BC
:1035B80007B17D604023F360B760A3680133A3605F
:1035C800012087E700207047002083E7002081E77B
:1035D80000207FE700296AD02DE9F84380460D4690
:1035E8000F68002F65D08C6804F104094E68B14556
:1035F80005D80422314938190BF098FE50B3631DE1
:103608009E4205D305222E4938190BF08FFE48B388
:10361800B14505D804222B4938190BF087FE40B371
:10362800B44202D23B5D222B2DD0B44206D23B5D80
:103638002D2B2DD0303BDBB2092B29D9B44202D235
:103648003B5D5B2B29D0B44236D23B5D7B2B29D026
:1036580000202FE00423C8F80C30AB680433AB60BB
:10366800012027E00120C8F80C00AA680532AA60EA
:1036780020E00223C8F80C300120C8F81400AA681A
:103688000432AA6016E029464046FFF74DF911E0DA
:1036980029464046FFF70CFB0CE02946404600F05F
:1036A80013F807E029464046FFF7FCFE02E0002039
:1036B80070470020BDE8F8830020FBE7E49F01087D
:1036C80004A001080CA00108CB68B3F57A7F6DD27D
:1036D8002DE9F04106460C460133CB600A688B6839
:1036E800D25C5B2A02D00020BDE8F08101338B60F8
:1036F8000846FFF7C5F984B1A3686268934203D20C
:103708002268D35C5D2B42D0A3686268934204D2DE
:10371800013BA36000252F461CE0A368013BA36082
:103728000020E1E70746A3680133A3602046FFF7BE
:10373800A7F921462846FFF74DFF10B32046FFF7AB
:103748009FF9ACB1A3686268934211D22268D35C36
:103758002C2B0DD1A84604F11000FFF77EFA054680
:1037680078B1002FDED0C8F80000C0F80480DAE78E
:103778003CB1A3686268934203D22268D35C5D2B94
:1037880007D0AFB13846FFF763FE0020ACE700254D
:103798002F46E368013BE36007B17D602023F360B7
:1037A800B760A3680133A36001209DE7002070473C
:1037B800002099E7F0B58BB015461E460024039407
:1037C800049405940694079408940994294B1C6062
:1037D8005C60044600B1B9B9002C49D001940023BB
:1037E8000293059A049B9A423DD2029215B1029B1C
:1037F80023442B601F4B01AA92E8030083E80300CF
:10380800002738460BB0F0BD039004911A4B93E89B
:1038180007000AAF07E907001846FFF71EFA074630
:103828000028D9D003A8FFF725FAFFF729F90146A0
:103838003846FFF7CFFE90B136B9002DE1D0039B93
:10384800059A13442B60DCE703A8FFF719F9059BD9
:10385800049A934203D2039AD35C002BEDD03846E6
:10386800FFF7F6FDB8E7002BC0D0013B0293BDE798
:103878002746C6E7041000200400002070B504465F
:1038880048B10D4616460CF063F833462A46411CEB
:103898002046FFF78FFF70BD08B500221146FFF7DD
:1038A800EDFF08BD08B5024A0121FFF755FC08BD28
:1038B8000400002008B50122FFF7A5FD08BD00009F
:1038C80070B504460D461648FFF7C7F9064670B1AD
:1038D8000823C360C0E906450FA3D3E900232046A7
:1038E8002946FCF761FF20B16FF000437361304651
:1038F80070BD00220B4B20462946FCF74BFF18B140
:103908004FF000437361F2E720462946FCF776FF43
:103918007061ECE7AFF300800000C0FFFFFFDF41FC
:10392800040000200000E0C170B582B005460E46D4
:1039380010461946FFF7C4FF044600230093074BBF
:10394800024631462846FFF7FCF810B1204602B07F
:1039580070BD2046FFF77CFD0024F7E70400002037
:1039680038B504460A48FFF778F9054640B11023F0
:10397800C36007492046FFF7D0F80446286108B11C
:10398800284638BD2846FFF763FD2546F8E700BFFF
:103998000400002070B582B005460E461046FFF7B9
:1039A800DFFF044600230093074B024631462846B2
:1039B800FFF7C7F810B1204602B070BD2046FFF7E8
:1039C80047FD0024F7E700BF0400002008B50348BE
:1039D800FFF743F908B14023C36008BD0400002085
:1039E80028B1007B082814BF002001207047002060
:1039F800704728B1007B102814BF002001207047B1
:103A080000207047C8B130B583B014461D46B1B127
:103A1800BAB1C3B1009313460A460F490BF042FBF3
:103A2800032812D12368013B0B2B10D82B68013BCC
:103A38001E2B0ED8002003B030BDFF207047FF209A
:103A4800F9E7FF20F7E7FF20F5E7FD20F3E7FC2083
:103A5800F1E7FB20EFE700BF14A0010800B583B031
:103A6800009313460A4605490BF01CFB032803D0B4
:103A7800002003B05DF804FB0120FAE720A001084C
:103A880010B588B004463D490BF0FCFD10B13C4B25
:103A980001221A703B4920460BF0F4FD10B1384B57
:103AA80002221A70364B1B78012B09D0344B1B7835
:103AB800022B37D0214634480BF098F908B010BDD6
:103AC80032480BF0F3F932480BF0F0F905AB06AACF
:103AD80007A92046FFF796FF0146F8B9059B069A05
:103AE80007992C480BF082F9079A2B4981FB023180
:103AF800D317C3EB6113642101FB13238DF807303F
:103B08009DF818308DF805309DF814308DF8063082
:103B1800002201A9214802F069FEC7E720480BF0FE
:103B280065F9C3E71F480BF0C1F91F480BF0BEF950
:103B380002AB03AA04A92046FFF790FF014601281B
:103B480003D01A480BF052F9B4E7029B039A049980
:103B580017480BF04BF99DF810308DF800309DF8A0
:103B68000C308DF801309DF808308DF802300022B5
:103B780069460A4802F053FD9CE700BF2CA00108E3
:103B88000C10002034A0010820A301083CA0010863
:103B98005CA0010874A001081F85EB51DC08002017
:103BA80094A00108ACA00108D0A001080CA101084C
:103BB800E4A0010810B50446012804D0022C12D054
:103BC800102C20D010BD0121174800F063FF0128F8
:103BD800F4D10121144800F05DFF0128F9D0134BFE
:103BE80001221A70EAE702210F4800F053FF00286B
:103BF800E6D102210C4800F04DFF0028F9D00B4B0C
:103C080002221A70DCE71021074800F043FF002861
:103C1800D8D11021044800F03DFF0028F9D0034B0B
:103C280003221A70CEE700BF0008014058080020A0
:103C380070B5A0B04FF6FF70FEF74EF92E4B1B780B
:103C4800012B1AD04FF4784400944FF6FF732B4A97
:103C580000210846FEF7D4FA00944FF6FF73284A6D
:103C680000210846FEF7CCFA142000F081FA4FF63E
:103C7800FF70FEF731F920B070BD4FF4FC6400947A
:103C88004FF6FF731F4A00210846FEF7B9FA009461
:103C98004FF6FF731C4A19210020FEF7B1FA1B4E9C
:103CA800706DFCF7D9FE0546B06DFCF7D5FE2946C8
:103CB800FCF796FA4FF06A51FCF792FA4FF06A5106
:103CC800FCF78EFAFCF7A4FC02460B46104902A842
:103CD8000BF0C6F900944FF6FF7302AA31210020B9
:103CE800FEF78EFA00944FF6FF730A4A4921002026
:103CF800FEF786FAB8E700BFD40800206CA10108D7
:103D080080A1010824A1010838A10108F0080020B9
:103D18004CA101085CA1010810B58CB0194C002217
:103D28000BA9204602F0DCFC00220AA9204602F07A
:103D3800C7FD9DF82A3000939DF829309DF82B2067
:103D4800114902A80BF08CF91F2400944FF6FF7359
:103D580002AA00213C20FEF753FA9DF82E3000936A
:103D68009DF82D309DF82C20084902A80BF078F911
:103D780000944FF6FF7302AA19214820FEF740FA73
:103D88000CB010BDDC08002094A10108A8A101080E
:103D980008B5FFF7C1FF08BD30B585B0002203A9FB
:103DA800374802F08DFD102009F0D6FA05469DF837
:103DB8000E3000939DF80D309DF80F2031490BF01F
:103DC8004FF9FFF703FE04462A462F49FFF7E2FDA5
:103DD8002E4B1868FCF71CFC02460B462C49204663
:103DE800FFF7A2FD2B4A2C492046FFF7D3FD2B4AAB
:103DF8002B492046FFF7CEFD2046FFF753FD04462A
:103E08002849294808F025FF08BB28480BF04EF838
:103E180007222749244808F01DFA014658BB2548BF
:103E28000BF044F820460BF093FD024602AB214606
:103E38001D4808F0F6FBB0B11B4808F06EFD284697
:103E480009F092FA204609F08FFA05B030BD1548FE
:103E580008F04FFF18B918480BF028F8D8E71748AA
:103E68000BF024F8D4E716480BF020F82146154843
:103E78000AF0BCFFE0E714480AF0B8FFDFE700BF2C
:103E8800DC08002094A10108B8A101081000002056
:103E9800C0A10108C8A10108D0A10108DCA101083E
:103EA800E8A10108ECA1010820100020F4A10108F4
:103EB80044A2010858A2010808A2010828A2010882
:103EC80070A2010888A2010890A2010808B5012281
:103ED8000449054808F0BEF900B908BDFFF75CFFC2
:103EE8000120FAE744A201082010002070B582B032
:103EF800FFF7ECFF00285DD001225D495D4808F01E
:103F0800A9F900285AD15B4BD3F80C4221465A48EC
:103F18000AF06CFF574D2146284608F012FDD5F8E7
:103F280008620021284608F00CFD701C09F014FAFC
:103F3800044601AB32460146284608F07CFA0028C0
:103F480046D04C4808F0E9FC2046FFF7A5FC05469A
:103F5800002845D049492846FFF7ACFC064618B169
:103F6800FFF747FD002842D145480AF09FFF454921
:103F78002846FFF79FFC064600283FD0FFF730FD94
:103F880000283BD073693BB100220023D6E9060123
:103F9800FCF7ECFB002831D1D6E90601FCF756FC0A
:103FA800394B1860FCF734FB02460B4637480AF0D9
:103FB8001DFF29E036480AF079FF9DE735480AF0E9
:103FC80075FF2C4BD3F80C4233480AF06FFF9DE77E
:103FD800019B0022E254214630480AF007FFB0E76F
:103FE8002F480AF063FF204609F0BEF9B2E73169AD
:103FF8002C4B19602C480AF0F9FEB8E72B480AF058
:1040080055FF214B2A4A1A602A492846FFF752FCD5
:10401800064610B1FFF7EDFCE0B927480AF046FF65
:10402800264B274A1A6027492846FFF743FC0646CD
:1040380010B1FFF7DEFCA0B923480AF037FF234B85
:10404800234A1A602846FFF703FA204609F08CF93C
:1040580002B070BD3169194B19601E480AF0C6FEDE
:10406800E1E73169194B19601B480AF0BFFEE9E71F
:1040780044A2010820100020F8A20108B8A10108F4
:1040880044A30108C0A101081000002054A301089E
:10409800ACA20108C0A20108E0A2010814A301080B
:1040A80024A301081810002038A3010864A30108FC
:1040B80000004040D0A1010884A30108141000208A
:1040C800C8A10108E8A10108A4A301081010002054
:1040D800DCA1010874A3010898A3010810B50446DF
:1040E8000E4B1A784FF47A73B3FBF2F30C4A10684C
:1040F800B0FBF3F000F0B4F868B90F2C01D9012037
:104108000AE0002221464FF0FF3000F08BF8054B03
:104118001C60002000E0012010BD00BF140000203A
:10412800000000201800002008B5074A136843F073
:1041380010031360032000F063F80020FFF7CEFFA0
:10414800FDF78EFC002008BD00200240034A1168DC
:10415800034B1B780B441360704700BF1C100020F2
:1041680014000020014B1868704700BF1C10002085
:1041780038B50446FFF7F6FF0546B4F1FF3F02D015
:10418800044B1B781C44FFF7EDFF401BA042FAD3F9
:1041980038BD00BF14000020002808DB0901C9B29F
:1041A80000F1604000F5614080F80013704700F0AE
:1041B8000F000901C9B2014B1954704714ED00E012
:1041C80000B500F00700C0F1070CBCF1040F28BFD0
:1041D8004FF0040C031D062B0FD9C31E4FF0FF3EF2
:1041E8000EFA0CF021EA000199400EFA03FE22EAC9
:1041F8000E0241EA02005DF804FB0023EEE700002E
:10420800074AD36823F4E0631B041B0C000200F484
:10421800E060034343F0BF6343F40033D360704767
:1042280000ED00E010B50446054BD868C0F3022045
:10423800FFF7C6FF01462046FFF7AEFF10BD00BFDF
:1042480000ED00E0002807DB00F01F024009012311
:104258009340024A42F82030704700BF00E100E076
:104268000138B0F1807F0BD24FF0E0235861054A46
:10427800F02182F823100020986107221A61704704
:104288000120704700ED00E030B40124056CAC401B
:10429800C56B6C60046863604368102B05D00368C5
:1042A80099600368DA6030BC704703689A600368F5
:1042B800D960F8E7002838D010B4024601681C4BD2
:1042C800994227D81B4B0B441B48A0FB03031B092F
:1042D8009B001364194BD363022382F821300868CA
:1042E8006FF30D10536894682343D468234314690B
:1042F80023435469234394692343D46923430343E1
:104308000B6000209063012382F8213082F820009E
:1043180010BC70470A4B0B440748A0FB03031B095A
:104328009B001364074BD363D6E70120704700BF97
:1043380007040240F8FFFDBFCDCCCCCC0000024002
:10434800F8FBFDBF0004024038B5044690F8200091
:10435800012832D0012084F8200094F82100C0B24E
:10436800012804D0002384F82030022038BD022020
:1043780084F821000020A0632568286820F0010047
:1043880028602046FFF780FFE36A5BB12268136864
:1043980043F00E0313602268136843F001031360AF
:1043A8000020E3E72268136823F0040313602268FF
:1043B800136843F00A031360EDE70220D6E70346CB
:1043C80090F82120D2B2022A06D004228263002269
:1043D80080F820200120704701680A6822F00E0248
:1043E8000A6001680A6822F001020A60026CC06B68
:1043F800012101FA02F2426083F82110002083F8BB
:104408002000704708B590F82130DBB2022B03D0AA
:1044180004238363012008BD0268136823F00E0398
:1044280013600268136823F00103136003684C4AA1
:1044380093424ED9783A934224D01432934230D0E2
:10444800143293422FD0143293422FD01432934215
:104458002FD0143293422FD0143293422FD002F52A
:10446800627293422ED0143293422DD0143293426A
:104478002CD01432934202D04FF4803203E04FF430
:10448800805200E00122374B5A60012380F8213026
:10449800002380F82030436B002B5ED09847002023
:1044A800B9E71022EFE74FF48072ECE74FF480523F
:1044B800E9E74FF48032E6E74FF48012E3E74FF084
:1044C8008072E0E70122DEE71022DCE74FF4807219
:1044D800D9E7254A934224D01432934225D0143286
:1044E800934224D01432934224D01432934224D0DD
:1044F8001432934224D01432934224D002F56272CB
:10450800934223D01432934222D01432934221D0C2
:104518001432934202D04FF4803203E04FF48052B9
:1045280000E00122114B5A60AFE71022FAE74FF47E
:104538008072F7E74FF48052F4E74FF48032F1E7E6
:104548004FF48012EEE74FF08072EBE70122E9E7C3
:104558001022E7E74FF48072E4E700205BE700BF32
:1045680080000240000402400800024000000240AF
:1045780038B5C36B1A6804682568016C04238B403E
:10458800134200F09B8015F0040F00F09780236819
:1045980013F0200F03D1236823F00403236003687A
:1045A8009A4A934246D9783A934224D01432934295
:1045B80028D01432934227D01432934227D0143291
:1045C800934227D01432934227D01432934227D0F3
:1045D80002F56272934226D01432934225D01432E7
:1045E800934224D01432934202D04FF4802203E045
:1045F8004FF4804200E00422854B5A60C36A03B13D
:10460800984738BD4022F7E74FF48062F4E74FF44B
:104618008042F1E74FF48022EEE74FF48002EBE7A7
:104628004FF08062E8E70422E6E74022E4E74FF42F
:104638008062E1E7774A934224D01432934225D02E
:104648001432934224D01432934224D01432934229
:1046580024D01432934224D01432934224D002F549
:104668006272934223D01432934222D0143293427E
:1046780021D01432934202D04FF4802203E04FF449
:10468800804200E00422644B5A60B7E74022FAE710
:104698004FF48062F7E74FF48042F4E74FF480224A
:1046A800F1E74FF48002EEE74FF08062EBE7042277
:1046B800E9E74022E7E74FF48062E4E702238B4012
:1046C800134200F0AB8015F0020F00F0A7802368BA
:1046D80013F0200F06D1236823F00A032360012377
:1046E80080F821300368494A93424BD9783A93427B
:1046F80024D0143293422DD0143293422CD0143249
:1047080093422CD0143293422CD0143293422CD0A2
:10471800143293422CD002F5627293422BD0143299
:1047280093422AD01432934229D01432934202D0B1
:104738004FF4003203E04FF4005200E00222344B01
:104748005A60002380F82030836A002B3FF459AF69
:10475800984756E72022F2E74FF40072EFE74FF44C
:104768000052ECE74FF40032E9E74FF40012E6E7B5
:104778004FF00072E3E70222E1E72022DFE74FF47F
:104788000072DCE7234A934224D01432934225D0A6
:104798001432934224D01432934224D014329342D8
:1047A80024D01432934224D01432934224D002F5F8
:1047B8006272934223D01432934222D0143293422D
:1047C80021D01432934202D04FF4003203E04FF468
:1047D800005200E00222104B5A60B2E72022FAE7AA
:1047E8004FF40072F7E74FF40052F4E74FF4003249
:1047F800F1E74FF40012EEE74FF00072EBE7022208
:10480800E9E72022E7E74FF40072E4E7800002407E
:1048180000040240080002400000024008238B40C8
:1048280013423FF4EEAE15F0080F3FF4EAAE2368EA
:1048380023F00E032360026CC16B012303FA02F21A
:104848004A60836380F82130002380F82030036BAE
:10485800002B3FF4D6AE9847D3E600BF70B582B0C0
:104868000024A446ABE0854DAB4214D00CD8A5F586
:104878008015AB420FD005F57025AB420BD0A5F5DE
:104888008015AB4210D106E07D4DAB4203D005F553
:104898008035AB4208D18B68002B5AD0012B53D0FE
:1048A8004261082400E0CC68BEF1FF0F53D80646E9
:1048B8004FEA8C0233680F25954023EA050304FA72
:1048C80002F2134333604B6813F0805F75D06D4B71
:1048D8009A6942F001029A619B6903F0010301930E
:1048E800019B4FEA9C02951C674B53F825600CF01E
:1048F8000305AD000F23AB4026EA0306634B98423D
:1049080030D003F58063984200F0968003F5806309
:10491800984200F0938003F58063984200F09080FD
:1049280003F58063984200F08D8003F58063984218
:1049380016D0062317E0CC680434B5E7CC680834F1
:10494800B2E7CC680C34AFE702610824ACE7002476
:10495800AAE70424A8E7061DACF108029200A9E71B
:10496800052300E00023AB4033430232464D45F8AF
:1049780022304B6813F4801F66D0454A936843EA97
:104988000E0393604B6813F4001F63D0404AD3684A
:1049980043EA0E03D3604B6813F4003F60D03C4AEF
:1049A800536843EA0E0353604B6813F4803F5DD0AD
:1049B800374A136843EA0E0313600CF1010C0B68C5
:1049C80033FA0CF258D0012202FA0CF203EA020E72
:1049D80032EA0303F1D14B68122B3FF644AF122B96
:1049E8003FF662AF01A555F823F000BF9F480008C5
:1049F800AF4800084549000857490008B148000871
:104A0800B1480008B1480008B1480008B14800089A
:104A1800B1480008B1480008B1480008B14800088A
:104A2800B1480008B1480008B1480008B14800087A
:104A38003F4900084B490008012394E7022392E705
:104A4800032390E704238EE7114A936823EA0E03B1
:104A5800936097E70E4AD36823EA0E03D3609AE778
:104A68000B4A536823EA0E0353609DE7084A13680C
:104A780023EA0E031360A0E702B070BD0000221005
:104A88000000311000100240000001400008014001
:104A9800000401408368194201D0012070470020BA
:104AA80070470AB10161704709040161704700004D
:104AB80008B5054B5B69034200D108BD024B58613C
:104AC800FFF778F8F9E700BF0004014038B512F4A1
:104AD800804F44D00468B4F850309BB291F800C0BD
:104AE80003EBCC03023304EB4304B4F80044C4F3EF
:104AF80009048B69A34228D31B1B8B618B697BB983
:104B0800056835F82C309BB223F4804323F07003FA
:104B180083F4005343F4004343F0800325F82C301A
:104B280012F0400F0ED002680D7832F825309BB293
:104B380023F4E04323F0700343F4004343F0C0033D
:104B480022F8253024B9204638BD00238B61D5E7EB
:104B580023460A894969006804F00AFFF3E70468F4
:104B6800B4F850309BB291F800C003EBCC03063385
:104B780004EB4304B4F80044C4F309048B69A3426A
:104B88002FD31B1B8B618B697BB9056835F82C30DB
:104B98009BB223F4804323F0700383F4005343F45F
:104BA800004343F0800325F82C3012F0400F0FD15A
:104BB800026891F800C032F82C309BB223F4E0432D
:104BC80023F0700343F4004343F0C00322F82C3071
:104BD800002CB8D023464A894969006804F0C8FE09
:104BE800B1E700238B61CEE770B586B0002800F0EE
:104BF8008180044690F8A932EBB1032384F8A932E6
:104C0800206803F044FF254655F8106BEC460FCD9D
:104C1800ACE80F002B68CCF80030231D0ECB3046D3
:104C280003F025FF054658B1022384F8A93201256F
:104C3800284606B070BD80F8A83208F077FADCE79D
:104C48000021206803F02DFF2B4616E05A1C02EBCA
:104C5800820104EBC1010120487002EB820104F8D3
:104C6800313004EBC1000021C17003EB830004EB79
:104C7800C0008163C1630164D3B261688B42E5D32C
:104C880016E005EB850304EBC303002283F86921D2
:104C980083F8685183F86B21C3F87821C3F87C2125
:104CA80005EB850304EBC303C3F880210135EDB29E
:104CB800A942E6D8254655F8106BEC460FCDACE86E
:104CC8000F002B68CCF80030231D0ECB304603F0C4
:104CD800EAFE054620B1022384F8A9320125A7E798
:104CE800002384F82430012384F8A932206804F0D2
:104CF8003DFA9DE701259BE738B590F8A832012BCE
:104D080011D00446012580F8A852006803F0B6FEC9
:104D18002946204608F01FFB206804F025FA0020E9
:104D280084F8A80238BD0220FCE770B505460C4699
:104D3800164612F0400F00F00E810268B2F85030AB
:104D48009BB2097803EBC103023302EB4302B2F8CA
:104D58000024C2F30902A36993424ED99B1AA361A6
:104D6800A369002B66D16378002B49D12B68B3F86F
:104D7800502092B2134403EB0113B3F80424C2F396
:104D88000902A3F80424B3F804246FEA42426FEA44
:104D9800524292B2A3F804242B686278002A3CD1CC
:104DA800B3F8502092B21344227803EB0213B3F8FD
:104DB8000C24C2F30902A3F80C24B3F80C246FEAFC
:104DC80042426FEA524292B2A3F80C242178284654
:104DD80008F0E0F916F4804F41D02A68217832F8BB
:104DE80021309BB223F4E04323F0700343F44043A3
:104DF80043F0800322F8213031E00023A361AFE7BC
:104E0800012BC9D12B68B3F8502092B2134403EB9D
:104E180001130022A3F80424BEE7012AD6D1B3F86F
:104E2800502092B21344227803EB02130022A3F815
:104E38000C24CBE716F4804F0DD0286830F82130C9
:104E48009BB223F4E04323F0700343F4404343F060
:104E5800800320F8213094F82430012B12D02A68DE
:104E6800217832F821309BB223F4E04323F0400349
:104E780083F0300343F4004343F0800322F82130E9
:104E8800002070BD636913446361E3691344E361FF
:104E9800216A2369994224D3C91A21626278002AB7
:104EA80044D12A68B2F8501089B20A44217802EB3A
:104EB8000112B2F80414C1F30901A2F804143E2B3C
:104EC8001BD9580913F01F0F00D10138B2F8041488
:104ED80089B2800280B2014341F40041A2F804146F
:104EE80026E021B9002384F824301346D6E70023AE
:104EF80084F8243023620B46D0E74BB9B2F8041487
:104F08006FEA41416FEA514189B2A2F804140FE0F7
:104F1800590813F0010F00D00131B2F8040480B22F
:104F2800890289B20143A2F8041401E0012A06D0DB
:104F38009BB222896169286804F020F98FE72A6802
:104F4800B2F8501089B20A44217802EB011299B2E2
:104F5800A2F80414ECE70268B2F850309BB2097862
:104F680003EBC103063302EB4302B2F80024C2F399
:104F78000902A36993424FD39B1AA361A369002B2B
:104F880067D16378002B4AD12B68B3F8502092B2CE
:104F9800134403EB0113B3F80424C2F30902A3F882
:104FA8000424B3F804246FEA42426FEA524292B2F0
:104FB800A3F804242B686278002A3DD1B3F8502066
:104FC80092B21344227803EB0213B3F80C24C2F311
:104FD8000902A3F80C24B3F80C246FEA42426FEAE2
:104FE800524292B2A3F80C242178284608F0D2F84D
:104FF80016F4804F7FF433AF2A68217832F82130D5
:105008009BB223F4E04323F0700343F4404343F09E
:10501800800322F8213022E70023A361AEE7012BA9
:10502800C8D12B68B3F8502092B2134403EB011394
:105038000022A3F80424BDE7012AD5D1B3F85020F3
:1050480092B21344227803EB02130022A3F80C2433
:10505800CAE716F4804F0DD1286830F821309BB28A
:1050680023F4E04323F0700343F4404343F0800308
:1050780020F8213094F82430012B7FF4F0AE6369D6
:1050880013446361E3691344E361216A2369994224
:1050980024D3C91A21622A686178002943D1B2F859
:1050A800501089B20A44217802EB0112B2F80C14AC
:1050B800C1F30901A2F80C143E2B1BD9580913F0AF
:1050C8001F0F00D10138B2F80C1489B2800280B2E7
:1050D800014341F40041A2F80C1426E021B9002351
:1050E80084F824301346D6E70023236284F824305A
:1050F8000B46D0E74BB9B2F80C146FEA41416FEA9E
:10510800514189B2A2F80C140FE0590813F0010FAD
:1051180000D00131B2F80C0480B2890289B201438F
:10512800A2F80C1401E0012906D09BB262896169DA
:10513800286804F023F892E6B2F8501089B20A44BD
:10514800217802EB011299B2A2F80C14EDE72DE9CF
:10515800F04105462868B0F8443013F4004F00F0D9
:105168009282B0F84440A3B214F00F0440F0E280F9
:1051780013F0100F6BD003889AB213F4006F40F04D
:105188009D8012F4004FE5D0038823F070031B05BF
:105198001B0D43F0800303802868B0F850309BB2A1
:1051A80095F8682103EBC203063300EB4303B3F819
:1051B8000034C3F30903C5F884318BB1D5F87C11E9
:1051C80071B1B5F86E2104F0D3FBD5F87C31D5F870
:1051D80084211344C5F87C310021284607F0CEFF0E
:1051E8002A68138899B213F4006FB3D101F44051BF
:1051F800B1F5405FAED0B2F850309BB21A44B2F865
:105208000C34C3F30903A2F80C34D5F878313E2BDB
:1052180077D9590913F01F0F00D10139B2F80C34AE
:105228009BB2890289B20B4343F40043A2F80C34C1
:105238002A6813889BB223F4804323F0700383F415
:10524800405343F4004343F08003138082E703880C
:105258009BB223F4E14323F070036FEA43436FEA00
:1052680053439BB203802A68B2F850309BB295F83A
:10527800281003EBC103023302EB4302B2F80034F7
:10528800C3F309036B64EA6B1A44EA6300212846F6
:1052980007F080FF95F82430002B3FF45BAF2B6CB0
:1052A800002B7FF457AF95F824302A6843F0800329
:1052B800A2F84C30002385F824304BE7B0F8503082
:1052C8009BB295F8682103EBC203063300EB430356
:1052D800B3F80034C3F30903C5F88431B5F86E2177
:1052E80005F52C7104F044FB2A68138823F0700339
:1052F8001B051B0D43F080031380284607F036FF7B
:1053080028E74BB9B2F80C346FEA43436FEA5343CA
:105318009BB2A2F80C348BE7590813F0010F00D0A8
:105328000131B2F80C3498B28B029BB20343A2F855
:105338000C347DE730F824309EB213F4004F4CD182
:1053480016F0800F3FF406AF621C02EB820105EBFA
:10535800C101286830F824309BB223F4E14323F0DC
:1053680070036FEA43436FEA53439BB220F824303B
:10537800CB78012B00F0F28016F4807F40F07E811C
:105388002868B0F850309BB2621C02EB820215F814
:10539800326003EBC603023300EB4303B3F8003477
:1053A800C3F3090304EB840205EBC202126C9A42B0
:1053B80040F24C8104EB840705EBC707D21A3A6424
:1053C80004EB840205EBC202126C002A40F045810E
:1053D8003146284607F0DEFEBCE630F8243023F0DC
:1053E80070031B051B0D43F0800320F8243004EBE9
:1053F8008401C90001F5B47105EB010804EB8403CD
:1054080005EBC30393F87431002B42D12868B0F838
:1054180050309BB204EB840205EBC20292F868217B
:1054280003EBC203063300EB4303B3F80074C7F37E
:10543800090717BB04EB840305EBC303D3F88421E6
:105448003A44C3F88421D3F87C213A44C3F87C2138
:10545800D3F880313BB104EB840305EBC303D3F8E5
:1054680078319F4275D204EB840305EBC30393F8AC
:105478006811284607F082FE62E704EB840105EB19
:10548800C1013B46B1F86E21D1F87C1104F070FAE5
:10549800D0E704EB840305EBC30393F86B31022BCD
:1054A80035D0296804EB840205EBC20292F8680142
:1054B80031F820309BB223F4E04323F0700343F427
:1054C800004343F0C00321F82030286892F868218F
:1054D80030F8223013F4804F20D0B0F850309BB20F
:1054E80003EBC203023300EB4303B3F80074C7F3C2
:1054F8000907002F9ED004EB840105EBC1013B4650
:10550800B1F87021D1F87C1104F032FA92E73246F2
:1055180041462846FFF7DAFA07468BE7B0F85030DD
:105528009BB203EBC203063300EB4303B3F80074EA
:10553800C7F30907002F3FF47DAF04EB840105EBA7
:10554800C1013B46B1F87221D1F87C1104F010FA80
:1055580070E74146286803F024FEF1E604EB840373
:1055680005EBC30300221A6493F83430FBB116F03C
:10557800400F37D04B781BBB2B68B3F8502092B242
:105588001344621C02EB820215F8322003EB02136B
:10559800B3F80424C2F30902A3F80424B3F80424DA
:1055A8006FEA42426FEA524292B2A3F804240134ED
:1055B80004EB840415F83410284607F0EBFDC9E520
:1055C800012BF4D12B68B3F8502092B21344621C1B
:1055D80002EB820215F8322003EB02130022A3F833
:1055E8000424E4E72A68631C03EB830305EBC30385
:1055F8005B78D3B9B2F850309BB21344621C02EB0B
:10560800820215F8322003EB0213B3F80C24C2F31C
:105618000902A3F80C24B3F80C246FEA42426FEA9B
:10562800524292B2A3F80C24C1E7012BBFD1B2F8C1
:1056380050309BB21344621C02EB820215F83220F0
:1056480003EB02130022A3F80C24B0E704EB840256
:1056580005EBC20200271764B2E604EB840205EBEF
:10566800C202D66B1E44D663526C04EB840405EB6D
:10567800C4041344636403F094FD6BE53246284682
:10568800FFF753FB66E50020BDE8F08190F8A832EB
:10569800012B0DD010B50446012380F8A83280F8FC
:1056A8002410006803F05AFD002084F8A80210BDF9
:1056B8000220704710B584B00446006803F058FD16
:1056C80010F4004F20D110F4806F21D110F4804FD6
:1056D8002FD110F4005F37D110F4805F3ED110F461
:1056E800006F40F0878010F4007F40F0AE8010F427
:1056F800807F27D02268B2F844309BB223F48073AD
:105708009BB2A2F844301DE02046FFF720FD19E0C7
:105718002268B2F844309BB223F480639BB2A2F8AB
:105728004430204607F047FD00212046FFF7AEFF32
:1057380008E02268B2F844309BB223F480439BB25D
:10574800A2F8443004B010BD2268B2F844309BB2CD
:1057580023F400539BB2A2F84430F3E72268B2F86E
:1057680040309BB223F004039BB2A2F84030226879
:10577800B2F840309BB223F008039BB2A2F8403045
:10578800204607F03BFD2268B2F844309BB223F470
:1057980080539BB2A2F84430D4E7226832F8231031
:1057A80004AA02EB430222F8101C0133DBB2072BD8
:1057B800F3D92268B2F840309BB243F00103A2F853
:1057C80040302268B2F840309BB223F001039BB20C
:1057D800A2F840302368B3F8442012F4806FF9D05F
:1057E800B3F8442092B222F4806292B2A3F8442023
:1057F80000230BE00023DAE7226804A901EB430148
:1058080031F8101C22F823100133DBB2072BF3D92F
:105818002268B2F840309BB243F00803A2F8403047
:105828002268B2F844309BB223F400639BB2A2F81A
:1058380044302268B2F840309BB243F00403A2F827
:105848004030204607F0CAFC7CE72268B2F84430B2
:105858009BB223F400739BB2A2F84430204607F0B1
:10586800A4FC6FE710B50446084611F0800F25D157
:1058780001F0070C0CEB8C01C90001F5B47E04EBB8
:105888000E010CEB8C0C04EBCC0C4FF0000E8CF8DA
:1058980069E100F0070008700A61CB70022B1AD08A
:1058A80094F8A832012B19D0012384F8A832206873
:1058B80003F00EF9002084F8A80210BD01F0070CCF
:1058C8000CF1010C0CEB8C0104EBC1014FF0010E43
:1058D80081F801E0DDE700230B71E1E70220ECE746
:1058E80010B504460B4611F0800F1FD101F00702D6
:1058F80002EB8201C90001F5B471014402EB820296
:1059080000EBC202002082F8690103F007030B7064
:1059180094F8A832012B13D0012384F8A832206808
:1059280003F0BBFA002084F8A80210BD01F00702BA
:10593800013202EB820100EBC10101204870E4E76B
:105948000220F2E710B501F0070C0CEB8C01C9003E
:1059580001F5B4710CEB8C0E00EBCE0ECEF87C2169
:10596800CEF880310024CEF884418EF869418EF853
:1059780068C10144006803F014FC204610BD01F022
:10598800070101EB810100EBC100D0F884017047E9
:1059980038B501F0070404F1010C0CEB8C0104EBA1
:1059A800840E00EBCE0ECEF83C20CEF8403001221B
:1059B8008EF84C20CEF848300025CEF8445000EB45
:1059C800C1035A7000F831401946006803F0E9FB3A
:1059D800284638BD38B501F007054268954231D8E8
:1059E80004460B4611F0800F1ED101EB8101C9005E
:1059F80001F5B471014403EB830300EBC3030022F8
:105A080083F8692101238B700D7094F8A832012B5B
:105A18001AD0012384F8A832206803F029FB5DB16D
:105A2800002084F8A80238BD6B1C03EB830100EB4F
:105A3800C10101224A70E5E704F52C71206803F0E2
:105A48009BFBEDE70120EEE70220ECE70B4601F0B7
:105A58000F014268914230D810B5044613F0800F08
:105A680021D103F0070202EB8201C90001F5B471EC
:105A7800014402EB820200EBC202002082F86901B5
:105A880000228A7003F007030B7094F8A832012BE8
:105A980015D0012384F8A832206803F00EFB0020FB
:105AA80084F8A80210BD03F00702013202EB82015C
:105AB80000EBC10101204870E2E701207047022095
:105AC800F0E790F8A832012B14D010B50446012352
:105AD80080F8A83211F0800F06D1006802F0F6FFB6
:105AE800002084F8A80210BD01F00701006802F048
:105AF800EBFFF5E70220704711F0800F0BD001F0A3
:105B08000701013101EB810100EBC10052B90273B9
:105B1800C3800020704701EB8101C90001F5B47111
:105B28000844F3E70122027303811B0C4381F0E769
:105B3800014B01221A62704700000E4282B0084BE6
:105B48001B68084AA2FB03235B0A00FB03F30193CB
:105B580000BF019B5A1E0192002BF9D102B0704779
:105B680000000020D34D6210002800F0F18170B5CC
:105B780082B00446036813F0010F2CD0994B5B6880
:105B880003F00C03042B1DD0964B5B6803F00C0349
:105B9800082B12D06368B3F5803F41D0002B55D154
:105BA80003F1804303F504331A6822F480321A6043
:105BB8001A6822F480221A6037E08A4B5B6813F473
:105BC800803FE7D0874B1B6813F4003F03D063681E
:105BD800002B00F0BF81236813F0020F75D0814BB2
:105BE8005B6813F00C0F5FD07E4B5B6803F00C030F
:105BF800082B54D02369002B00F08A807A4B0122AD
:105C08001A60FEF7AFFA0546764B1B6813F0020FD1
:105C180075D1FEF7A7FA401B0228F5D903209EE1AB
:105C2800704A136843F480331360636843B3FEF724
:105C380099FA05466B4B1B6813F4003FCBD1FEF76E
:105C480091FA401B6428F5D9032088E1B3F5A02F09
:105C580009D0644B1A6822F480321A601A6822F458
:105C680080221A60E1E703F18043A3F53C331A6808
:105C780042F480221A601A6842F480321A60D4E72B
:105C8800FEF770FA0546574B1B6813F4003FA2D085
:105C9800FEF768FA401B6428F5D903205FE1514BF1
:105CA8005B6813F4803FA5D14E4B1B6813F0020FBD
:105CB80003D02369012B40F04F814A4A136823F02F
:105CC800F803616943EAC1031360236813F0080FFE
:105CD80033D0A369002B5CD0434B0122C3F8802446
:105CE800FEF740FA05463F4B5B6A13F0020F21D1DD
:105CF800FEF738FA401B0228F5D903202FE1394A6C
:105D0800136823F0F803616943EAC1031360DCE711
:105D1800354B00221A60FEF725FA0546314B1B6801
:105D280013F0020FD1D0FEF71DFA401B0228F5D957
:105D3800032014E10120FFF701FF236813F0040F8B
:105D480000F09680274BDB6913F0805F34D1254B38
:105D5800DA6942F08052DA61DB6903F0805301931B
:105D6800019B0125214B1B6813F4807F26D0E36833
:105D7800012B3DD0002B53D103F1804303F50433AD
:105D88001A6A22F001021A621A6A22F004021A62DE
:105D980033E0154B0022C3F88024FEF7E3F90546EB
:105DA800104B5B6A13F0020FC7D0FEF7DBF9401BFC
:105DB8000228F5D90320D2E00025D3E70B4A13685F
:105DC80043F480731360FEF7CDF90646074B1B6852
:105DD80013F4807FCBD1FEF7C5F9801B6428F5D971
:105DE8000320BCE000100240000042420070004066
:105DF8005F4A136A43F001031362E36833B3FEF7A3
:105E0800B1F906465A4B1B6A13F0020F2FD1FEF761
:105E1800A9F9801B41F288339842F3D903209EE008
:105E2800052B09D0524B1A6A22F001021A621A6A2B
:105E380022F004021A62E0E74D4B1A6A42F00402AB
:105E48001A621A6A42F001021A62D6E7FEF78AF964
:105E58000646474B1B6A13F0020F08D0FEF782F97B
:105E6800801B41F288339842F3D9032077E0E5B9E3
:105E7800E369002B72D03E4A526802F00C02082AED
:105E880056D0022B17D03B4B00221A66FEF76AF950
:105E98000446374B1B6813F0007F47D0FEF762F9C2
:105EA800001B0228F5D9032059E0314AD36923F0B1
:105EB8008053D361DCE72F4B00221A66FEF752F9B4
:105EC80005462B4B1B6813F0007F06D0FEF74AF9F6
:105ED800401B0228F5D9032041E0236AB3F5803F2F
:105EE8001AD023494B6823F47413226A606A024368
:105EF80013434B601F4B01221A66FEF733F9044621
:105F08001B4B1B6813F0007F0ED1FEF72BF9001B0B
:105F18000228F5D9032022E0154A536823F40033F8
:105F2800A1680B435360DCE7002018E0002016E06E
:105F3800012B16D00E4B5B6803F48031226A914224
:105F480011D103F47013626A93420ED1002006E067
:105F580001207047012002E0012000E0002002B08B
:105F680070BD0120FBE70120F9E70120F7E700BF3A
:105F780000100240000042420F4B5B6803F00C0225
:105F8800082A01D00D487047C3F383420C49885C46
:105F980013F4803F0BD0084B5B68C3F34043094AB6
:105FA800D35C064A02FB00F0B0FBF3F07047064BE7
:105FB80003FB00F0704700BF0010024000127A0097
:105FC80018D9010814D9010800093D00002800F07B
:105FD800A08070B50D460446524B1B6803F00703BA
:105FE8008B420BD24F4A136823F007030B4313600D
:105FF800136803F007038B4240F08D80236813F089
:10600800020F17D013F0040F04D0474A536843F423
:10601800E0635360236813F0080F04D0424A5368C2
:1060280043F460535360404A536823F0F003A16877
:106038000B435360236813F0010F31D06368012BC1
:1060480020D0022B25D0384A126812F0020F64D0F3
:1060580035494A6822F0030213434B60FEF782F881
:106068000646314B5B6803F00C036268B3EB820FA2
:1060780016D0FEF777F8801B41F288339842F0D9A2
:10608800032045E0284A126812F4003FE0D10120BD
:106098003EE0254A126812F0007FD9D1012037E08E
:1060A800204B1B6803F00703AB420AD91D4A13684B
:1060B80023F007032B431360136803F00703AB4275
:1060C8002DD1236813F0040F06D0174A536823F420
:1060D800E063E1680B435360236813F0080F07D0AF
:1060E800114A536823F46053216943EAC10353609A
:1060F800FFF742FF0C4B5B68C3F303130B4AD35CF7
:10610800D8400B4B18600B4B1868FDF7E7FF0020D1
:1061180070BD012070470120FAE70120F8E701204F
:10612800F6E700BF0020024000100240FCA601086C
:106138000000002018000020014B1868704700BFBD
:106148000000002008B5FFF7F7FF044B5B68C3F3B6
:106158000223034AD35CD84008BD00BF00100240A8
:10616800F4A6010808B5FFF7E7FF044B5B68C3F323
:10617800C223034AD35CD84008BD00BF00100240C8
:10618800F4A6010870B582B00446036813F0010F45
:1061980036D03F4BDB6913F0805F49D13C4BDA695D
:1061A80042F08052DA61DB6903F080530193019B6E
:1061B8000125384B1B6813F4807F3BD0344B1B6A96
:1061C80013F4407313D0626802F440729A420ED0FE
:1061D8002F4A136A23F440702F490126C1F84064FE
:1061E8000026C1F84064106213F0010F36D1284A26
:1061F800136A23F4407361680B431362002D3ED188
:10620800236813F0020F06D0214A536823F4404351
:10621800A1680B435360236813F0100F34D01C4A55
:10622800536823F4800361690B43536000202CE01A
:106238000025BEE7174A136843F480731360FDF71F
:1062480091FF0646134B1B6813F4807FB6D1FDF708
:1062580089FF801B6428F5D9032016E0FDF782FF2B
:1062680006460B4B1B6A13F0020FC0D1FDF77AFFED
:10627800801B41F288339842F3D9032005E0D369A3
:1062880023F08053D361BBE7002002B070BD00BF8C
:1062980000100240007000400000424208B501387A
:1062A8000F2863D8DFE800F03557622F6262623248
:1062B80062626262626262082F4B5A68186810F064
:1062C800807054D0C2F383432C49C85C12F4803FD9
:1062D80015D0294B5B68C3F34043294AD25C294B4C
:1062E800B3FBF2F303FB00F0234B5B6813F4800F5E
:1062F8003DD14000244BA3FB0030400837E0234B3E
:1063080003FB00F0F0E7FFF737FE30E0FFF734FE5D
:106318002DE0194B1B6A40F202321A40B2F5817F18
:1063280026D003F44073B3F5007F04D0B3F5407F63
:1063380009D000201BE0104A526A12F0020FF5D073
:1063480049F6404013E00C4B186810F400300ED0AA
:106358004FF224400BE0FFF705FF074B5B68C3F3E0
:10636800813301335B00B0FBF3F000E0002008BD8F
:106378004FF40040FBE700BF001002402CD9010891
:1063880028D9010800127A00ABAAAAAA00093D0080
:1063980000B5036899691FFA81FED8699A691FFADE
:1063A80082FCE64505D0D86980B240EA02405DF833
:1063B80004FB80B240EA0140F9E70368186A5B6AA7
:1063C8009BB243EA00407047002302E001330A38D9
:1063D800C0B20928FAD81B01DBB218437047030979
:1063E80003EB830300F00F0000EB4300C0B27047DB
:1063F80010F0030F14D10D4BA3FB00235B0964229B
:1064080002FB13039BB26BB9084BA3FB0023DB0908
:106418004FF4C87202FB130080B228B901207047FC
:106428000020704701207047002070471F85EB51FE
:1064380000F5FA6C022921D801EB4103C1EBC30135
:106448001E4BA3FB013102EB5103634400F2CF70F2
:1064580003EB90031A4AA2FB0020A3EB501303EBB3
:10646800D01304331748A0FB03201A1A00EB52007C
:106478008008C0EBC000181AC0B2704701EB410396
:10648800C1EBC3010D4BA3FB013102EB5103634484
:1064980003EB9C030A4AA2FB0C12A3EB521303EB77
:1064A800D21302330748A0FB03201A1A00EB52004C
:1064B8008008C0EBC000181ADEE700BF398EE33849
:1064C8001F85EB51254992242DE9F8430746894653
:1064D80090F80F80457B867B002403E01E2E15D89C
:1064E800013601344C4533D20C2DFAD80123AB4088
:1064F80041F2AA521342F1D113F4256F10D113F0CF
:10650800040FEED01B2E12D80136EAE70C2D02D06C
:1065180001350126E5E708F1010801263546E0E7DF
:106528001D2E01D80136DCE701350126D9E71C2EDE
:1065380004D01D2ED5D101350126D2E71FFA88F0E7
:10654800FFF756FF08B10136CBE701350126C8E74A
:1065580087F80F80E9B27973F2B2BA734046FFF751
:1065680067FF3873BDE8F88338B50446FDF7FAFDD0
:10657800054623685A6812F0200F07D1FDF7F2FD8F
:10658800401BB0F57A7FF4D9032004E05A6842F042
:1065980010025A60002038BD38B5044602685368B6
:1065A80023F010035360FDF7DDFD054623685B68A3
:1065B80013F0200F07D1FDF7D5FD401BB0F57A7F0A
:1065C800F4D9032000E0002038BD38B505460C4654
:1065D800FFF7CAFF08B1012038BD2B68220C9A6169
:1065E8002B68A4B2DC612846FFF7D6FF0028F3D059
:1065F8000120F1E738B505460C46FFF7B5FF08B1AD
:10660800012038BD2B68220C1A622B68A4B25C6288
:106618002846FFF7C1FF0028F3D00120F1E770B545
:10662800002857D00D460646002955D0037C012B7B
:1066380054D00123037402234374BAB90B784C78FD
:10664800C4EB0414A4004FF4616202FB03448B788A
:106658001C4421463046FFF7B8FF0546C8B104235D
:106668007374002333740125284670BD0878FFF73A
:10667800B6FE4FF4616303FB00F46878FFF7AFFEE2
:10668800C0EB001004EB8004A878FFF7A8FE0444D0
:10669800DFE73268536823F0050353603046FFF79D
:1066A8008CFEB0F1FF3F01D0844204D801237374FB
:1066B80000233374D8E700F5A83101F5C0713046DE
:1066C800FFF798FF0028F1D0042373740023337474
:1066D8000125C9E70125C7E70125C5E70225C3E765
:1066E80000286FD02DE9F8430C46154607460029C7
:1066F8006AD003685B6813F0040F02D00120BDE87C
:10670800F883FFF745FE0646334BA3FB0023DB0A5D
:106718004FF4616202FB13023049A1FB02014809F0
:10672800C1F347116170C0EB0010A2EB8002A270A8
:106738002B4A964210D82370002D4BD02078FFF7B3
:1067480043FE20706078FFF73FFE6070A078FFF787
:106758003BFEA0700020D2E7224AA2FB03284FEAA2
:10676800181808EB4802A3EBC20323703846FFF75A
:1067780024FE8146B0F1FF3F06D0864202D2A0EB4C
:10678800060901E04FF0FF39174B03FB1866314645
:106798003846FFF71AFFC8B9B9F1FF3F0AD009EB2D
:1067A80006013846FFF726FF90B941463846FFF7FD
:1067B8008BFEC1E749463846FFF71CFF0028F4D096
:1067C80001209CE701207047012098E7012096E707
:1067D800012094E7002092E7C5B3A29189888888B0
:1067E8007F510100ABAAAAAA8051010000285AD003
:1067F80038B50D460446002957D0037C012B56D0E6
:106808000123037402234374BAB9CB78C3734B785A
:1068180043738B788373A27B617BE07BFFF708FE71
:10682800207328702046FFF7B3FD224B984211D8F9
:10683800012363740020207438BDC878FFF7CFFDAA
:10684800E0736878FFF7CBFD6073A878FFF7C7FDA2
:10685800A073E0E7184DA5FB00352D0C174B03FB83
:10686800150529462046FFF7B0FE28B104236374B6
:10687800002323740120DFE72046FFF79EFDB0F1D7
:10688800FF3FD5D08542D3D900F5A83101F5C071B5
:106898002046FFF7AFFE0028CAD004236374002304
:1068A80023740120C8E7012070470120C4E70220B3
:1068B800C2E700BF8F5F010007452EC2805101006B
:1068C8002DE9F04182B00023ADF804308DF8063090
:1068D80000B30C4617460546F1B11A4601A9FFF761
:1068E800FFFE0646E8B92B7B2370E87BE07095F83D
:1068F8000D8084F80180AD7BA57077B1FFF764FD4A
:10690800E0704046FFF760FD60702846FFF75CFDC9
:10691800A07002E0012600E00126304602B0BDE882
:10692800F0810126F9E7704710B5044603681A6834
:1069380012F0020F03D05B6813F0020F06D1074B69
:106948004FF400325A610123637410BDFFF7EBFF67
:106958002268536823F002035360F0E70004014003
:10696800C0B138B505460268536823F00803536080
:10697800FDF7F8FB04462B685B6813F0080F07D196
:10698800FDF7F0FB001BB0F57A7FF4D9032000E097
:10699800002038BD01207047002850D010B50446AB
:1069A800437C4BB1022363742046FFF7D9FF38B10B
:1069B80004236374012010BD0374FAF771FFF1E733
:1069C8002046FFF7D1FD28BB2268536823F0070350
:1069D8005360A36823B11B4A136B23F001031363AD
:1069E800184AD36A23F46073A1680B43D3626368BF
:1069F800B3F1FF3F12D02268C3F3034191602268CC
:106A08009BB2D3602046FFF7C7FD88B104236374A7
:106A18000120D0E7042363740120CCE70120FFF7AD
:106A28003DFC08B1431EE6E7042363740120C2E776
:106A38000023E37301236373A3736374BBE701202B
:106A4800704700BF006C0040704703681A6812F076
:106A5800010F1CD010B504465A6812F0010F10D06F
:106A68005B6813F0040F0DD0FFF7EEFF23686FF09B
:106A780004025A60042363742268536823F00103F4
:106A8800536010BDFAF77CFD01236374F4E7704787
:106A9800890001F1804101F5D84192B20A6070473E
:106AA800890001F1804101F5D841086880B270473A
:106AB80070B582B0044600230193006801F0F7FC2A
:106AC800054610B1284602B070BD206801F0B8FF35
:106AD80038B90123A364A36C012B0BD02E4628469A
:106AE80014E00023A364206801F0E1FC0028F2D040
:106AF8000546E7E70021206801F040FE0028EDD0B8
:106B08004FF08055DEE7019B01330193019A4FF660
:106B1800FE739A4213D896B90021206801F02EFE20
:106B2800E0B91249206801F0D7FE0646C0B9002135
:106B3800206801F0A7FCC30FE5D01E46E3E7019AE1
:106B48004FF6FE739A420ED810F0804302D001230C
:106B58006364B7E7002262641D46B3E70546B1E700
:106B68004FF08055AEE74FF08075ABE7000010C1DD
:106B780070B581B104460E46016D0904006801F044
:106B880015FE054608B1284670BD0021206801F0B1
:106B980079FC3060F7E74FF00065F4E72DE9F04F36
:106BA80087B005460C4616469B46DDF840A0FDF723
:106BB800D9FA002C36D0814695F83470FFB2012FEF
:106BC80040F005810023AB6306EB0B03EA6D9342AB
:106BD8002ED8032385F834302B680022DA626B6CD8
:106BE800012B00D076024FF0FF3300934FEA4B237E
:106BF8000193902302930223039300230493012318
:106C080005936946286801F040FCBBF1010F14D9CF
:106C180002232B633146286801F036FDA0B9DDF860
:106C2800048038E0AB6B43F00063AB630127D3E02B
:106C3800AB6B43F00073AB63CEE001232B633146AB
:106C4800286801F009FDE9E72B68654A9A63AB6B90
:106C58000343AB63012385F8343000232B63BBE087
:106C6800286801F0ECFB2070C0F307236370C0F3C1
:106C78000743A370000EE0700434A8F1040801363D
:106C8800072EEDD9FDF76EFAA0EB0900504510D29A
:106C9800BAF1000F0DD02868466B40F22A331E4027
:106CA80015D1436B13F4004FECD0B8F1000FE9D0C5
:106CB800E6E72B684A4A9A63AB6B43F00043AB6341
:106CC800012385F8343000232B63032784E0436BCA
:106CD80013F4807F05D0BBF1010F02D96B6C032B35
:106CE80038D12B685A6B12F0080F44D15A6B12F046
:106CF800020F4CD15A6B12F0200F54D12868436B05
:106D080013F4001F5BD0B8F1000F58D001F097FBC7
:106D18002070C0F307236370C0F30743A370000E0D
:106D2800E0700434A8F10408FDF71CFAA0EB090090
:106D3800504502D2BAF1000FE0D12B68284A9A6375
:106D4800AB6B43F00043AB63012385F83430002379
:106D58002B6341E001F0E0FC03460028C1D02A681B
:106D68001F499163AA6B1343AB63012385F8343041
:106D780000232B6330E01A4A9A63AB6B43F0080395
:106D8800AB63012385F8343000232B6324E0144AD5
:106D98009A63AB6B43F00203AB63012385F834308D
:106DA80000232B6318E00E4A9A63AB6B43F0200371
:106DB800AB63012385F8343000232B630CE040F2E9
:106DC8003A538363012385F83430002704E0AB6B22
:106DD80043F00053AB630127384607B0BDE8F08F96
:106DE800FF0540002DE9F04F8BB005460C461646CE
:106DF8009B46DDF850A0FDF7B5F9002C37D080464A
:106E080095F83470FFB2012F40F0E2800023AB63A5
:106E180006EB0B03EA6D93422FD8032385F8343031
:106E28002B680022DA626B6C012B00D076024FF0DF
:106E3800FF3304934FEA4B230593902306930023D3
:106E4800079308930123099304A9286801F01DFBFF
:106E5800BBF1010F16D920232B633146286801F0B6
:106E680043FC0190019BABB9DDF8149040E0AB6B9B
:106E780043F00063AB630127AFE0AB6B43F00073F3
:106E8800AB63AAE010232B633146286801F014FC99
:106E98000190E7E72B68534A9A63AB6B019A134357
:106EA800AB63012385F8343000232B6395E0237806
:106EB8000393627843EA02230393A27843EA0243E6
:106EC8000393E27843EA026303930434A9F10409C3
:106ED80003A9286801F0B6FA0136072EE7D9FDF7AD
:106EE80041F9A0EB0800504510D2BAF1000F0DD0BF
:106EF8002868466B40F21A331E4015D1436B13F4D1
:106F0800804FECD0B9F1000FE9D0E6E72B68354A9D
:106F18009A63AB6B019A1343AB63012385F8343052
:106F280000232B63032758E0436B13F4807F05D0BD
:106F3800BBF1010F02D96B6C032B18D12B685A6B6C
:106F480012F0080F24D15A6B12F0020F2CD15A6B91
:106F580012F0100F34D0234A9A63AB6B43F010033E
:106F6800AB63012385F8343000232B6335E001F04F
:106F7800D3FB03460028E1D02A681A499163AA6B1B
:106F88001343AB63012385F8343000232B6324E0DB
:106F9800144A9A63AB6B43F00803AB63012385F88B
:106FA800343000232B6318E00E4A9A63AB6B43F02E
:106FB8000203AB63012385F8343000232B630CE014
:106FC80040F23A529A63012385F83430002704E0EE
:106FD800AB6B43F00053AB63012738460BB0BDE8F9
:106FE800F08F00BFFF0540000346426E920F0A7003
:106FF800426EC2F383624A7090F8672002F003027F
:107008008A7090F86620CA7090F865200A7190F826
:1070180064204A71826E120DCA80B0F86A2002F0AC
:107028000F020A72826EC2F3C0324A72826EC2F3D3
:1070380080328A72826EC2F34032CA72826EC2F3A2
:1070480000320A7300224A73426C002A40F086809C
:10705800806E40F6FC7202EA8002D86E42EA9072B4
:107068000A61DA6EC2F3C2620A7593F86F2002F001
:1070780007024A75DA6EC2F342528A75DA6EC2F3B3
:107088008242CA75DA6EC2F3C2320A760A690132DE
:107098005A65087E00F00700023082405A6591F870
:1070A80008C00CF00F0C012000FA0CF09865400A9B
:1070B80000FB02F2DA654FF400721A66DA6EC2F368
:1070C80080324A76DA6EC2F3C6128A76DA6E02F037
:1070D8007F02CA761A6FD20F0A771A6FC2F341720B
:1070E8004A771A6FC2F382628A771A6FC2F38352A1
:1070F800CA771A6FC2F3405281F82020002081F825
:107108002100B3F8722002F0010281F822201A6FE0
:10711800C2F3C03281F823201A6FC2F3803281F89B
:1071280024201A6FC2F3403281F825201A6FC2F367
:10713800003281F826201A6FC2F3812281F82720B5
:107148001A6FC2F3012281F828201B6FC3F346038C
:1071580081F82930012381F82A307047012A11D19A
:10716800826E120402F47C12B0F86E0002430A61C7
:107178000A69013292025A65DA654FF400729A651B
:107188001A669BE7026805499163826B42F0805258
:107198008263012083F83400704700BFFF05400078
:1071A80070B590B004460123ADF81230006801F0C4
:1071B80052F900286CD0636C032B45D1636C032B08
:1071C8005DD1636C032B1DD0BDF812102165090435
:1071D800206801F046FB054600285BD100212068A5
:1071E80001F050F960660421206801F04BF9A066AF
:1071F8000821206801F046F9E0660C21206801F0BA
:1072080041F920670421206801F03CF9000DE06491
:1072180005A92046FFF7E8FE00283ED1226D12049A
:107228000023206801F092FA054698BB234653F8DC
:10723800106B93E807008DE80700043494E80E000B
:10724800304601F0E3F825E0206801F0F5FA05463C
:1072580000BB0021206801F015F96067042120684F
:1072680001F010F9A0670821206801F00BF9E06728
:107278000C21206801F006F9C4F880009EE70DF1A2
:107288001201206801F092FB0546002899D001E020
:107298004FF08065284610B070BD4FF08055F9E773
:1072A80070B58AB0044600230493059306930793A8
:1072B8000893762309930AAB13E907008DE80700C2
:1072C80004AB0ECB206801F0A1F818B101252846BF
:1072D8000AB070BD05461A4E0023C6F8A0302068D3
:1072E80001F0B5F80123C6F8A0300220FCF740FFF2
:1072F8002046FFF7DDFB30B1012584F83450A36B3D
:107308000343A363E3E72046FFF74AFF30B10125B3
:1073180084F83450A36B0343A363D8E74FF4007198
:10732800206801F081F90028D1D0236805499963C4
:10733800A36B0343A363012584F83450C7E700BF58
:1073480000003042FF054000A8B110B5044690F88F
:10735800343063B1032384F834302046FFF7A0FFAC
:1073680058B9A0632063012384F8343010BD037733
:10737800FAF7D6FAEEE7012070470120F6E7436CEA
:107388000B60836C4B60C36C8B60036DCB60436D8B
:107398000B61836D4B61C36D8B61036ECB61002004
:1073A800704710B582B004460023019301A9FFF786
:1073B800DFFB10B1A36B0343A3630198C0F3432021
:1073C80002B010BD002856D010B50446436A33B940
:1073D8004368B3F5827F05D00023C36102E0002330
:1073E800036143610023A36294F85130002B3CD021
:1073F800022384F851302268136823F04003136095
:10740800636803F48273A26802F404421343E268D7
:1074180002F400621343226902F002021343626914
:1074280002F001021343A26902F400721343E269F5
:1074380002F038021343226A02F080021343A26A60
:1074480002F40052216813430B60638B226803F037
:10745800040353602268D36923F40063D3610020D6
:107468006065012384F8513010BD84F850302046FF
:10747800FAF7BCFABCE70120704760B370B50E4656
:10748800154604468369B3F5807F26D090F84130CD
:10749800E3B1214651F8080B00F01EFFA2683146FF
:1074A800206800F04DFF236BA2682946606800F051
:1074B8006FFF2268A16852F8213043F0010342F8B7
:1074C8002130012384F84130002070BD80F840301D
:1074D800F9F78CFFDDE7012070470120F5E710B4CC
:1074E800036A046A24F001040462846924F0F00C3D
:1074F8004CEA021223F00A030B438261036210BCB8
:10750800704710B4036A046A24F0100404628469A2
:1075180024F4704C4CEA023223F0A00343EA01132E
:107528008261036210BC7047836823F070030B43C9
:1075380043F0070383607047704770477047704790
:10754800704710B5044603681A6912F0020F11D08B
:10755800DA6812F0020F0DD06FF002021A610123EF
:10756800037703689B6913F0030F70D0FFF7E6FFFA
:107578000023237723681A6912F0040F12D0DA68FF
:1075880012F0040F0ED06FF004021A610223237761
:1075980023689B6913F4407F5FD02046FFF7CEFF36
:1075A8000023237723681A6912F0080F12D0DA68CB
:1075B80012F0080F0ED06FF008021A610423237727
:1075C8002368DB6913F0030F4ED02046FFF7B6FFA0
:1075D8000023237723681A6912F0100F12D0DA6893
:1075E80012F0100F0ED06FF010021A6108232377E3
:1075F8002368DB6913F4407F3DD02046FFF79EFFE8
:107608000023237723681A6912F0010F03D0DA6880
:1076180012F0010F36D123681A6912F0800F03D0D7
:10762800DA6812F0800F34D123681A6912F0400F1B
:1076380003D0DA6812F0400F32D123681A6912F0C9
:10764800200F03D0DA6812F0200F30D110BDFFF7F9
:1076580074FF2046FFF773FF8AE72046FFF76DFFA8
:107668002046FFF76CFF9BE72046FFF766FF2046A2
:10767800FFF765FFACE72046FFF75FFF2046FFF7FF
:107688005EFFBDE76FF001021A612046FFF754FF65
:10769800C1E76FF080021A61204600F052F9C3E793
:1076A8006FF040021A612046FFF74AFFC5E76FF006
:1076B80020021A61204600F043F9C7E70368244A0C
:1076C800904212D002F5006290420ED0B0F1804F85
:1076D8000BD0A2F59832904207D002F58062904212
:1076E80003D002F58062904203D123F070034A6808
:1076F8001343174A904212D002F5006290420ED00E
:10770800B0F1804F0BD0A2F59832904207D002F525
:107718008062904203D002F58062904203D123F444
:107728004073CA68134323F080034A691343036014
:107738008B68C3620B688362054B984203D003F5DC
:107748000063984201D10B690363012343617047C9
:10775800002C014040B310B5044690F83D30F3B119
:10776800022384F83D30214651F8040BFFF7A6FFA9
:10777800012384F8463084F83E3084F83F3084F89A
:10778800403084F8413084F8423084F8433084F83B
:10779800443084F8453084F83D30002010BD80F82E
:1077A8003C30FAF74BFADBE70120704710B48468E5
:1077B80024F47F4C42EA03220A4342EA0C02826024
:1077C80010BC704790F83C30012B78D010B50446B7
:1077D800012380F83C30022380F83D30026893682A
:1077E80023F47F4323F0770393600B68602B4CD01E
:1077F80023D8402B54D011D8202B03D00AD80BB152
:10780800102B05D119462068FFF78EFE002028E0CE
:10781800012026E0302BF5D0012022E0502B0AD1A0
:10782800CA6849680068FFF75AFE50212068FFF7C8
:107838007BFE002015E0012013E0B3F5805F3AD00D
:10784800B3F5005F14D0702B37D1CB684A688968CC
:107858000068FFF7ABFF2268936843F077039360F3
:107868000020012384F83D30002384F83C3010BD0B
:10787800CB684A6889680068FFF798FF22689368B0
:1078880043F4804393600020EBE7CA6849680068C6
:10789800FFF737FE60212068FFF746FE0020E0E78B
:1078A800CA6849680068FFF71AFE40212068FFF798
:1078B8003BFE0020D5E70020D3E70120D1E70220D6
:1078C8007047000090F83C20012A34D010B40346D9
:1078D800012280F83C20022280F83D20026850688E
:1078E800946820F0700C086840EA0C0050601A6830
:1078F8001248824212D000F5006082420ED0B2F1E6
:10790800804F0BD0A0F59830824207D000F58060F8
:10791800824203D000F58060824204D124F08004C2
:10792800496821439160012283F83D20002083F8B3
:107938003C0010BC70470220704700BF002C01407B
:1079480070477047026802F10C0353E8003F23F0C8
:10795800C0030C3242E800310029F3D1202380F81B
:1079680041307047026802F10C0353E8003F23F4EA
:1079780090730C3242E800310029F3D1026802F119
:10798800140353E8003F23F00103143242E80031A6
:107998000029F3D1036B012B05D0202380F8423056
:1079A800002303637047026802F10C0353E8003FA9
:1079B80023F010030C3242E800310029F3D1ECE740
:1079C80090F84130DBB2212B01D002207047836848
:1079D800B3F5805F17D0036A5A1C02621A780368ED
:1079E8005A60C38C9BB2013B9BB2C3844BB90268FB
:1079F800D36823F08003D3600268D36843F0400360
:107A0800D360002070470369002BE4D1036A1B8808
:107A18000268C3F308035360036A02330362E0E7B2
:107A280010B504460268136923F44053C1680B4338
:107A3800136183680269134342691A430168CB687A
:107A480023F4B05323F00C031343CB60026853694B
:107A580023F4407381690B4353610268134B9A42C4
:107A680020D0FEF76FFB024602EB820202EB820295
:107A780063689B00B2FBF3F20D48A0FB0231490991
:107A8800642303FB11231B013233A0FB03035B09AF
:107A980003F0F00202EB011203F00F032168134414
:107AA8008B6010BDFEF75EFB0246DDE70038014043
:107AB8001F85EB512DE9F84305460F4616469946B2
:107AC800DDF820802B681C6837EA04040CBF012409
:107AD8000024B4422DD1B8F1FF3FF3D0B8F1000F24
:107AE80005D0FCF73FFBA0EB09004045EAD92A681E
:107AF80002F10C0353E8003F23F4D0730C3242E840
:107B080000310029F3D12A6802F1140353E8003F39
:107B180023F00103143242E800310029F3D1202375
:107B280085F8413085F84230002385F8403003203D
:107B380000E00020BDE8F88360B310B5044690F873
:107B4800413013B3242384F841302268D36823F4E6
:107B58000053D3602046FFF763FF2268136923F4BC
:107B6800904313612268536923F02A035361226802
:107B7800D36843F40053D36000206064202384F862
:107B8800413084F84230606310BD80F84030FAF725
:107B9800A9F8D7E7012070472DE9F04182B01E46C9
:107BA80090F84130DBB2202B4BD104460D4690466D
:107BB80000294AD00AB9012044E000234364212364
:107BC80080F84130FCF7CEFA0746A4F82480A4F8E0
:107BD8002680A368B3F5805F02D04FF000080FE05D
:107BE8002369FBB14FF000080AE038F8023B22682D
:107BF800C3F308035360E28C92B2013A92B2E28472
:107C0800E38C9BB28BB100963B4600228021204634
:107C1800FFF750FFD8B9002DE7D015F8012B2368DE
:107C28005A60E8E7A8460025EAE700963B460022A6
:107C380040212046FFF73EFF58B9202384F8413001
:107C480000E0022002B0BDE8F0810120FAE703203D
:107C5800F8E70320F6E72DE9F04182B01E4690F8D8
:107C68004230DBB2202B53D104460D469046002902
:107C780052D00AB901204CE000234364222280F844
:107C880042200363FCF76EFA0746A4F82C80A4F898
:107C98002E80A368B3F5805F02D04FF0000817E08C
:107CA800236913B14FF0000812E0A84600250FE041
:107CB80023685B68C3F3080328F8023B03E02368E2
:107CC8005B682B700135E28D92B2013A92B2E2857F
:107CD800E38D9BB2BBB100963B4600222021204693
:107CE800FFF7E8FED0B9002DE2D0A368B3F5805FB6
:107CF800E5D013B92369002BE1D023685B6803F052
:107D08007F032B70DEE7202384F84230002000E058
:107D1800022002B0BDE8F0810120FAE70320F8E76D
:107D2800704708B50168CA6822F04002CA6020227C
:107D380080F84120FFF7F4FF002008BD7047704726
:107D4800704710B5446A23685A6994F84130DBB229
:107D5800212B10D023685A6902F0400294F842306F
:107D6800DBB2222B11D0636C43F01003636420460E
:107D7800FFF7E6FF10BD02F08002002AEAD00023D8
:107D8800E3842046FFF7DEFDE4E7002AEBD000237A
:107D9800E3852046FFF7E6FDE5E708B5406A0023DE
:107DA800C385C384FFF7CCFF08BD90F84230DBB22F
:107DB800222B69D18368B3F5805F4FD0826AB3F50F
:107DC800805F04D0002B56D10369002B53D1036880
:107DD8005B681370836A01338362C38D9BB2013B76
:107DE8009BB2C385002B51D100B583B00268D3681C
:107DF80023F02003D3600268D36823F48073D36030
:107E08000268536923F001035361202380F842304C
:107E180000234363036B012B33D100230363026800
:107E280002F10C0353E8003F23F010030C3242E840
:107E380000310029F3D103681A6812F0100F06D038
:107E4800002201921A6801925B680193019B818D5F
:107E5800F9F772FB002003B05DF804FB0269002A01
:107E6800ACD1826A03685B68C3F308031380836A32
:107E780002338362B1E703685B6803F07F03137022
:107E8800A8E7FFF75BFFE5E702207047002070478F
:107E980010B582B0044602681368D068516913F0BF
:107EA8000F0F09D113F0200F0CD010F0200F09D0BC
:107EB8002046FFF77AFF16E011F0010115D110F402
:107EC800907F12D1216B012979D013F0800F03D054
:107ED80010F0800F40F0138113F0400F03D010F022
:107EE800400F40F0108102B010BD13F0010F06D012
:107EF80010F4807F03D0626C42F00102626413F0D8
:107F0800040F04D019B1626C42F00202626413F0EB
:107F1800020F04D019B1626C42F00402626413F0DB
:107F2800080F07D010F0200F00D119B1626C42F091
:107F380008026264626C002AD5D013F0200F02D0C8
:107F480010F0200F29D123685B6903F04003626CAD
:107F580012F0080F00D163B32046FFF703FD236832
:107F68005B6913F0400F20D0226802F1140353E834
:107F7800003F23F04003143242E800310029F3D1D6
:107F8800E36B73B1624A5A63E06BFCF73BFA002873
:107F9800A9D0E06B436B9847A5E72046FFF705FF9C
:107FA800D1E72046FFF7CCFE9DE72046FFF7C8FE45
:107FB80099E72046FFF7C4FE0023636493E713F0B4
:107FC800100F82D010F0100F3FF47FAF0023019301
:107FD8001368019353680193019B536913F0400F91
:107FE80051D0E26B13685B689BB2002B3FF47BAF08
:107FF800A18D99427FF677AFE3859369202B37D01F
:10800800226802F10C0353E8003F23F480730C321A
:1080180042E800310029F3D1226802F1140353E841
:10802800003F23F00103143242E800310029F3D164
:10803800226802F1140353E8003F23F0400314328E
:1080480042E800310029F3D1202384F8423000238C
:108058002363226802F10C0353E8003F23F0100366
:108068000C3242E800310029F3D1E06BFCF7A7F9A4
:1080780002236363A18DE38D9BB2C91A89B220469E
:10808800F9F75AFA2FE7A18DE38D9BB2C91A89B285
:10809800E38D9BB2002B3FF426AF00293FF423AFBA
:1080A800226802F10C0353E8003F23F490730C326A
:1080B80042E800300028F3D1226802F1140353E8A3
:1080C800003F23F00103143242E800300028F3D1C6
:1080D800202384F8423000232363226802F10C0332
:1080E80053E8003F23F010030C3242E80030002828
:1080F800F3D1022363632046F9F71EFAF3E620461C
:10810800FFF75EFCEFE62046FFF70BFEEBE600BF4D
:10811800A37D000808B5406A01234363036B012B64
:1081280002D0FFF70CFE08BD818D4908F9F704FA63
:10813800F9E708B50346406A1B681B6813F0200F6F
:108148002BD10023C385026802F10C0353E8003FDA
:1081580023F480730C3242E800310029F3D102681D
:1081680002F1140353E8003F23F00103143242E8FC
:1081780000310029F3D1026802F1140353E8003FEB
:1081880023F04003143242E800310029F3D12023C0
:1081980080F84230036B012B07D000234363036B45
:1081A800012B0FD0FFF7CAFD08BD026802F10C03CE
:1081B80053E8003F23F010030C3242E80031002955
:1081C800F3D1EAE7818DF9F7B7F9EDE730B583B078
:1081D800044613468162828500254564222280F880
:1081E8004220C26B1F489062E26B1F48D062E26B6C
:1081F8001E481063E26B556320680A46011DE06B58
:10820800FCF7A2F8019523681A6801925B6801934C
:10821800019B23695BB1226802F10C0353E8003F1C
:1082280043F480730C3242E800310029F3D122680C
:1082380002F1140353E8003F43F00103143242E80B
:1082480000310029F3D1226802F1140353E8003FFA
:1082580043F04003143242E800310029F3D10020F2
:1082680003B030BD3B8100081D8100084B7D00082C
:1082780090F84230DBB2202B29D110B582B00446E9
:1082880039B312B9012002B010BD012303630023E2
:108298004363FFF79BFF0028F5D1236B012B01D027
:1082A8000120F0E70023019323681A6801925B68B4
:1082B8000193019B226802F10C0353E8003F43F04D
:1082C80010030C3242E800310029F3D1DBE7022029
:1082D80070470120D7E7000010B40A6850F8223030
:1082E80023F0010340F822308B68082B24D00024A7
:1082F8004A6822431343CA6813430A6913434A6905
:108308001343CA6913430A6A13434A6A13438A6ABE
:108318001343CA6A13430A6B13438A691A434B6BA4
:108328001A43096850F82140044B2340134340F88E
:108338002130002010BC70474024D9E78000F0FFAE
:1083480000B5013250F8223003F0404C0B68D1F8E8
:1083580004E043EA0E13D1F808E043EA0E23D1F80B
:108368000CE043EA0E43D1F810E00EF1FF3E43EA79
:108378000E53D1F814E0AEF1020E43EA0E63896998
:108388000B434CEA030340F8223000205DF804FB5D
:10839800B3F5804F05D06FF0704340F822300020CD
:1083A800704730B450F82230094C1C400B684D68B7
:1083B80043EA05138D6843EA05238D692B43C96891
:1083C80043EA01431C4340F82240002030BC704778
:1083D8000000F0CF0B4B1B680B4AA2FB03235B0A80
:1083E80041F2883202FB03F31A46013B3AB1426B71
:1083F80012F0800FF8D0C5238363002070474FF038
:108408000040704700000020D34D621084B00DF189
:10841800040C8CE80E000B461343039A1343049A8A
:108428001343059A1343069A1343426822F4FD4204
:1084380022F07F0213434360002004B07047D0F855
:10844800800070470B68C0F8803000207047032315
:10845800036000207047006800F0030070470B6855
:1084680083604B688A681343CA6813430A691343D5
:10847800C2686FF30B021343C360002070470069A2
:10848800C0B270471430405870470B6843624B685D
:1084980083628B68CA6813430A6913434A691343A2
:1084A800C26A22F0F7021343C3620020704710B576
:1084B80086B00446002301930293039304934FF478
:1084C8008063059301A9FFF7CAFF2046FFF782FFE3
:1084D80006B010BD38B504460D46504B1B685049D0
:1084E800A1FB03135B0A03FB02F21346013A002BBC
:1084F8005DD0636B13F0450FF7D013F4006FF4D120
:10850800636B13F0040F06D1636B13F0010F05D0F2
:108518000120A0634DE00420A0634AE0C523A363C3
:108528002046FFF7ACFFA84201D0012041E000211E
:108538002046FFF7A7FF03463A481840C8B3002B68
:1085480038DB13F0804F38D113F0005F37D113F0C8
:10855800805F36D113F0006F36D113F0806F36D1BB
:1085680013F0807F36D113F4000F36D113F4800F47
:1085780036D113F4001F36D113F4801F36D113F40B
:10858800802F36D113F4003F36D113F4803F36D113
:1085980013F4004F36D113F4804F36D113F4005F33
:1085A80036D113F0080F36D04FF4000001E04FF039
:1085B800004038BD4FF00070FBE74020F9E780200D
:1085C800F7E74FF48070F4E74FF40070F1E74FF4E9
:1085D8008060EEE74FF40060EBE74FF48050E8E787
:1085E8004FF40050E5E74FF48040E2E74FF40040D5
:1085F800DFE74FF40030DCE74FF48020D9E74FF491
:108608000020D6E74FF48010D3E74FF40010D0E7EE
:108618004FF48000CDE74FF48030CAE70000002017
:10862800D34D621008E0FFFD30B587B004460191D4
:108638001025029540230393002304934FF480638D
:10864800059301A9FFF70BFF41F28832294620461E
:10865800FFF740FF07B030BD30B587B00446019141
:108668001125029540230393002304934FF480635C
:10867800059301A9FFF7F3FE41F288322946204607
:10868800FFF728FF07B030BD30B587B00446019129
:108698001225029540230393002304934FF480632B
:1086A800059301A9FFF7DBFE41F2883229462046EF
:1086B800FFF710FF07B030BD30B587B00446019111
:1086C8001825029540230393002304934FF48063F5
:1086D800059301A9FFF7C3FE41F2883229462046D7
:1086E800FFF7F8FE07B030BD30B587B004460191FA
:1086F8001925029540230393002304934FF48063C4
:10870800059301A9FFF7ABFE41F2883229462046BE
:10871800FFF7E0FE07B030BD30B587B00446002350
:1087280001930C2502954022039204934FF4806331
:10873800059301A9FFF793FE034A29462046FFF750
:10874800C9FE07B030BD00BF00E1F50530B587B000
:1087580004460192072502954023039300230493BE
:108768004FF48063059301A9FFF779FE41F288323F
:1087780029462046FFF7AEFE07B030BD30B587B0BA
:10878800044601913725029540230393002304935F
:108798004FF48063059301A9FFF761FE41F2883227
:1087A80029462046FFF796FE07B030BD30B587B0A2
:1087B800044601910D250295402303930023049359
:1087C8004FF48063059301A9FFF749FE41F288320F
:1087D80029462046FFF77EFE07B030BD0146144B00
:1087E8001B68144AA2FB03235B0A41F2883202FB8E
:1087F80003F31A46013BBAB14A6B12F0450FF8D0A1
:1088080012F4006FF5D14B6B13F0040F06D1486BCF
:1088180010F0010005D1C5238B63704704208863DD
:1088280070470120886370474FF00040704700BFD1
:1088380000000020D34D621010B586B00446002316
:10884800019302220292C022039204934FF48063A0
:10885800059301A9FFF703FE2046FFF7BFFF06B007
:1088680010BD10B586B00446019109230293C023B8
:108878000393002304934FF48063059301A9FFF742
:10888800EEFD2046FFF7AAFF06B010BD0146104BCB
:108898001B68104AA2FB03235B0A41F2883202FBE1
:1088A80003F31A46013B82B14A6B12F0450FF8D028
:1088B80012F4006FF5D1486B10F0040002D1C52303
:1088C8008B6370470420886370474FF000407047FF
:1088D80000000020D34D621010B586B0044641F068
:1088E800004141F48011019129230293402303930D
:1088F800002304934FF48063059301A9FFF7AFFDAC
:108908002046FFF7C3FF06B010BD0000F8B50546C6
:108918000E461746234B1B68234AA2FB03235B0A18
:1089280041F2883202FB03F31A46013B8AB36C6BAF
:1089380014F0450FF8D014F4006FF5D16B6B13F0F9
:10894800040F06D16B6B13F0010F05D00120A8634B
:1089580021E00420A8631EE02846FFF790FDB042FE
:1089680001D0012017E0C523AB6300212846FFF79B
:1089780089FD034610F4604008D013F4804F0BD1F2
:1089880013F4004F0BD04FF4805004E01B0C3B80D5
:1089980001E04FF00040F8BD4FF40050FBE74FF402
:1089A8008030F8E700000020D34D621070B586B023
:1089B80004460D46002301930326029640220392A3
:1089C80004934FF48063059301A9FFF748FD2A46F5
:1089D80031462046FFF79AFF06B070BD0146164B98
:1089E8001B68164AA2FB03235B0A41F2883202FB8A
:1089F80003F31A46013BE2B14A6B12F0450FF8D077
:108A080012F4006FF5D14B6B13F0040F0BD14B6BC5
:108A180013F001030AD1486B10F040000BD040223C
:108A28008A6318467047042088637047012088636A
:108A380070474FF00040704700000020D34D62108F
:108A480010B586B004464FF4D573019308230293FA
:108A580040230393002304934FF48063059301A9F3
:108A6800FFF7FDFC2046FFF7B9FF06B010BD84B044
:108A780001A880E80E00002004B0704703460020DB
:108A8800A3F844004FF43F42A3F840207047B0F8E1
:108A9800403023F47C535B045B0CA0F8403000208A
:108AA80070470020704784B0844601A880E80E0013
:108AB8000123ACF840300020ACF84000ACF844008A
:108AC800ACF8500004B07047002070470020704791
:108AD80010B5034691F800C030F82C2092B222F469
:108AE800EC4222F0700292B2C878032861D8DFE81D
:108AF80000F0555C0258002048F2800E42EA0E024F
:108B080023F82C2091F800C033F82C2092B222F4DC
:108B1800E04222F0700242EA0C0242EA0E0223F816
:108B28002C200A7B002A40F0DC804A78002A51D0A9
:108B3800B3F8502092B21A440C7802EB0412B1F840
:108B480006C04FEA5C0C4FEA4C0CA2F800C40C7843
:108B580033F8242012F0400F0CD033F8242092B2BE
:108B680022F4E04222F0700242F4004242F0C002D5
:108B780023F82420CA78012A1DD0097833F8212047
:108B880092B222F4E04222F0400282F0200242F443
:108B9800004242F0800223F8212017E142F40072DB
:108BA800AAE742F4C0620020A6E742F480620020EF
:108BB800A2E70120A0E7097833F8212092B222F435
:108BC800E04222F0400242F4004242F0800223F8E0
:108BD8002120FBE0B3F8502092B21A440C7802EB43
:108BE8000412B1F806C04FEA5C0C4FEA4C0CA2F82C
:108BF80008C4B3F8502092B21A440C7802EB04125D
:108C0800B2F80CC4CCF3090CA2F80CC40C693E2CC5
:108C180039D94FEA541E14F01F0F01D10EF1FF3E4F
:108C2800B2F80CC41FFA8CFC4FEA8E2E1FFA8EFE87
:108C38004CEA0E0C4CF4004CA2F80CC40C7833F837
:108C4800242012F4804F0CD033F8242092B222F45E
:108C5800E04222F0700242F4404242F0800223F8DF
:108C68002420097869BB33F8212092B222F480428B
:108C780022F0700282F4405242F4004242F0800234
:108C880023F82120A2E04CB9B2F80C446FEA44441E
:108C98006FEA5444A4B2A2F80C44CFE74FEA540C4C
:108CA80014F0010F01D00CF1010CB2F80C44A4B27D
:108CB8004FEA8C2C1FFA8CFC44EA0C04A2F80C44F2
:108CC800BCE733F8212092B222F4804222F07002ED
:108CD80082F4005242F4004242F0800223F821203C
:108CE80074E0CA78022A72D00C7833F8242092B241
:108CF80022F4E24222F0700242F4004242F0800282
:108D080023F82420B3F8502092B21A4491F800C0F6
:108D180002EB0C12B1F808C04FEA5C0C4FEA4C0C9D
:108D2800A2F800C4B3F8502092B21A4491F800C0D7
:108D380002EB0C12B1F80AC04FEA5C0C4FEA4C0C7B
:108D4800A2F808C44A78002A50D10C7833F82420B5
:108D580012F4804F0CD033F8242092B222F4E0426F
:108D680022F0700242F4404242F0800223F82420AC
:108D78000C7833F8242012F0400F0CD033F824205C
:108D880092B222F4E04222F0700242F4004242F031
:108D9800C00223F8242091F800C033F82C2092B2A6
:108DA80022F4804222F0700282F4405248F2800499
:108DB800224323F82C20097833F8212092B222F498
:108DC800E04222F04002224323F8212010BD0C7813
:108DD80033F8242092B222F4E04222F0700242F4E6
:108DE800014242F0800223F824208BE70C7833F804
:108DF800242012F4804F0CD033F8242092B222F4AD
:108E0800E04222F0700242F4404242F0800223F82D
:108E180024200C7833F8242012F0400F0CD033F8BB
:108E2800242092B222F4E04222F0700242F400427E
:108E380042F0C00223F82420CA78012A1ED00C78F8
:108E480033F8242092B222F4E04222F0400282F069
:108E5800200242F4004242F0800223F824200978DC
:108E680033F8212092B222F4804222F0700242F4B8
:108E7800004242F0800223F82120A7E70C7833F85B
:108E8800242092B222F4E04222F0400242F400424E
:108E980042F0800223F82420E1E70B7B002B46D127
:108EA8004B7813B30A7830F8223013F0400F0CD007
:108EB80030F822309BB223F4E04323F0700343F4EC
:108EC800004343F0C00320F822300A7830F82230FB
:108ED8009BB223F4E04323F0400343F4004343F000
:108EE800800320F82230002070470A7830F82230BA
:108EF80013F4804F0CD030F822309BB223F4E043B7
:108F080023F0700343F4404343F0800320F82230F9
:108F18000A7830F822309BB223F4804323F07003A0
:108F280043F4004343F0800320F82230DBE74B781A
:108F3800002B4ED10A7830F8223013F4804F0CD031
:108F480030F822309BB223F4E04323F0700343F45B
:108F5800404343F0800320F822300A7830F822306A
:108F680013F0400F0CD030F822309BB223F4E043CA
:108F780023F0700343F4004343F0C00320F8223089
:108F88000A7830F822309BB223F4E04323F07003D0
:108F980043F4004343F0C00320F822300A7830F845
:108FA80022309BB223F4804323F0700348F2800CF4
:108FB80043EA0C0320F822300A7830F822309BB2BA
:108FC80023F4E04323F0400343EA0C0320F8223063
:108FD80089E70A7830F8223013F4804F0CD030F843
:108FE80022309BB223F4E04323F0700343F4404360
:108FF80043F0800320F822300A7830F8223013F04A
:10900800400F0CD030F822309BB223F4E04323F019
:10901800700343F4004343F0C00320F822300A7879
:1090280030F822309BB223F4E04323F0700343F47A
:10903800404343F0800320F822300A7830F8223089
:109048009BB223F4E04323F0400348F2800C43EA48
:109058000C0320F822300A7830F822309BB223F42F
:10906800804323F0700343EA0C0320F822303AE7E8
:109078004B788BB10A7830F822309BB223F4E04366
:1090880023F0400383F0100343F4004343F08003CC
:1090980020F82230002070470A7830F822309BB23E
:1090A80023F4804323F0700383F4805343F4004394
:1090B80043F0800320F82230ECE70B7B002B4BD1E8
:1090C8004B7833B30A7830F8223013F0400F0CD0C5
:1090D80030F822309BB223F4E04323F0700343F4CA
:1090E800004343F0C00320F82230CB78012B33D063
:1090F8000A7830F822309BB223F4E04323F040038F
:1091080083F0200343F4004343F0800320F8223027
:1091180022E00A7830F8223013F4804F0CD030F86F
:1091280022309BB223F4E04323F0700343F440431E
:1091380043F0800320F822300A7830F822309BB2BE
:1091480023F4804323F0700383F4405343F4004333
:1091580043F0800320F822300020704711B98023A3
:10916800A0F84C300020704700207047002070475E
:10917800B0F8440080B270470020704701335B08A4
:1091880000EB420000F5806008E00A7891F801C021
:1091980042EA0C2220F8042B0231013B002BF4D1C7
:1091A800704770B505460C464A78012A3BD00B7BC0
:1091B800002B40F0A6828B690A69934240F28482B0
:1091C8009B1A8B61B5F850309BB22B44217803EB86
:1091D8000113B3F80C14C1F30901A3F80C143E2AC7
:1091E80040F27682510912F01F0F00D10139B3F80D
:1091F8000C2492B2890289B20A4342F40042A3F8CD
:109208000C24227835F822309BB223F4804323F0D3
:10921800700383F4405343F4004343F0800325F87C
:109228002230002070BD8E6909698E4200D90E4631
:10923800237B73B3E378022B4DD0236A9B1B2362F5
:10924800217835F8213013F0400F00F0F581002A1D
:1092580040F0E281B5F850309BB22B4403EB011388
:10926800B3F80C24C2F30902A3F80C243E2E40F2F2
:10927800BA81710916F01F0F00D10139B3F80C2417
:1092880092B2890289B20A4342F40042A3F80C243C
:10929800CBE1B6B23346E28861692846FFF76EFF34
:1092A800B5F850309BB22B44227803EB0213A3F895
:1092B8000464227835F822309BB223F4E04323F08B
:1092C800400383F0300343F4004343F0800325F860
:1092D80022300020A6E7236A994280F0668122782E
:1092E80035F822309BB223F4E04323F0700343F4B3
:1092F800014343F0800325F82230236A9B1B236235
:10930800227835F8223013F0400F00F0A7806378F8
:10931800B3BBB5F850309BB22B4403EB0213B3F840
:109328000C24C2F30902A3F80C243E2E0FD97109AC
:1093380016F01F0F00D10139B3F80C2492B289023C
:1093480089B20A4342F40042A3F80C241AE04EB949
:10935800B3F80C246FEA42426FEA524292B2A3F881
:109368000C240FE0720816F0010F00D00132B3F898
:109378000C1489B2920292B20A43A3F80C2401E0B9
:10938800012B30D0B3B2628961692846FFF7F6FE37
:10939800636933446361236A226993422DD99B1B15
:1093A80023626378002B45D1B5F850309BB22B442B
:1093B800227803EB0213B3F80424C2F30902A3F8DA
:1093C80004243E2E1DD9710916F01F0F00D1013952
:1093D800B3F8042492B2890289B20A4342F40042E3
:1093E800A3F8042428E0B5F850309BB22B4403EBD3
:1093F8000213B2B2A3F80C24C4E7002222621E466C
:10940800CFE74EB9B3F804246FEA42426FEA5242FA
:1094180092B2A3F804240FE0720816F0010F00D0EE
:109428000132B3F8041489B2920292B20A43A3F843
:10943800042401E0012B06D0B3B2228961692846D1
:10944800FFF79CFE35E7B5F850309BB22B442278E5
:1094580003EB0213B2B2A3F80424EDE76378B3BBBD
:10946800B5F850309BB22B4403EB0213B3F8042435
:10947800C2F30902A3F804243E2E0FD9710916F08D
:109488001F0F00D10139B3F8042492B2890289B2BE
:109498000A4342F40042A3F804241AE04EB9B3F890
:1094A80004246FEA42426FEA524292B2A3F80424BB
:1094B8000FE0720816F0010F00D00132B3F804145F
:1094C80089B2920292B20A43A3F8042401E0012B64
:1094D80030D0B3B2228961692846FFF74FFE63692D
:1094E80033446361236A226993422DD99B1B23620B
:1094F8006378002B45D1B5F850309BB22B442278C5
:1095080003EB0213B3F80C24C2F30902A3F80C24EA
:109518003E2E1DD9710916F01F0F00D10139B3F87D
:109528000C2492B2890289B20A4342F40042A3F899
:109538000C2428E0B5F850309BB22B4403EB0213FF
:10954800B2B2A3F80424C4E7002222621E46CFE781
:109558004EB9B3F80C246FEA42426FEA524292B213
:10956800A3F80C240FE0720816F0010F00D00132A6
:10957800B3F80C1489B2920292B20A43A3F80C24ED
:1095880001E0012B06D0B3B2628961692846FFF772
:10959800F5FD8EE6B5F850309BB22B44227803EBEC
:1095A8000213B2B2A3F80C24EDE7217835F8212094
:1095B80092B222F4E24222F0700242F4004242F0F7
:1095C800800225F82120B5F8502092B22A4421784B
:1095D80002EB01129BB2A2F8043422896169284681
:1095E800FFF7CCFD65E64EB9B3F80C246FEA4242AA
:1095F8006FEA524292B2A3F80C2416E0720816F0F1
:10960800010F00D00132B3F80C1489B2920292B261
:109618000A43A3F80C2408E0B5F850309BB22B4459
:1096280003EB0113B2B2A3F80C24B3B262896169E7
:109638002846FFF7A3FD3CE6B2BBB5F850309BB215
:109648002B4403EB0113B3F80424C2F30902A3F873
:1096580004243E2E0FD9710916F01F0F00D10139CD
:10966800B3F8042492B2890289B20A4342F4004250
:10967800A3F8042421E04EB9B3F804246FEA424267
:109688006FEA524292B2A3F8042416E0720816F068
:10969800010F00D00132B3F8041489B2920292B2D9
:1096A8000A43A3F8042408E0B5F850309BB22B44D1
:1096B80003EB0113B2B2A3F80424B3B2228961699F
:1096C8002846FFF75BFDF4E500228A611A4679E532
:1096D8004AB9B3F80C246FEA42426FEA524292B296
:1096E800A3F80C248DE5510812F0010F00D00131C8
:1096F800B3F80C2492B2890289B20A43A3F80C2465
:109708007FE5CB78022B4DD0012B40F02F81896962
:109718002369994240F2E680C91AA161F2B9B5F805
:10972800502092B22A44217802EB0112B2F80414B4
:10973800C1F30901A2F804143E2B40F2D78058095E
:1097480013F01F0F00D10138B2F8041489B2800257
:1097580080B2014341F40041A2F804146278002A5F
:1097680040F0F680B5F8502092B22A44217802EBF6
:109778000112B2F80C14C1F30901A2F80C143E2B23
:1097880040F2CD80590913F01F0F00D10139B2F80A
:109798000C349BB2890289B20B4343F40043A2F80C
:1097A8000C342EE5F2B9B0F850309BB203440A7875
:1097B80003EB0213B3F80424C2F30902A3F8042448
:1097C8000A693E2A31D9510912F01F0F00D1013917
:1097D800B3F8042492B2890289B20A4342F40042DF
:1097E800A3F804246378002B51D1B5F850309BB20C
:1097F8002B44227803EB0213B3F80C24C2F30902BA
:10980800A3F80C2422693E2A28D9510912F01F0F07
:1098180000D10139B3F80C2492B2890289B20A4303
:1098280042F40042A3F80C2433E04AB9B3F8042404
:109838006FEA42426FEA524292B2A3F80424D1E797
:10984800510812F0010F00D00131B3F8042490B28E
:109858008A0292B20243A3F80424C3E74AB9B3F8D0
:109868000C246FEA42426FEA524292B2A3F80C24E7
:109878000FE0510812F0010F00D00131B3F80C24A9
:1098880090B28A0292B20243A3F80C2401E0012BA1
:109898001DD0E369002B3FF4B4AC227835F82210D0
:1098A80044F2400303EA01008B4302D000287FF40E
:1098B800A8AC35F822309BB223F4E04323F07003C0
:1098C80043F4004343F0C00325F8223099E4B5F887
:1098D80050309BB22B44227803EB0213228AA3F860
:1098E8000C24D6E70023A3610B4617E74BB9B2F85F
:1098F80004146FEA41416FEA514189B2A2F8041495
:109908002CE7590813F0010F00D00131B2F8040414
:1099180080B2890289B20143A2F804141EE74BB948
:10992800B2F80C346FEA43436FEA53439BB2A2F890
:109938000C3466E4590813F0010F00D00131B2F875
:109948000C3498B28B029BB20343A2F80C3458E44F
:10995800012A7FF456ACB5F8502092B22A442178F7
:1099680002EB01129BB2A2F80C344AE4012059E43C
:1099780010B45C0800EB420000F5806007E030F8A6
:10998800042B0A70C2F307224A700231013C002CF2
:10999800F5D113F0010F01D003880B7010BC70478C
:1099A80038B51D4C21461D4803F08CFA1C4B187025
:1099B800012221461B4802F01DFC1B4B187018BBE6
:1099C8001A4805F073FA1A4805F070FA194D686DCF
:1099D800F7F742F80446A86DF7F73EF82146F6F780
:1099E800FFFB4FF06A51F6F7FBFB4FF06A51F6F7B1
:1099F800F7FBF6F70DFE02460B460F4805F0F6F9A1
:109A08000E4B01221A7038BD0D4805F04FFA0B4B6A
:109A180000221A70F7E700BF7C14002054D901080F
:109A2800801400204C1200201C00002084A2010891
:109A3800B4A30108F0080020C8A30108D408002036
:109A4800E8A301080020704700B583B000931346CF
:109A58000A4601460348FDF7A1F800B1012003B00A
:109A68005DF804FBF008002000B583B000931346AE
:109A78000A4601460348FDF7B5F900B1012003B0D5
:109A88005DF804FBF008002008B50348FDF789FCE1
:109A9800043818BF012008BDF008002008B50146A9
:109AA8000148FDF76CFC08BDF008002082B00123D6
:109AB8008DF807309DF8070002B0704708B5FFF72A
:109AC800F5FF012801D0012008BD0248FDF73CFC44
:109AD800FAE700BFF0080020202303800048704701
:109AE8006C00002020230380004870474C000020B1
:109AF80020230380004870472C0000200A2303809D
:109B0800004870472000002038B50446037CE3B9BC
:109B18004FF400730222012103F0B8FB0125C4F8B9
:109B28006C514FF4007302228121204603F0AEFBF2
:109B3800E5624FF41B7003F009FCC4F8B802A0B149
:109B4800204600F042F9002038BD402302220121BE
:109B580003F09CFB0125C4F86C51402302228121AB
:109B6800204603F093FBE562E3E70220ECE738B513
:109B78000446012103F095FB0025C4F86C518121AE
:109B8800204603F08EFBE562204600F04AF9D4F83F
:109B9800B80218B103F0DEFBC4F8B852002038BD93
:109BA8002DE9F04182B006460C46D0F8B872002381
:109BB800ADF806300B7813F0600536D0202D40F054
:109BC800B4804A78FE2A05D0FF2A1DD000F0B1FEE5
:109BD8000225ADE04A8812B9CA88012A05D0214673
:109BE800304600F0A6FE0225A2E013F0800FF6D062
:109BF800D0F8BC329B699847386001223946304614
:109C080001F0A4F9002593E04A8842B9CA8832B91C
:109C180013F0800F03D100F0F7F8002588E0214603
:109C2800304600F086FE022582E091F80180B8F106
:109C38000B0F76D8DFE808F0062D75757575757504
:109C48007575152290F89C32032B03D000F071FE35
:109C580002256DE002220DF1060101F077F9454673
:109C680066E090F89C32032B03D000F062FE0225D8
:109C78005EE00122391D01F069F959E090F89C3243
:109C8800032B02D18B787B6052E000F052FE022554
:109C98004EE0097903F00DFB2179304603F001FB12
:109CA800A38894F90420002A19DB03F00F0303EBBF
:109CB800830306EB83030022C3F85821337C4BBB94
:109CC8004FF4007302220121304603F0DFFA01232A
:109CD800C6F86C312179304600F04EF928E003F0DF
:109CE8000F0303EB830306EB830300229A61337CA3
:109CF8004BB94FF4007302228121304603F0C6FAB3
:109D08000123F362E6E7402302228121304603F073
:109D1800BDFAF5E7402302220121304603F0B6FAE6
:109D2800D5E700F006FE022502E000F002FE02255B
:109D3800284602B0BDE8F08108B500F093F800208D
:109D480008BD08B500F000F9002008BD09B1C0F849
:109D5800BC120020704710B51346D0F8B842D4F8AA
:109D680014229C469A4200D293B2D4F83422A2EB31
:109D78000C02C4F83422002284F838220422227209
:109D88000A46812103F0CCFA10BD38B50446D0F854
:109D9800B85295F8183223B9D5F814320BB16B7A4A
:109DA8003BB18121204603F08CFA6B7A022B04D058
:109DB80038BD012103F085FAF3E71F2305F5037287
:109DC8000121204603F0B4FAF2E738B50446D0F88A
:109DD800B85200202872687285F85D0285F85C0226
:109DE800D4F8BC321B6898470121204603F061FA79
:109DF8008121204603F05DFA1F2305F50372012136
:109E0800204603F095FA38BD08B5D0F8B8220023EB
:109E18001372012151721F2302F5037203F088FAAD
:109E280008BDD0F8B83200221A72704738B5054616
:109E3800D0F8B8420A4BC4F82C3284F83812002300
:109E480023720D2304F50B72812103F069FA1F2395
:109E580004F503720121284603F06AFA38BD00BFF1
:109E68005553425310B50446D0F8B8120B7A022B5A
:109E780008D006D3033BDBB2012B02D80021FFF741
:109E8800D5FF10BD01F21B2291F8191200F060FBFA
:109E98000028F6DA01212046FFF7C8FFF1E70000A5
:109EA80038B50546D0F8B842D4F81032C4F8303284
:109EB800D4F81432C4F83432012103F041FA1F28CF
:109EC80004D1D4F80C221F4B9A420CD0202305222F
:109ED80094F81912284600F0EFF802236372284616
:109EE800FFF753FF38BD94F819120129EED894F8FA
:109EF8001A32002BEAD0102BE8D804F21B2228468D
:109F080000F026FB00280CDB237A013BDBB2022B96
:109F1800E8D962898AB104F10C012846FFF71BFFD2
:109F2800E0E7237A052B03D02846FFF72EFFD9E771
:109F380001212846FFF77AFFD4E700212846FFF7DA
:109F480075FFCFE75553424310B50446D0F8B832F1
:109F58001A7A72B1012A0ED103F21B2293F8191250
:109F680000F0F6FA002806DA01212046FFF75EFF26
:109F780001E0FFF795FF10BD10B5D0F8B842637A3D
:109F8800022B08D011F0800F04D0012B02D0012140
:109F9800FFF74CFF10BD812103F093F90023637292
:109FA800F8E7000010B4D0F8B842537813F0010F66
:109FB8000DD00723638105E0013B9BB20F4AD15CBA
:109FC800E2181173002BF7D1002010BC7047D0F8AD
:109FD800BC32D86901EBC10100EB81000179053180
:109FE80013798B4200D90B46638104E0013B9BB295
:109FF800C15CE2181173002BF8D1E5E74CD90108D0
:10A00800D0F8B8020823438105E0013B9BB2044A1B
:10A01800D15CC2181173002BF7D10020704700BF24
:10A0280044D90108D0F8B8020823438105E0013B70
:10A038009BB2044AD15CC2181173002BF7D10020DF
:10A04800704700BF3CD9010810B4D0F8B8420023CB
:10A0580004E0E118002008730133DBB2112BF8D9B2
:10A06800702323730C23E37494F85C3294F85D1224
:10A078008B420FD003F1470104EBC1010879A073AB
:10A08800487A2076097A61760133DBB284F85C324B
:10A09800042B08D0122363811379122B00D8638113
:10A0A800002010BC7047002384F85C32F2E7D0F837
:10A0B800B832002058817047D0F8B80290F85D3265
:10A0C80003F1470100EBC1010A7100220A72013352
:10A0D800DBB280F85D32042B00D0704780F85D2237
:10A0E800FBE770B50446D0F8B862D6F814324BB91D
:10A0F8000D46D0F8BC329B680846984758B90023EB
:10A10800738170BD2023052296F81912FFF7D4FF3A
:10A118004FF0FF30F5E73A23022229462046FFF7A1
:10A12800CBFF052333724FF0FF30EAE770B582B0FA
:10A1380005460E46D0F8B842002306E0E2184FF074
:10A14800000C82F80CC001339BB20B2BF6D9D5F862
:10A15800BC325B680DF10602694630469847D0B9B3
:10A168000823E373009A531E190E2174C3F30741A1
:10A178006174C3F30723A374013AE27402232375BD
:10A18800BDF80630002262751A0AA275E3750C2321
:10A19800638102B070BD3A23022231462846FFF798
:10A1A8008BFF4FF0FF30F4E770B505460E46D0F848
:10A1B800B842D0F8BC325B6804F25E2204F518712C
:10A1C80030469847B8B9D4F86022531E190E217347
:10A1D800C3F307416173C3F30723A373013AE2731F
:10A1E800B4F85E320022227462741A0AA274E3740C
:10A1F8000823638170BD3A23022231462846FFF7BF
:10A208005BFF4FF0FF30F5E708B51A44D0F8B832D5
:10A21800D3F860329A4201D8002008BD21230522D4
:10A22800FFF74AFF4FF0FF30F7E72DE9F8430646FE
:10A238000F46D0F8B842D4F86852B4F85E3203FB3F
:10A2480005F5B5F5007F28BF4FF40075D0F8BC229E
:10A25800D2F8109004F10C08B5FBF3F39BB2D4F8D4
:10A26800642241463846C84700281DDBABB2424647
:10A278008121304603F054F8D4F86432B4F85E22F1
:10A28800B5FBF2F21344C4F86432D4F868329B1A6E
:10A29800C4F86832D4F83422521BC4F8342263B9A3
:10A2A80003232372002009E0112304223946304693
:10A2B800FFF702FF4FF0FF3000E00020BDE8F88311
:10A2C800F8B506460F46D0F8B842237A73BB154650
:10A2D80094F91832002B31DAD0F8BC329B68084662
:10A2E8009847A0BBAA78EB781B0443EA02632A7953
:10A2F80043EA02236A791A43C4F86422E9792B7A7B
:10A3080043EA0123C4F8683239463046FFF77CFF38
:10A3180000282FDB02232372D4F81422D4F86832E1
:10A32800B4F85E1201FB03F39A4219D14FF400739B
:10A33800638139463046FFF778FFF8BD20230522B0
:10A3480094F81912FFF7B8FE4FF0FF30F5E73A23FB
:10A35800022239463046FFF7AFFE4FF0FF30ECE7F8
:10A368002023052294F819123046FFF7A5FE4FF076
:10A37800FF30E2E74FF0FF30DFE72DE9F84306460C
:10A388008846D0F8B842D4F86852B4F85E3203FB75
:10A3980005F5B5F5007F28BF4FF40075D0F8BC224D
:10A3A800D2F8149004F10C07B5FBF3F39BB2D4F880
:10A3B800642239464046C84700281ADBD4F864228C
:10A3C800B4F85E32B5FBF3F10A44C4F86422D4F859
:10A3D8006822521AC4F86822D4F83412491BC4F807
:10A3E80034127AB900213046FFF720FD0020BDE87D
:10A3F800F8830323042241463046FFF75DFE4FF001
:10A40800FF30F4E702FB03F3B3F5007F28BF4FF4F6
:10A4180000739BB23A460121304602F089FF0020C2
:10A42800E5E72DE9F04106460F46D0F8B842237A11
:10A43800002B6AD1154694F91832002B40DBD0F86E
:10A44800BC329B6808469847002842D1D6F8BC32EF
:10A45800DB68384698478046002843D1AA78EB78CD
:10A468001B0443EA02632A7943EA02236A791A43FE
:10A47800C4F86422E9792B7A43EA0123C4F86832E4
:10A4880039463046FFF7C0FE002842DBD4F8683270
:10A49800B4F85E2202FB03F3D4F814229A422AD1BC
:10A4A800B3F5007F28BF4FF40073012121729BB2DE
:10A4B80004F10C02304602F03BFF4046BDE8F08153
:10A4C8002023052294F81912FFF7F6FD4FF0FF3804
:10A4D800F3E73A23022239463046FFF7EDFD4FF005
:10A4E800FF38EAE72723022239463046FFF7E4FD22
:10A4F8004FF0FF38E1E72023052294F8191230467F
:10A50800FFF7DAFD4FF0FF38D7E7FFF736FF804651
:10A51800D3E74FF0FF38D0E710B5D0F8B8425378FA
:10A5280013F0020F0AD1D4F86832D4F86422FFF786
:10A538006BFE002809DB0020608110BD2423052262
:10A54800FFF7BAFD4FF0FF30F7E74FF0FF30F4E7C1
:10A5580008B513785A2B5FD8DFE803F02E5E5E3219
:10A568005E5E5E5E5E5E5E5E5E5E5E5E5E5E365E2B
:10A578005E5E5E5E5E5E423A5E5E3E5E5E5E5E4A67
:10A588005E4E5E5E525E565E5E5E5E5A5E5E5E5E0B
:10A598005E5E5E5E5E5E5E5E5E5E5E5E5E5E5E5ED3
:10A5A8005E5E5E5E5E5E5E5E5E5E5E5E5E5E5E5EC3
:10A5B8005E5E5E5E5E5E4600FFF793FD002008BDAE
:10A5C800FFF742FD0020FAE7FFF7ECFC0020F6E772
:10A5D800FFF76DFD0020F2E7FFF769FD0020EEE7C9
:10A5E800FFF70EFD0020EAE7FFF71CFD0020E6E775
:10A5F800FFF79CFD0020E2E7FFF7D6FD0020DEE72D
:10A60800FFF75EFE0020DAE7FFF70BFF0020D6E732
:10A61800FFF782FF0020D2E720230522FFF74CFD39
:10A628004FF0FF30CBE798B108B50346D0F8B40235
:10A6380010B10020C3F8B40209B1C3F8B012012167
:10A6480083F89C121A70184602F0DEFD002008BD3F
:10A658000220704719B1C0F8B412002070470220D8
:10A66800704708B502F00AFE002008BD08B5D0F80A
:10A67800B4322BB11B68984700B908BD0220FCE72B
:10A688000220FAE708B5D0F8B4325B689847002092
:10A6980008BD38B5044600F52A75284600F035F996
:10A6A8000123C4F89432B4F8AE32C4F8983294F85E
:10A6B800A81201F01F03012B08D0022B0BD07BB985
:10A6C8002946204600F0D0FA002038BD2946204609
:10A6D80000F0FEFAF8E72946204600F029FBF3E7E8
:10A6E80001F08001204602F0ECFDEDE738B50446A4
:10A6F8000D4691BB1346D0F89422032A03D0052AAD
:10A7080024D0084633E0D0F86011D0F86421914293
:10A718000DD9891AC0F860118A4206D98AB2194639
:10A72800204600F028FC284621E092B2F7E7D0F84E
:10A73800B4321B691BB190F89C22032A04D020462E
:10A7480000F021FC284612E09847F8E70021C0F8FD
:10A75800941202F0B6FD284609E0D0F8B4329B699D
:10A7680033B190F89C22032A04D19847002038BDC1
:10A778000220FCE70220FAE738B504460D46002916
:10A7880053D11346D0F89422022A0CD0042A00D0C0
:10A798001AB98021204602F094FD94F8A032012BCA
:10A7A8003ED0284638BD026A416A8A421BD8C2692F
:10A7B800B2FBF1F301FB13232BB9914203D8D0F874
:10A7C80098329A421CD3D4F8B432DB681BB194F89F
:10A7D8009C22032A21D08021204602F072FD2046C7
:10A7E80000F0DCFBD9E7521A026292B2194600F077
:10A7F800BAFB00231A461946204602F099FDCCE719
:10A808000022114600F0AFFB0021C4F898120B4655
:10A818000A46204602F08CFDBFE720469847DAE753
:10A82800002384F8A0322846BCE7D0F8B4325B692C
:10A8380033B190F89C22032A04D198470020B1E74D
:10A848000220AFE70220ADE770B50446402300229E
:10A85800114602F01BFD0125C4F858514026C4F8E2
:10A868006461334600228021204602F00FFDA56175
:10A87800666284F89C520023C4F894326360C4F87A
:10A88800A432D4F8B8322BB1D4F8B4325B680021C2
:10A8980020469847002070BD01740020704790F84A
:10A8A8009C3280F89D32042380F89C320020704747
:10A8B80090F89C32042B01D00020704790F89D320C
:10A8C80080F89C32F8E708B590F89C32032B01D049
:10A8D800002008BDD0F8B432DB69002BF8D09847C7
:10A8E800F6E70346002002E00130C0B201331A78CF
:10A8F800002AF9D1704708B54B88012B00D008BD54
:10A90800C0F8A43200F03FFBF9E70B7803704B78EE
:10A9180043708B78CA7803EB022343800B794A791A
:10A9280003EB022383808B79CA7903EB0223C3806C
:10A93800704710B50446802102F0C3FC0021204670
:10A9480002F0BFFC10BD30B583B005460C460023AD
:10A95800ADF806304A88130A013B062B00F2A480A2
:10A96800DFE803F004182CA2A2869300D0F8B032D6
:10A978001B680DF10601007C9847BDF806201AB146
:10A98800E388002B40F09480E388002B00F09A8045
:10A9980003B030BD037C43B9D0F8B4329B6A0DF1E3
:10A9A8000600984702234370E7E7D0F8B432DB6A21
:10A9B8000DF10600984702234370DEE7D2B2052A5C
:10A9C80052D8DFE802F003101D2A3744D0F8B0321D
:10A9D8005B6823B10DF10601007C9847CDE721465D
:10A9E800FFF7A7FFD4E7D0F8B0329B6823B10DF189
:10A9F8000601007C9847C0E72146FFF79AFFC7E7A2
:10AA0800D0F8B032DB6823B10DF10601007C98471D
:10AA1800B3E72146FFF78DFFBAE7D0F8B0321B69DC
:10AA280023B10DF10601007C9847A6E72146FFF700
:10AA380080FFADE7D0F8B0325B6923B10DF10601B4
:10AA4800007C984799E72146FFF773FFA0E7D0F805
:10AA5800B0329B6923B10DF10601007C98478CE761
:10AA68002146FFF766FF93E72146FFF762FF8FE76E
:10AA7800037C33B9D0F8B4325B6B0DF1060098470C
:10AA88007BE72146FFF755FF82E7037C43B9D0F8FF
:10AA9800B4321B6B0DF106009847072343706CE72F
:10AAA8002146FFF746FF73E72146FFF742FF6FE7AE
:10AAB8009A4228BF1A46ADF806200146284600F0FB
:10AAC80045FA61E7284600F05EFA61E738B50446C2
:10AAD8008B88F3B9CB88E3B94B887F2B19D803F05F
:10AAE8007F0590F89C32032B0CD080F89E522946A3
:10AAF80002F00EFC204600F046FA35B1022384F835
:10AB08009C3209E0FFF715FF06E0012384F89C3228
:10AB180002E02046FFF70DFF38BD000038B50446B7
:10AB28000D468978284B197001290ED890F89C3267
:10AB3800022B0ED0032B21D02946FFF7FAFE224B19
:10AB480019782046FFF79EFD02E02946FFF7F1FE3F
:10AB580038BD81B14160032380F89C32FFF786FD40
:10AB6800022803D0204600F00EFAF1E729462046D5
:10AB7800FFF7DFFEECE700F006FAE9E789B1436882
:10AB880099421DD0D9B2FFF77DFD0F4B197861604E
:10AB98002046FFF76BFD02280DD0204600F0F3F9A0
:10ABA800D6E7022380F89C324160FFF76BFD204610
:10ABB80000F0E9F9CCE729462046FFF7BAFEC7E7D7
:10ABC80000F0E1F9C4E700BF8114002008B5CB8884
:10ABD800012B0AD190F89C32022B09D9032B11D1F1
:10ABE8000122011D00F0B2F901E0FFF7A2FE08BD45
:10ABF8005BB23BB10146002341F8083F012200F057
:10AC0800A5F9F4E7FFF795FEF1E708B590F89C324F
:10AC1800013B022B12D8CB88022B0CD10123C36035
:10AC2800D0F8A4320BB10323C360022200F10C0157
:10AC380000F08CF908BDFFF77CFEFBE7FFF779FE13
:10AC4800F8E708B590F89C32013B022B09D84B88ED
:10AC5800012B00D008BD0023C0F8A43200F093F9FE
:10AC6800F8E7FFF766FEF5E708B50B7803F0600331
:10AC7800202B05D0402B03D043B1FFF75AFE03E049
:10AC8800D0F8B4329B689847002008BD4B78092B50
:10AC98001BD8DFE803F011171A141A08051A0E0B4F
:10ACA800FFF751FEF0E7FFF711FFEDE7FFF736FF7B
:10ACB800EAE7FFF78BFFE7E7FFF7A7FFE4E7FFF710
:10ACC8001AFEE1E7FFF7BDFFDEE7FFF732FEDBE73D
:10ACD80038B505460C460B7803F06003202B06D0E8
:10ACE800402B04D01BB1FFF724FE002038BD95F897
:10ACF8009C32013B022B16D82379012B0ED8D5F8AC
:10AD0800B4329B68214628469847E388002BECD14B
:10AD18000028EAD1284600F036F9E6E72146284619
:10AD2800FFF707FEE1E721462846FFF702FEDCE7CA
:10AD380070B505468B880C7804F06004202C07D089
:10AD4800DAB2402C04D05CB1FFF7F3FD002405E033
:10AD5800D5F8B4329B68284698470024204670BD31
:10AD6800202C09D04E78012E33D0032E0AD0002E85
:10AD780055D0FFF7DEFDF1E7D0F8B4329B6898476D
:10AD88000446EBE790F89C32022B04D0032B11D039
:10AD9800FFF7CFFDE2E70AB1802A03D12846FFF783
:10ADA800C8FDDBE7114602F08CFA8021284602F044
:10ADB80088FAD3E74B8823B91AB1802A01D0CB8807
:10ADC8001BB1284600F0DFF8C8E7114602F079FA0F
:10ADD800F7E790F89C32022B04D0032B11D0FFF731
:10ADE800A8FDBBE70AB1802A03D12846FFF7A1FDD9
:10ADF800B4E7114602F065FA8021284602F061FAAC
:10AE0800ACE74B88002BA9D112F07F0F03D128465D
:10AE180000F0B9F8A2E7114602F05BFAF7E790F8FC
:10AE28009C02022806D0032829D02846FFF781FD76
:10AE3800344693E70AB1802A13D113F0800F15D155
:10AE480002F07F0202EB8202910001F5A871294409
:10AE5800043100230B600222284600F077F83446BC
:10AE68007CE72846FFF765FD344677E702F07F0266
:10AE780002EB82029100103129440431E9E75BB208
:10AE8800002B1FDB02F00F0000EB800005EB8000B9
:10AE9800D0F8580120B3002B27DB02F07F0303EB27
:10AEA80083039C0004F5A8742C4404340AB1802A56
:10AEB80024D10023236002222146284600F046F8C8
:10AEC80034464BE702F00F0000EB800005EB8000F2
:10AED80080690028DFD12846FFF72BFD34463DE77F
:10AEE8002846FFF726FD344638E702F07F0303EBD8
:10AEF80083039C0010342C440434D7E711462846B9
:10AF080002F0EFF910B101232360D4E70023236096
:10AF1800D1E7D0B170B50D4616460446FFF7E1FCFF
:10AF2800431C5B009BB233802B7003236B7002239E
:10AF380007E001345A1CD2B2E8540233DBB20021D4
:10AF4800A95420780028F4D170BD704708B513467D
:10AF58000222C0F89422C36103620A46002102F06B
:10AF6800DFF9002008BD08B513460A46002102F0A3
:10AF7800D7F9002008BD08B513460A46002102F09B
:10AF8800D7F9002008BD08B50423C0F8943200237F
:10AF98001A46194602F0C4F9002008BD08B5052371
:10AFA800C0F8943200231A46194602F0C1F900206D
:10AFB80008BD000008B5044B03EB800252685268D4
:10AFC8000344187A904708BDA414002008B5084B1C
:10AFD8001B5C53B9064B01221A5403EB80025268DA
:10AFE80012680344187A904708BD0020FCE700BFA8
:10AFF800A414002038B5044C04EB80056D68AD68D6
:10B008000444207AA84738BDA414002038B5044C5D
:10B0180004EB80056D68ED680444207AA84738BDC4
:10B02800A414002010B5044B03EB80046468246961
:10B038000344187AA04710BDA414002008B5074B94
:10B0480001221A70FEF73AFD20B9044A137803F07A
:10B05800FE031370014B187808BD00BFC400002020
:10B0680008B5074B01221A70FEF70EFD20B9044AF5
:10B07800137803F0FE031370014B187808BD00BF66
:10B08800C400002010B5084611461A46094BFEF7C1
:10B09800DBFC10B10123184610BD074CFEF7F4FC89
:10B0A80003460028F7D0631E0CB11C46F6E70123BF
:10B0B800F1E700BF00E1F505A086010010B50846DC
:10B0C80011461A46094BFEF7CFFC10B1012318466A
:10B0D80010BD074CFEF7D8FC03460028F7D0631EC6
:10B0E8000CB11C46F6E70123F1E700BF00E1F505C6
:10B0F800A086010030B589B0124B187810F0010411
:10B108001AD1154603291BD8DFE801F002040A10FA
:10B118000C4612E06846FEF7C1FC069B2B600CE06B
:10B128006846FEF7BBFC079B2B8006E06846FEF7E7
:10B13800B5FC079B2B6000E00324204609B030BD16
:10B148000424FAE7C400002004E011F8012B00F8F9
:10B15800012B1A46531E002AF7D1704702E000F867
:10B16800011B1A46531E002AF9D1704710B4034632
:10B1780000201446013A34B113F8010B11F801CB41
:10B18800B0EB0C00F5D010BC7047034600E001336B
:10B19800187808B18842FAD17047000030B4002509
:10B1A8002B4601E001250133012B1ED803EB430296
:10B1B8001C4C54F82220002AF4D0D0F80042A242B5
:10B1C800F1D103EB4304174A02EB84025468D0F828
:10B1D80008229442E7D103EB4304124A02EB8402AB
:10B1E8001489B0F806229442DDD1022B0CD0B1B9F3
:10B1F80003EB43030B4A02EB83035B89B3F5807FC0
:10B208000BD0002030BC70472DB9022901D0122084
:10B21800F8E70020F6E70020F4E71020F2E7102016
:10B22800F0E700BF84140020002000E0013001286E
:10B2380006D800EB40029300034AD358002BF5D1FF
:10B24800023818BF012070478414002010B500236D
:10B2580000E00133012B1CD803EB43022D4C54F8BA
:10B268002240D0F800229442F3D103EB4304294A48
:10B2780002EB84025468D0F808229442E9D103EB27
:10B288004304244A02EB84021489B0F8062294424B
:10B29800DFD1022B0AD041B303EB43011D4A02EB75
:10B2A800810252899ABB4FF4807226E00023012B59
:10B2B80007D803EB4302174C54F822200AB1013394
:10B2C800F5E7022B21D0134C03EB430C04EB8C0263
:10B2D800D0F800E244F82CE0D0F808425460B0F806
:10B2E8000602108100205081D5E703EB4301094A8B
:10B2F80002EB81025289013292B203EB4300054905
:10B3080001EB80014A81581C10BD0020FCE7002099
:10B31800FAE700BF84140020013801281BD800EB8D
:10B3280040020F4B03EB82035B89B3F5807F03D0A8
:10B3380053B1013B9BB200E0002300EB4001084AF7
:10B3480002EB8102538143B900EB400083000020E7
:10B35800034AD0507047022070470020704700BF52
:10B3680084140020002302E010BC70470133012B35
:10B3780017D803EB43020B4951F822208242F5D13A
:10B3880010B403EB4302920000248C500133012BCC
:10B39800EAD803EB4302034951F822208242F5D14F
:10B3A800EFE7704784140020D0F824320433490AA8
:10B3B800D0F8002292F80222B1FBF2F101E0091A5A
:10B3C8000833186818B18142F9D2586808447047A0
:10B3D8000246C87E8B7E43EA002092F80032032B97
:10B3E80000D070474A7D0B7D43EA022340EA0340C0
:10B3F800F7E78176C1F30723C376C1F307430375E3
:10B40800090E4175704700002DE9F84F89460C6810
:10B4180000E0013423782F2BFBD05C2BF9D0D0F837
:10B4280018A20B2220215046FFF798FE002633462B
:10B438004FF00808374619E0BF00FFB246464FF004
:10B448000B0812E015F0800F25D129463148FFF787
:10B458009CFE00285AD1A5F14103DBB2192B20D854
:10B4680047F002070AF8065001365B4603F1010B64
:10B47800E55C202D1FD92F2D1DD05C2D1BD02E2D26
:10B4880001D0B045DED8B8F1080F3DD12E2DD3D06C
:10B498000620BDE8F88F47F00307803D1E4B5D5D31
:10B4A800D3E7A5F16103DBB2192BDBD847F001071D
:10B4B800203DEDB2D6E75C44C9F80040202D14D8F1
:10B4C80004232EB39AF80020E52A10D0B8F1080F0B
:10B4D80011D007F00302012A10D007F00C07042F3F
:10B4E8000FD08AF80B300020D3E70023E9E70522C4
:10B4F8008AF80020EAE7BF00FFB2EAE743F010034A
:10B50800EBE743F00803ECE70620C2E70620C0E7B4
:10B518000620BEE700A4010868D9010801460068B2
:10B5280038B102461378202B06D93A2B04D00132C1
:10B53800F8E74FF0FF3070473A2B01D000207047F2
:10B5480010B4034613F8010B3038092808D89A427A
:10B5580002D04FF0FF3005E030B901320A6001E057
:10B568004FF0FF3010BC70474FF0FF30FAE7F8B5E6
:10B5780090F804520DB92846F8BD0446D0F82C724C
:10B5880001233A46014690F80102FFF73FFD0546C0
:10B59800D0B9002384F80432D4F82032FB1AD4F846
:10B5A80018229342E7D294F803620AE0D4F81832DA
:10B5B8001F4401233A46214694F80102FFF726FD6D
:10B5C800013E012EF2D8D6E70125D4E770B5D0F8B0
:10B5D8002C328B4202D10026304670BD04460D46FF
:10B5E800FFF7C5FF06460028F6D101232A46214663
:10B5F80094F80102FFF7FEFC10B101264FF0FF3569
:10B60800C4F82C52E8E7000010B50446002380F87F
:10B6180004324FF0FF33C0F82C32FFF7D7FF98BB46
:10B62800024694F8FF1194F8FE3143EA01231BB255
:10B6380017498B422AD194F8391094F838301B04F2
:10B6480043EA016394F8371043EA012394F836106B
:10B658000B4323F07F430F498B4213D094F85510C6
:10B6680094F854301B0443EA016394F8531043EAF6
:10B67800012394F852100B4323F07F4305498B4272
:10B6880000D00122104610BD0322FBE70222F9E791
:10B6980055AAFFFF46415400B0B108B5D0F80032B2
:10B6A80043B193F8001229B1B3F80612B0F8042296
:10B6B800914201D0092008BD93F80102FFF77AFCF6
:10B6C80010F00100F7D0F5E7092070472DE9F043A5
:10B6D80085B005461746002303600846FFF71EFF9E
:10B6E800061EC0F29E819F4B53F82640002C00F0A6
:10B6F8009D812C6094F800327BB194F80102FFF729
:10B7080059FC10F0010508D1002F00F08B8110F0D2
:10B71800040F00F087810A2584E1002384F80032B1
:10B72800F0B284F80102FFF751FC10F0010F40F06D
:10B738007F811FB110F0040F40F07C81002120466A
:10B74800FFF762FF0546012800F095800027032DCA
:10B7580000F07281002D40F07181227BE37A43EA88
:10B7680002231BB2B3F5007F40F06A81E27DA37D1E
:10B7780053EA02230DD194F8272094F826301B04AD
:10B7880043EA026394F8252043EA022394F824202C
:10B798001343C4F81832217C84F803124A1ED2B22B
:10B7A800012A00F24F8103FB01F1607B84F8020259
:10B7B800002800F04981421E104240F04781A67CD3
:10B7C800627C42EA06221646A4F8082212F00F0FFD
:10B7D80040F03E8194F814C0E27C52EA0C220ED16B
:10B7E80094F823C094F82220120442EA0C6294F8D8
:10B7F80021C042EA0C2294F820C042EA0C0294F8D4
:10B808000FE094F80EC05CEA0E2C00F023810CEBDC
:10B81800010909EB16194A45C0F01E81A2EB09027D
:10B82800B2FBF0FE8242C0F0198140F6F5729645EF
:10B838003AD94FF6F572964577D84FF0020835E0B9
:10B84800002304AA02EB810242F8103C01310329CB
:10B8580013D80B0103F5DF7323441A79002AEFD0BC
:10B86800D87A9A7A120442EA0062587A42EA0022A6
:10B878001B7A1343E5E70021E9E700260BE0394688
:10B888002046FFF7C1FE054600283FF460AF0136A9
:10B89800032E3FF65CAF04AB03EB860353F8107C32
:10B8A800002FECD10225F2E74FF001080EF1020E4D
:10B8B800C4F814E2C4F81C720CEB0702C4F8202286
:10B8C80007EB0900C4F82802B8F1030F30D0002EA6
:10B8D80000F0C8800A44C4F82422B8F1020F3DD011
:10B8E8000EEB4E010EF0010202EB510202F2FF12C2
:10B8F800B3EB522FC0F0B8804FF0FF33C4F81032CA
:10B90800C4F80C32802384F80532B8F1030F2DD027
:10B9180084F80082144A138801339BB21380A4F878
:10B9280006322046FFF71EFD7CE04FF00308BDE716
:10B93800002E40F0958094F82F1094F82E201204D1
:10B9480042EA016294F82D1042EA012294F82C1080
:10B958000A43C4F824224FEA8E02C7E74FEA4E0290
:10B96800C4E700BFA01400209C14002094F83120E4
:10B9780094F8303043EA02231BB2012BC8D1791C5A
:10B988002046FFF723FE0028C2D1002384F80532A1
:10B9980094F8FF2194F8FE3143EA02231BB2334A9C
:10B9A8009342B5D1E278A3781B0443EA0263627834
:10B9B80043EA0223227813432D4A9342A8D194F8EC
:10B9C800E72194F8E6311B0443EA026394F8E52181
:10B9D80043EA022394F8E4211343264A934297D179
:10B9E80094F8EB2194F8EA311B0443EA026394F8D3
:10B9F800E92143EA022394F8E8211343C4F81032FA
:10BA080094F8EF2194F8EE311B0443EA026394F8AA
:10BA1800ED2143EA022394F8EC211343C4F80C32D5
:10BA280076E70B25284605B0BDE8F0830C25F9E735
:10BA38000325F7E70A25F5E70125F3E70D25F1E7E3
:10BA48000D25EFE70D25EDE70D25EBE70D25E9E7DA
:10BA58000D25E7E70D25E5E70D25E3E70D25E1E7EA
:10BA68000D25DFE70D25DDE70D25DBE755AAFFFFEF
:10BA7800525261417272416138B50446FFF777FD51
:10BA8800054658B994F80032032B09D00022114614
:10BA980094F80102FFF7C6FA00B10125284638BD1F
:10BAA80094F80532012BF1D14FF4007200212046A1
:10BAB800FFF754FB552384F8FE31AA2384F8FF319D
:10BAC8005223237063706123A3704122E2707221B4
:10BAD80084F8E41184F8E51184F8E62184F8E73164
:10BAE800D4F8103284F8E831C3F3072284F8E92146
:10BAF800C3F3074284F8EA211B0E84F8EB31D4F82B
:10BB08000C3284F8EC31C3F3072284F8ED21C3F337
:10BB1800074284F8EE211B0E84F8EF31D4F81C227A
:10BB28000132C4F82C220123214694F80102FFF7C0
:10BB38006DFA002384F80532A8E70239D0F81432E8
:10BB4800023B8B4206D990F80232D0F8280201FB5A
:10BB5800030070470020704701295CD9F8B50546F5
:10BB68000C46D0F814328B4257D990F80032022B89
:10BB780029D0032B37D0012B51D101EB5106D0F836
:10BB8800201201EB5621FFF721FD10B14FF0FF30D5
:10BB980044E0771CC6F30806AE5DD5F8201201EB29
:10BBA80057212846FFF712FD00283AD1C7F30807A6
:10BBB800EB5D46EA032014F0010F01D000092DE0E7
:10BBC800C0F30B002AE0D0F8201201EB1421FFF794
:10BBD800FDFC48BB640004F4FF742B195B78285DF6
:10BBE80040EA03201AE0D0F8201201EBD411FFF745
:10BBF800EDFCE0B9A40004F4FE742B19DA78987807
:10BC0800000440EA02605B7840EA03202B5D184399
:10BC180020F0704002E0012070470120F8BD0120AB
:10BC2800FCE74FF0FF30F9E74FF0FF30F6E74FF051
:10BC3800FF30F3E7F8B50746A0F80612D0F8084237
:10BC4800012C44D00E46D0F80032D3F81422A24278
:10BC58003FD9F4B993F80022032A17D0CCB9B3F826
:10BC68000822B24237D9D3F82402C7F80C42D0B31D
:10BC780000EB1610C7F81002D7F8003206F00F01D3
:10BC880003EB4113C7F814320020F8BDD3F824425F
:10BC9800E4E793F802522D01AE4212D32146D7F8B9
:10BCA8000002FFF759FF0446B0F1FF3F15D0012805
:10BCB80015D9D7F80032D3F81432834211D9761B3C
:10BCC800EAE72146D7F80002FFF737FFCDE7022061
:10BCD800DBE70220D9E70220D7E70120D5E70220D9
:10BCE800D3E70220D1E70220CFE701297CD92DE94B
:10BCF800F04105460C461646D0F814328B4275D9E9
:10BD080090F80032022B3CD0032B4DD0012B70D180
:10BD180001EB5107D0F8201201EB5721FFF756FC31
:10BD2800002864D107F10108C7F3080714F00104DB
:10BD38001DD0EB5D03F00F0343EA0613DBB2EB55AE
:10BD4800012385F80432D5F8201201EB5821284642
:10BD5800FFF73CFC00284AD1C8F308084CB1C6F3E9
:10BD6800071305F80830012385F804323FE0F3B2E1
:10BD7800E5E715F80830C6F3032223F00F03134351
:10BD8800EFE7D0F8201201EB1421FFF71FFC70BB7E
:10BD9800640004F4FF742B192E55C6F307225A7059
:10BDA800012385F8043222E0D0F8201201EBD411E7
:10BDB800FFF70CFCD8B9A40004F4FE742919CA785A
:10BDC8008B781B0443EA026303F0704333432E5518
:10BDD800C6F307224A70C6F307428A701B0ECB705F
:10BDE800012385F8043202E0022070470220BDE8F2
:10BDF800F0810220FBE7F8B505460F4641B9D0F8B7
:10BE08000C629EB1D0F81432B34210D801260EE06D
:10BE1800FFF7A2FE034601284BD9B0F1FF3F4DD0F2
:10BE2800D5F81422824249D83E4600E0012634461D
:10BE38000CE021462846FFF78FFE034678B1B0F1A3
:10BE4800FF3F3BD0012839D0B44236D00134D5F871
:10BE58001432A342EDD8012E2DD90224E9E76FF060
:10BE6800704221462846FFF740FF0346D0B997B9EC
:10BE7800C3B9C5F80C42D5F81032B3F1FF3F1FD053
:10BE8800013BC5F8103295F8053243F0010385F8F7
:10BE98000532234612E0224639462846FFF725FF99
:10BEA8000346E5E7012B01D0012307E04FF0FF33FC
:10BEB80004E0012302E0002300E000231846F8BD57
:10BEC8002346FBE72DE9F843B0F806526B1C9AB2FB
:10BED800002A00F0838004460F46D0F81022002A7A
:10BEE8007ED013F00F060BD10132C0F81022D0F823
:10BEF8000C1289B9D0F80022B2F808229A4271D9F6
:10BF08000135A4F80652D4F8003203EB4613C4F8FE
:10BF180014320020BDE8F883D0F8000290F802221D
:10BF2800013A12EA1318EBD1FFF716FE81460128F1
:10BF38005AD9B0F1FF3F59D0D4F80002D0F81432E2
:10BF48004B4541D8002F53D0D4F80C12FFF753FFBC
:10BF5800814600284ED001284ED0B0F1FF3F4DD089
:10BF6800D4F80002FFF703FB08B10120D2E74FF431
:10BF780000720021D4F80002FFF7F0F8D4F800723C
:10BF880049463846FFF7D9FDC7F82C02D4F80032E5
:10BF980093F80222424511D9012283F80422D4F8E9
:10BFA8000002FFF7E4FA58BBD4F80022D2F82C328A
:10BFB8000133C2F82C3208F10108E7E7D3F82C2244
:10BFC800A2EB0802C3F82C22C4F80C924946D4F814
:10BFD8000002FFF7B2FDC4F8100291E7042099E7C8
:10BFE800042097E7042095E7022093E7012091E7D2
:10BFF80004208FE707208DE702208BE7012089E7DF
:10C00800012087E738B504460021FFF713FE0546EF
:10C0180040B1284638BD00212046FFF753FF0546AA
:10C028000028F6D1D4F81012D4F80002FFF7CEFA9F
:10C0380005460028EDD1D4F8140203785BB1C37A21
:10C0480013F0080FE7D10B22D4F81812FFF78EF877
:10C058000028E0D1DDE70425DBE710B582B004460F
:10C0680001910B782F2B01D05C2B01D1013101916B
:10C078000023C4F80832019B1B781F2B1DD901A986
:10C088002046FFF7C1F90346F8B92046FFF7BAFF83
:10C09800D4F81832DA7A0346D0B912F0040F14D162
:10C0A800D4F81412CB7A13F0100F18D0D4F8000279
:10C0B800FFF78EF9C4F80802E1E700212046FFF7F0
:10C0C800B9FD03460022C4F81422184602B010BD78
:10C0D8000428FAD112F0040FF7D10523F5E7052358
:10C0E800F3E770B504460E460021FFF7A3FD0246AC
:10C0F800D8B9002508E00135B54216D001212046FF
:10C10800FFF7E0FE024680B9D4F81012D4F8000216
:10C11800FFF75CFA024640B9D4F814321B78E52BD5
:10C12800E9D0002BE7D00025E8E7042A01D0104623
:10C1380070BD0722FBE738B504460121FFF7D1FFA0
:10C14800054608B1284638BDD4F81012D4F80002C4
:10C15800FFF73CFA05460028F4D120220021D4F844
:10C168001402FEF7FBFF0B22D4F81812D4F81402BD
:10C17800FEF7EAFFD4F80032012283F80422E1E74F
:10C18800F8B501292DD904460D46D0F814328B4252
:10C198002AD9002700E03546D4F81432AB4221D919
:10C1A80029462046FFF7D8FC0646D8B101281DD0FD
:10C1B800B0F1FF3F1CD0002229462046FFF795FD2D
:10C1C800074678B9D4F81032B3F1FF3FE3D0013312
:10C1D800C4F8103294F8053243F0010384F80532AC
:10C1E800D9E702273846F8BD0227FBE70227F9E717
:10C1F8000127F7E770B584B00190009116460391C6
:10C2080003A8FFF78BF9041E1DDB114B53F82450CC
:10C218002DB12846FFF7A6F8002385F80032019BC8
:10C2280013B1002283F80022094A42F8243063B18E
:10C23800012E02D0002004B070BD0022694601A87A
:10C24800FFF744FAF7E70B20F5E70020F3E700BF14
:10C25800A01400202DE9F043ADF50F7D01910028D1
:10C2680000F0E580144606460023C0F8003202F0CC
:10C278001F0802F01E073A4601A986A8FFF726FA0A
:10C28800054620B128460DF50F7DBDE8F08303ABC8
:10C298008C93019906A8FFF7E0FEDDF82C9205467D
:10C2A80048B9B9F1000F5AD0391E18BF012106A8A4
:10C2B800FEF774FF054614F01C0F00F0A480002D53
:10C2C80059D0042D4DD048F00808DDF82C9215B946
:10C2D80018F0080F5BD1002DD4D118F0080F01D049
:10C2E80048F02008869BD3F82C32C6F81C32C6F8D2
:10C2F8002092B8F1010F94BF0021012106A8FEF792
:10C30800A5FFC6F82802002800F0938086F8068268
:10C31800002486F80742869F49463846FFF758F8B2
:10C32800C6F8100299F81F2099F81E301B0443EA3A
:10C33800026399F81D2043EA022399F81C2013434D
:10C34800C6F80C32C6F80842C6F81842C6F82442A5
:10C35800C6F80072B7F80632A6F8043292E7062546
:10C36800A9E7FEF761FF08B91225ACE706A8FFF7B1
:10C37800E2FE0546A7E799F80B3013F0110F04D138
:10C3880014F0040FA3D00825A1E707259FE7FDF7C0
:10C3980059FB89F80E00C0F3072389F80F30C0F362
:10C3A800074389F81030000E89F81100002489F835
:10C3B8000B4089F81C4089F81D4089F81E4089F80F
:10C3C8001F4049468698FFF703F807462146484626
:10C3D800FFF70FF88698012380F80432002F3FF406
:10C3E8007AAFD0F82C423946FFF7CAFE0546002836
:10C3F8007FF471AF8698013FC0F80C722146FFF7B1
:10C40800E5F8054667E7002D7FF465AF99F80B302E
:10C4180013F0100F09D114F0020F3FF45CAF13F0C2
:10C42800010F3FF458AF072555E7042553E70925C1
:10C4380028E7022526E72DE9F04F83B004460F468A
:10C44800164698460023C8F80030FFF725F90190F2
:10C45800002840F0D18094F807320193002B40F077
:10C46800CB8094F8063213F0010F00F0D780D4F88F
:10C478000C52D4F80832ED1AB54276D3354674E03A
:10C48800D4F824321BB12046FEF78EFF83E0D4F89F
:10C498001412FFF761FB7EE04FF0020A84F807A24E
:10C4A800CDF804A0A8E04FF0010A84F807A2CDF85F
:10C4B80004A0A1E04FF0020A84F807A2CDF804A076
:10C4C8009AE094F8063213F0400F05D0D4F8180219
:10C4D800A0EB0900504502D34FEA4A2639E04FF451
:10C4E8000072214607EB4020FEF72EFEF4E7D4F851
:10C4F80018224A451DD094F8063213F0400F0DD08B
:10C50800012321469BF80102FEF780FD002877D120
:10C5180094F8063223F0400384F80632D4F8000277
:10C5280001234A46214690F80102FEF763FD0028E0
:10C538006DD1C4F81892D4F80812C1F30801C1F5F6
:10C548000076B54200D22E46324621443846FEF7E0
:10C55800FBFD3744D4F808323344C4F80832D8F81D
:10C5680000303344C8F80030AD1B002D44D0D4F857
:10C578000812C1F30803002BDDD1D4F8000290F8AB
:10C588000262013EF6B216EA51260CD100297FF468
:10C5980077AFD4F8100201287FF67EAFB0F1FF3FE5
:10C5A80081D0C4F81402D4F800B2D4F81412584652
:10C5B800FFF7C3FA814600283FF47CAFB1444FEA45
:10C5C800552AB5F5007F92D306EB0A039BF80222A1
:10C5D800934201D9A2EB060A53464A4639469BF8CC
:10C5E8000102FEF707FD00283FF46BAF4FF0010A88
:10C5F80084F807A2CDF804A0019803B0BDE8F08F35
:10C608004FF0010A84F807A2CDF804A0F4E74FF030
:10C61800010A84F807A2CDF804A0EDE707230193E7
:10C62800EAE72DE9F04F83B004460F4615469846D1
:10C638000023C8F80030FFF72FF80190002853D1E5
:10C6480094F807320193002B4ED194F8063213F078
:10C65800020F00F00081D4F80832EB42C0F0BF802E
:10C668000025BCE0D4F82432002B41D02046FEF748
:10C678009BFE0346002B00F0DF80012B3ED0B3F178
:10C68800FF3F42D0C4F81432D4F810220AB9C4F8D3
:10C69800103294F8063213F0400F3DD1D4F800B2AE
:10C6A800D4F814125846FFF748FA814600284CD0AF
:10C6B800B1444FEA552AB5F5007F64D306EB0A0367
:10C6C8009BF80222934201D9A2EB060A53464A4636
:10C6D80039469BF80102FEF799FCE8B34FF0010ACE
:10C6E80084F807A2CDF804A0019803B0BDE8F08F44
:10C6F800D4F81412FFF77FFB0346BBE74FF0020A9A
:10C7080084F807A2CDF804A0EEE74FF0010A84F8F8
:10C7180007A2CDF804A0E7E7D4F800020123D4F873
:10C728001822214690F80102FEF770FC30B994F8FF
:10C73800063223F0400384F80632AFE74FF0010ACF
:10C7480084F807A2CDF804A0CEE74FF0020A84F8D7
:10C7580007A2CDF804A0C7E7D4F81812A1EB090185
:10C76800514502D34FEA4A262DE04FF4007207EBF9
:10C7780041212046FEF7E8FC94F8063223F04003F6
:10C7880084F80632EEE7D4F818324B4505D0D4F8D1
:10C798000822D4F80C329A423ED3C4F81892D4F83E
:10C7A8000802C0F30800C0F50076B54200D22E4654
:10C7B800324639462044FEF7C7FC94F8063243F067
:10C7C800400384F806323744D4F808323344C4F8B6
:10C7D8000832D8F800303344C8F80030AD1B5DB3D8
:10C7E800D4F80812C1F30803002BD8D1D4F80002FA
:10C7F80090F80262013EF6B216EA51267FF449AF7C
:10C8080000297FF42FAFD4F81032002B7FF435AF16
:10C81800FFF7F1FA03462DE701234A4621469BF824
:10C828000102FEF7E7FB0028B7D04FF0010A84F8B1
:10C8380007A2CDF804A057E7D4F80832D4F80C22A0
:10C84800934201D9C4F80C3294F8063243F020031D
:10C8580084F8063248E70723019345E738B50446CC
:10C86800FEF71AFF00BB94F8063213F0200F1BD016
:10C8780013F0400F11D0D4F800020123D4F8182285
:10C88800214690F80102FEF7C1FB002843D194F835
:10C89800063223F0400384F80632D4F81C12D4F888
:10C8A8000002FEF793FE00B138BDD4F82052EB7AAF
:10C8B80043F02003EB7294F80C322B77B4F80C3267
:10C8C8001B0A6B7794F80E32AB7794F80F32EB773C
:10C8D800D4F810122846FEF78CFDFDF7B3F8A875BA
:10C8E800C0F30723EB75C0F307432B76000E687679
:10C8F8000023AB74EB7494F8063223F0200384F819
:10C908000632D4F80032012283F80422D4F8000257
:10C91800FFF7B2F8C8E70120C6E710B50446FFF7ED
:10C928009DFF00B110BD2046FEF7B6FE0028F9D1E4
:10C93800D4F82802FEF7F0FC0028F3D1C4F800026E
:10C94800F0E72DE9F84F04460D46FEF7A5FE06462A
:10C95800002840F0798194F80732002B40F0738169
:10C96800D4F82432002B00F09D80B5F1FF3F4BD066
:10C97800D4F80C72AF4200D32F46C4F80872002FC7
:10C9880000F0628107F1FF3841462046FEF70CFDB2
:10C998000146C4F81402D4F800522846FFF7CDF82F
:10C9A800002873D095F80212013901EA582101EBE9
:10C9B8000008C7F30807002F00F04681D4F81822B2
:10C9C800424500F0418194F8063213F0400F0DD033
:10C9D8000123214695F80102FEF718FB002859D1DA
:10C9E80094F8063223F0400384F80632D4F80002A3
:10C9F80001234246214690F80102FEF7FBFA00287F
:10CA08004CD1C4F818821FE1984658F804BBD4F8F2
:10CA180010A2BAF1000F2CD04FF0020909F1020957
:10CA28005146002701370D46D4F80002FFF794F865
:10CA38000146012815D9B0F1FF3F16D001358542CE
:10CA4800F0D0CB4505D3434643F8087BC8F804A08B
:10CA58009846D4F80032D3F814328B420BD98A4660
:10CA6800DCE7022684F80762EEE0012684F8076214
:10CA7800EAE04FF00209D4F82432C3F80090D9450F
:10CA880000F2E5800023C8F80030DDE0022684F8D3
:10CA98000762D9E0012684F80762D5E0012684F808
:10CAA8000762D1E0D4F80C32AB4205D294F80622E2
:10CAB80012F0020F00D11D46D4F808320022C4F843
:10CAC80008220DB3D4F8000290F802824FEA4828F1
:10CAD80083B16A1EB2FBF8F2013BB3FBF8F18A425C
:10CAE80008D3C8F100021340C4F80832EF1AD4F88A
:10CAF800145207E0D4F81032002B3FD0C4F8143297
:10CB08002F461D46002D67D1D4F80832C3F3080319
:10CB18002BB3D4F81822AA4221D094F8063213F085
:10CB2800400F0FD0D4F800020123214690F80102EB
:10CB3800FEF76CFA00287ED194F8063223F0400301
:10CB480084F80632D4F8000201232A46214690F8D8
:10CB58000102FEF74FFA002871D1C4F81852D4F830
:10CB68000832D4F80C2293426ED9C4F80C3294F8E7
:10CB7800063243F0200384F8063265E00021FFF70F
:10CB88003AF90346012805D0B0F1FF3F06D0C4F8B2
:10CB98001002B3E7022684F8076255E0012684F8FC
:10CBA800076251E02946D4F80002FEF7D5FF054692
:10CBB800B5F1FF3F31D0012D33D9D4F80032D3F885
:10CBC8001432AB422DD9C4F81452D4F80832434475
:10CBD800C4F80832A7EB080747450DD994F8063280
:10CBE80013F0020FDED02946D4F80002FFF703F94C
:10CBF80005460028DCD14746D4F808323B44C4F83F
:10CC08000832C7F30803A3B12946D4F80002FEF797
:10CC180094FF50B100EB572576E7012684F80762A8
:10CC280012E0022684F807620EE0022684F8076202
:10CC38000AE01D4668E7012684F8076204E0012639
:10CC480084F8076200E01E463046BDE8F88F1126DA
:10CC5800FAE730B587B00191002848D00446002291
:10CC680001A905A8FEF732FD054628B10023C4F83E
:10CC78000032284607B030BD059BC4F8003202AB2D
:10CC8800C4F8183201992046FFF7E7F9054638BB82
:10CC9800D4F8141241B1CB7A13F0100F1FD00598B5
:10CCA800FEF796FBC4F80802059BB3F80632A4F811
:10CCB800043200212046FEF7BDFF054680B9D4F8AE
:10CCC80008321BB90023C4F81C3209E000212046B1
:10CCD800FEF7BCFAC4F81C0210B9122502E00525BB
:10CCE800042D02D0002DC4D0C0E70525BEE70925D4
:10CCF800BFE72DE9F04FADF5117D0390FCF7A2FEDB
:10CD08000446012203A988A8FEF7E0FC054620B1E5
:10CD180028460DF5117DBDE8F08F05AB8E9303997C
:10CD280008A8FFF79AF9002800F09F80042801D08E
:10CD38000546EDE700218898FFF75DF8064618B12B
:10CD4800012802D1022504E00725B6F1FF3F00F0D3
:10CD58008A8025B131468898FFF712FAD8E7889873
:10CD6800FEF705FC05460028F4D1DDF8208231469F
:10CD78004046FEF7E2FE07464FF4007200214046A7
:10CD8800FEF7ECF90B2220214046FEF7E7F94FF0B9
:10CD98002E0B88F800B0102388F80B305FFA84FA5D
:10CDA80088F816A0C4F3072988F81790C4F3074336
:10CDB800019388F81830230E029388F81930314609
:10CDC8004046FEF716FB08F1200420224146204683
:10CDD800FEF7BAF988F821B08A99889B93F800225F
:10CDE800032A1CD02046FEF704FB889B93F80242D6
:10CDF800DCB107F1010B8898C0F82C72012380F888
:10CE08000432FEF7B4FB054678B94FF400720021EE
:10CE18004046FEF7A3F9013CE4B25F46E8E7D3F8E1
:10CE280024328B42DED10021DCE7002D92D108A804
:10CE3800FFF781F9054600288CD18D981023C3721D
:10CE480080F816A080F81790019B0376029B437622
:10CE58003146FEF7CEFA8898012380F80432FEF7AF
:10CE68000BFE054654E7012574E7082550E7000046
:10CE7800134B5B7ADBB2012B01D90120704710B448
:10CE880004460F4B93F809C05FFA8CFC002003F8A6
:10CE98000C0093F809C003EB8C0CCCF804405C7AC6
:10CEA8001C4422725A7A541CE4B25C7230320A7002
:10CEB8003A234B702F238B70C87010BC704700BF8B
:10CEC800A414002008B50022FFF7D2FF08BD000017
:10CED80008B500220F491048FDF7A5FB70B90F49A6
:10CEE8000D48FDF7B7FB60B90D490B48FCF72EFF5D
:10CEF80050B90948FDF7B5FB48B908BDF4F770FB10
:10CF0800EDE7F4F76DFBEFE7F4F76AFBF1E7F4F709
:10CF180067FBF2E7FC000020B01400208C00002022
:10CF28001801002012230B8000487047E8000020F9
:10CF380004230B8000487047E4000020002393423C
:10CF48001ED200B510E00CF1370C01F813C0000137
:10CF58004FEA430C0CF1010C4FF0000E01F80CE005
:10CF68000133DBB2934209D24FEA107CB0F1204F73
:10CF7800E9D20CF1300C01F813C0E8E75DF804FBC6
:10CF88007047000038B50B4BD3F8E807D3F8EC47E7
:10CF9800D3F8F037C01800D138BD074D082229460C
:10CFA800FFF7CCFF042205F110012046FFF7C6FF6A
:10CFB800F2E700BF00F0FF1FCA00002008B51A23DF
:10CFC8000B80FFF7DFFF014808BD00BFC800002045
:10CFD80008B50A4628B905490548FDF79AFF0348E8
:10CFE80008BD02490248FDF794FFF8E774170020CE
:10CFF80010A4010810B50A46034C21460348FDF762
:10D0080088FF204610BD00BF7417002024A4010823
:10D0180008B50A4628B905490548FDF77AFF0348C7
:10D0280008BD02490248FDF774FFF8E774170020AD
:10D0380038A4010808B50A4628B905490548FDF786
:10D0480068FF034808BD02490248FDF762FFF8E798
:10D058007417002044A40108034B586D08609B6DA9
:10D0680013800020704700BFF008002000207047A0
:10D07800002070470020704770B5084615461E46C8
:10D088000B4B32462946FCF7EFFC38B9094CFCF744
:10D09800FBFC18B1601E44B10446F8E73246294645
:10D0A800054801F0A3FE002070BD0220FCE700BF88
:10D0B80000E1F505A086010054A4010870B50846F2
:10D0C80015461E460B4B32462946FCF7BDFC38B9BF
:10D0D800094CFCF7D9FC18B1601E44B10446F8E7C6
:10D0E80032462946054801F081FE002070BD022025
:10D0F800FCE700BF00E1F505A086010080A4010857
:10D1080008B5044801F0D2FEFCF7D8FC00B908BD08
:10D118000220FCE7ACA40108022805D8DFE800F0EB
:10D1280005040200012070470220704702680E4B78
:10D138009A4200D0704700B583B003F5DA33DA6954
:10D1480042F40002DA61DB6903F400030193019BF6
:10D15800002203211420F7F765F81420F7F772F876
:10D1680003B05DF804FB00BF005C004008B500F5A3
:10D178002C71D0F8EC02FDF78CFA08BD08B501EB6C
:10D18800810300EBC303D3F87C21D0F8EC02FDF750
:10D19800ADFA08BD08B501EB810300EBC303DA6BF8
:10D1A800D0F8EC02FDF7E8FA08BD08B5D0F8EC02B3
:10D1B800FDF789FB08BD10B504468368022B09D129
:10D1C8000121D4F8EC02FDF767FBD4F8EC02FDF777
:10D1D8003BFB10BDF4F704FAF2E7000010B5044673
:10D1E800D0F8EC02FDF75BFBA36923B1024A13698F
:10D1F80043F00603136110BD00ED00E008B5D0F858
:10D20800EC02FDF755FB08BD10B504461948C0F8F7
:10D21800EC42C4F8C002184B0360082343600223A1
:10D22800836000238361C3610362F7F7DDFCE8B91B
:10D23800182300221146D4F8C002F8F75DFC5823E1
:10D2480000228021D4F8C002F8F756FC9823002267
:10D258008121D4F8C002F8F74FFCD823002201211D
:10D26800D4F8C002F8F748FC002010BDF4F7B8F96C
:10D27800DEE700BFE41B0020005C004008B5D0F8E2
:10D28800C002F7F739FDFFF747FF08BD08B5944618
:10D298001A466346D0F8C002F8F7E4FAFFF73CFFF5
:10D2A80008BD08B5D0F8C002F8F71AFBFFF734FF3D
:10D2B80008BD08B5D0F8C002F8F703FCFFF72CFF4B
:10D2C80008BD08B5D0F8C002F8F784FBFFF724FFC3
:10D2D80008BD08B5D0F8C002F8F7B8FBFFF71CFF87
:10D2E80008BDD0F8C03211F0800F08D101F07F01DD
:10D2F80001EB810103EBC10393F86A01704701F068
:10D308007F01013101EB810103EBC103987870477C
:10D3180008B5D0F8C002F8F7B9F9FFF7FDFE08BD67
:10D3280008B5D0F8C002F8F733FBFFF7F5FE08BDE3
:10D3380008B5D0F8C002F8F705FBFFF7EDFE08BD09
:10D3480008B5D0F8C002F8F71AFB08BD00487047C6
:10D358007419002070477047024B0146186800F0A6
:10D368000BB800BFC0060020024B0146186802F047
:10D3780093BB00BFC00600202DE9F04F01F10B055B
:10D38800162D064683B024D8102900F2AD8000F08F
:10D39800A7FA102518234FF0020CB84F3B445C68DD
:10D3A800A3F10802944200F01D8130466368E268E8
:10D3B800A16823F00303CA60234491605A680834C3
:10D3C80042F001025A6000F091FA204603B0BDE82D
:10D3D800F08F35F0070500F18780A94200F28480BC
:10D3E80000F07EFAB5F5FC7FC0F06F816B0A7FD044
:10D3F800042B00F21E81AB0903F1390C03F1380E3E
:10D408004FEACC009D4F384444680838A04207D101
:10D418000DE0002AE16880F2DF80884207D00C46E0
:10D42800636823F003035A1B0F2AF2DDF446DFF882
:10D4380050823C69444500F0BC80636823F00309CE
:10D44800A9EB05030F2B00F34581002BC7E90488DE
:10D4580080F22F81B9F5007FD7F804E080F0C98009
:10D4680001234FEAD9014FEA5919194403FA09F37C
:10D4780057F831204EEA030E07EBC103083BA260C0
:10D48800E360C7F804E047F83140D46001204FEA70
:10D49800AC039840704532D810EA0E0F07D12CF033
:10D4A800030C400010EA0E0F0CF1040CF9D007EB46
:10D4B800CC0AD646E146DEF80C300BE059681C462B
:10D4C80021F003014A1B0F2ADB6800F3BF80002A02
:10D4D80080F2E2809E45F1D109F1010919F0030FAC
:10D4E8000EF1080EE7D11FE10C23336000246CE72E
:10D4F8004FF400704FF0400C4FF03F0E82E7BC68CD
:10D50800636823F00309A94503D3A9EB05030F2B8F
:10D5180052DC5C4B08201B6803F1100804EB09037C
:10D52800009302F007FA584A83461368A844013367
:10D5380005D008F1FF388044434203EA0808414611
:10D54800304602F099F9B0F1FF3F82464E4A00F0AA
:10D55800DC8004EB0903834200F2D5804B4B0BF1CE
:10D56800FF31186840448446186040F0FB801AEA8E
:10D57800010F40F0F780D7F808A0C84448F001022E
:10D58800CAF804205446424B1968814238BF1860D3
:10D59800404B1968814238BF186022F00308A8453B
:10D5A800A8EB050301D30F2B06DC304600F09EF9EB
:10D5B8009CE7D7F804E069E7621943F0010345F0F6
:10D5C800010565603046BA600834536000F08EF992
:10D5D800204603B0BDE8F08FA2683046D1602344EE
:10D5E8008A60EBE6DC68A3427FF4DFAE0CF1020C44
:10D5F8001DE7B9F5206F4FEA59227DD3142A00F2AE
:10D60800118102F15C03DB005B32F918FB58083921
:10D61800994203D1ECE09B68994204D05A6822F001
:10D6280003024A45F7D8D968C4E902318C60DC6046
:10D638002CE7142B6CD9542B00F2FD802B0B03F133
:10D648006F0C03F16E0E4FEACC00DBE6D4F808C08D
:10D658003046661945F001056560CCF80C30C3F812
:10D6680008C042F00103C7E90466C6E9028873608E
:10D67800625000F03BF90834A7E600BF40010020E3
:10D6880048010020041F002038010020D41E00207B
:10D69800001F0020FC1E002021444A68304642F04A
:10D6A80001024A6054F8082FD3609A6000F01EF90E
:10D6B8008BE6A144D9F80430304643F00103C9F899
:10D6C800043000F013F908347FE64FEAD50C05F171
:10D6D800080362E6621943F0010145F0010565603F
:10D6E8003046C7E90422C2E90288516044F809308B
:10D6F80000F0FCF8083468E64FEA991202F13903A1
:10D70800DB00383281E7BC4224D0BC68626844E759
:10D7180003F15C0C03F15B0E4FEACC0072E65AF899
:10D728000839534540F0D8801CF0030F0CF1FF3C3A
:10D73800F5D17B6823EA00037B60400098423FF6FE
:10D74800DEAE18B9DBE6400009F104091842FAD048
:10D75800CC46ACE6614B0BF1FF31186808EB000CC6
:10D76800C3F800C01068013070D004EB0902AAEBBE
:10D77800020262441A601AF00702CDE9002340D081
:10D78800C2F108029244D04408EA01005A44121A2D
:10D7980002EA010B5946304602F06EF8421C019B22
:10D7A80071D0A0EB0A0000EB0B08186848F00102E2
:10D7B8005844BC42C7F808A01860CAF804203FF4CF
:10D7C800E1AEB9F10F0F44D94FF0050C6168A9F12A
:10D7D8000C0222F0070201F00101114361600F2AD7
:10D7E80004EB0201C1E901CC55D8DAF80420C9E6F6
:10D7F8000120921000FA02F24EEA020EC7F804E085
:10D8080012E70AEB08020A40ABEB020202EA010B3C
:10D818005946304602F030F8431C019BC1D1DDF86F
:10D8280000B0C2E7542A18D84FEA193202F16F0340
:10D83800DB006E32E9E6B3F5AA7F18D8EB0B03F1EB
:10D84800780C03F1770E4FEACC00DBE5C2F800A0B4
:10D8580091E70123CAF80430A7E6B2F5AA7F25D8D4
:10D868004FEAD93202F17803DB007732CDE640F295
:10D878005452934225D8AB0C03F17D0C03F17C0E76
:10D888004FEACC00BEE5009A4FF0000B083A9044EE
:10D89800A8EB0A0889E7304604F10801009302F072
:10D8A800FBF8009BD7F808A018689EE740F254538D
:10D8B8009A420DD84FEA994202F17D03DB007C328F
:10D8C800A3E64FF47E704FF07F0C4FF07E0E99E583
:10D8D8004FF47E737E2298E67B682EE7D41E0020E4
:10D8E800014802F023B800BF48200020014802F098
:10D8F8001FB800BF4820002003460A4602490868AE
:10D90800194600F003B800BFC00600202DE9F84F03
:10D918001646002900F096800C46804606F10B0555
:10D92800FFF7DEFF54F8041C162DA4F1080921F0B6
:10D93800030758D81025AE4258D8AF4260DABF4B1B
:10D9480009EB070C9A68DCF80400624500F0908047
:10D9580020F0010363445B68DB0768D420F0030010
:10D968003B189D4247DDCB0712D454F8083CA9EB7D
:10D97800030BDBF8043023F00302104400EB070A22
:10D98800554540F3F68007EB020A554540F3CC8035
:10D9980031464046FFF7F0FC0646002800F021819A
:10D9A80054F8043CA0F1080223F001034B449342CD
:10D9B80000F0B4803A1F242A00F2D780132A00F21C
:10D9C800A28003462246116819605168596092681E
:10D9D8009A602146404602F05FF84046FFF786FF0E
:10D9E8003046BDE8F88F35F00705A4D50C23C8F8F4
:10D9F8000030002618E01F46DCE90223D3609A6055
:10DA0800D9F804307A1B0F2A03F0010309EB070049
:10DA18001DD83B43C9F80430436843F00103436011
:10DA28004046FFF763FF26463046BDE8F88FC90732
:10DA3800AED454F8083CA9EB030BDBF8043023F010
:10DA48000302A0E71146BDE8F84FFFF795BC2B434A
:10DA580009EB050142F00102C9F804304A60436845
:10DA6800083143F001034360404602F015F8D7E758
:10DA780020F00300C21905F1100C624580F2928073
:10DA8800CA0785D454F8082CA9EB020BDBF804204C
:10DA980022F00302104400EB070AD4453FF773AFA6
:10DAA8005E46DBF80C1056F8080F3A1F242AC160AE
:10DAB800886000F2B080132A40F2AB8021681B2AEC
:10DAC800CBF808106168CBF80C1000F2AA80083473
:10DAD8000BF110022168116061685160A1689160C2
:10DAE800AAEB05020BEB050142F0010299604A60BE
:10DAF800DBF80430404603F001032B43CBF8043035
:10DB0800FFF7F4FE90E723681B2A0360636843600D
:10DB18003DD804F1080200F1080354E750F8043C2A
:10DB280023F003031F446BE75E463A1FDBF80C3013
:10DB380056F8081F242ACB60996023D8132A1FD9C6
:10DB480023681B2ACBF808306368CBF80C303CD824
:10DB580008340BF1100322681A6062685A60A268E0
:10DB68009A6034465746D9464AE7214601F010FBE9
:10DB78002FE7DCE902135E46CB603A1F9960D5E7D0
:10DB88003346E8E72146304601F002FBE9E7A3689F
:10DB9800242A8360E368C36027D004F1100200F1EF
:10DBA800100310E7521B09EB050142F001029960CE
:10DBB8004A6054F8043C404603F001032B4344F800
:10DBC800043CFFF793FE26462EE7A368242ACBF8E9
:10DBD8001030E368CBF8143010D010340BF1180370
:10DBE800B9E74046FFF782FE03E7236904F118020C
:10DBF80003616369436100F11803E4E6236918349B
:10DC0800CBF8183054F8043CCBF81C300BF1200347
:10DC1800A1E732465EE72146304601F0B9FA074BE4
:10DC28005EE7A168242ACBF81010E168CBF814103D
:10DC380006D010340BF118024CE700BF4001002059
:10DC480022691834CBF8182054F8042CCBF81C207F
:10DC58000BF120023EE700BF2DE9F04F9FB0884648
:10DC68000792002100220024CDE904128346414690
:10DC78001A9419910F4611F8012B2D2A5ED801A08C
:10DC880050F822F063DE000845DD000845DD000895
:10DC980045DD000845DD000845DD000845DD0008D4
:10DCA80045DD000845DD00087BDC00087BDC00085A
:10DCB8007BDC00087BDC00087BDC000845DD000815
:10DCC80045DD000845DD000845DD000845DD0008A4
:10DCD80045DD000845DD000845DD000845DD000894
:10DCE80045DD000845DD000845DD000845DD000884
:10DCF80045DD000845DD000845DD000845DD000874
:10DD080045DD00087BDC000845DD000845DD00082E
:10DD180045DD000845DD000845DD000845DD000853
:10DD280045DD000845DD000845DD000845DD000843
:10DD3800E5E3000845DD0008F9E300080021089143
:10DD4800302A00F09580002309932F2A144640F2C8
:10DD5800EF844FF0000938464E464D4613E0013037
:10DD6800082D1990C8BF09EB89090478C6BF02EBD2
:10DD78004902A2F13009A3F130062F2C224605F101
:10DD8800010540F3B48006EB8603392C02EB43030C
:10DD9800E5DD0122AB4901F0C9FA002879D1199AC9
:10DDA8001346013219925C78002D40F08D85302C95
:10DDB80040F03B8513461846013319931C78302CE4
:10DDC800F9D0C2F101021044A4F13103082B37D86D
:10DDD800199F012539464FF0000A431CA4F1300E63
:10DDE8000C93002006EB86060EEB46064B1C199397
:10DDF8004C78A4F13002092A00F2E082964619997B
:10DE08000130002AF2D00128D8BF05F1010C40F3F7
:10DE1800878400EB050C0CF1FF340A9703E07E00C1
:10DE2800AC4200F07C84082D06EB860705F101055D
:10DE3800F5DD102DDCBF09EB89094FEA4909EFE749
:10DE4800652C40F0D8824FF0000A0123CDF830A0AD
:10DE58000A93099B034340F0BF82079B00260027D3
:10DE68000BB1C3F80080304639461FB0BDE8F08FCB
:10DE78007A7802F0DF02582A00F0128401371997E5
:10DE88003A78302AFAD0002A00F0818201230993D7
:10DE98005BE70020AA460C900A90652C34D0452CEC
:10DEA80032D000231093002D7AD1099B034340F010
:10DEB8006E820A9B002BD0D1692C00F0898400F374
:10DEC8005F84492C00F084844E2CC6D15E4919A881
:10DED80002F004FA0028C0D0199B1B78282B00F008
:10DEE800A5855A4801F062FD06460F4651E2012217
:10DEF800544901F01BFA0028CBD1199BAA465A1C99
:10DF080019925C780C9074E7002DA2D0DDF864803B
:10DF180008F10103199398F801402B2C00F059825D
:10DF28002D2C00F04E824FF0000CA4F1300109298D
:10DF380000F23F82302C199B0AD1013319931C78C7
:10DF4800302CFAD0A4F13102082AAAD8A4F1300161
:10DF58005A1C19925C782F2C40F3FE8396460B933B
:10DF680008E0013219929EF80140A3F130012F2CEC
:10DF780006DD964601EB8103392C04EB4303F0DD03
:10DF88000B9BD21A082A40F3E78344F61F631093C9
:10DF9800BCF1000F87D0109B5B421093002D84D0FA
:10DFA8000C9A109BBAF1000F08BFAA469B1A102DB5
:10DFB80030460B932C46A8BF1024F2F707FB024605
:10DFC8000B46092DCDE9042316DD214B03EBC403D1
:10DFD80053E91223F2F7ECFE02464846904689467A
:10DFE800F2F7F4FA02460B4640464946F2F7B2F910
:10DFF8000F2DCDE904012DDC0B9B002B00F02083B5
:10E008000B9B40F35282162B40F3AD830B9AC5F15C
:10E01800250393421EDBDDE904230D4CC5F10F05F2
:10E0280004EBC501D1E90001F2F7C2FE0B9B5D1BB1
:10E0380004EBC504D4E90023F2F7BAFE06460F46FE
:10E04800A7E100BFBCA40108CCA401088CA2010868
:10E0580098DC01080B9B2C1B1C44002C40F3D1813D
:10E0680014F00F000AD0DDE90423354901EBC001A3
:10E07800D1E90001F2F79CFECDE9040134F00F0369
:10E0880040D0B3F59A7F00F3B883102B4FEA2314DE
:10E0980040F31E85DDE9040100232A4A09979046CA
:10E0A80099461746E20704D5D8E90023F2F780FE1F
:10E0B80001236410012C09F1010908F10808F1D1C4
:10E0C8003A46099F0BB1CDE90401059B02EBC90152
:10E0D800A3F154730593DDE90423D1E90001F2F7B4
:10E0E80067FE194B194A0B409342CDE9040100F22F
:10E0F8008483174A934240F241844FF0FF33154C12
:10E10800CDE9043400230A932B4652463946584633
:10E11800009602F07DFA1490002800F06E83109AA1
:10E128000C9B4FF0000A9B1A0B9ACDF824A0002AEA
:10E13800A8BF0023109322EAE2731593E5E000BF1D
:10E1480098DC010870DC01080000F07F0000A07C6A
:10E158000000907CFFFFEF7FD21A1F2AA4EB020475
:10E1680000F33282012393401E4600250A9BA044F7
:10E178004C44A14598444B46A8BF23464345A8BFF5
:10E188004346002B04DDE41AA8EB0308A9EB0309B6
:10E19800109B002B00F3BE81002C00F3D4810B9B55
:10E1A800002B00F30782B8F1000F00F3F781B9F1F3
:10E1B800000F08DD51464A46584602F00BFC8246DD
:10E1C800002800F0F4813A4658461A9902F098FC63
:10E1D8000990002800F0EB810023099AD168D360E8
:10E1E8001191514602F06CFC0028C0F2EA83DDF878
:10E1F800149000F076835146099802F01DFE002223
:10E208004FF0804304460D46F2F7C4FA002800F0A8
:10E218007181119B002B40F0E381049B002B40F09F
:10E228006B82C9F31303002B40F00D8200222046B5
:10E238002946A94BF2F7A4FA002840F04983204662
:10E24800A64B29460022F2F7B3FD03460C46CDE95A
:10E25800123401F100430E900F93DFF88482A14B32
:10E2680009EA08089845DDE90E4500F0C0810A9BD7
:10E278001BB3B8F1D46F20D895A3D3E90023DDE907
:10E288001201F2F787FAA0B1DDE91201F2F7A2FF55
:10E29800012838BF0120F2F799F9119BCDE9120145
:10E2A800002B40F0BD8201F1004316901793DDE981
:10E2B800164505F1D663A3EB0805DDE90C0102F06C
:10E2C800DBFC02460B4620462946F2F771FDDDE9E4
:10E2D8000C23F2F73FF80C46CDE904010A9B23B959
:10E2E8007F4B2340984500F0B78158461A9902F0B1
:10E2F80033F93946584602F02FF95146584602F08C
:10E308002BF95846099902F027F9149C5846616878
:10E3180002F0FCF80746002800F04981226904F160
:10E328000C01023292000C30F2F7CCFC1CAB0193CA
:10E338001BAB00935846DDE904341A46CDE90C348A
:10E34800234602F01BFD1A90002800F005810121E8
:10E35800584602F005FA8246002800F028811B9BE7
:10E36800002BC0F21581109ADDF8548003EB0209E6
:10E378000A9A1C9C9B1A23445B4A013B9342C4F1B2
:10E388003604FFF6E9AE012300251E46EEE6002618
:10E398000027079A0AB1199B1360089B002B3FF4CA
:10E3A80062AD07F100431F46304639461FB0BDE84D
:10E3B800F08F0023CDF86480109374E501230A934D
:10E3C8006BE54FF0010C08F10203199398F802402D
:10E3D800ABE54FF0000CF6E7002597E50022089220
:10E3E800791C19917A78002A3FF437AD0F46A7E4D3
:10E3F80001220892F4E7452C3FF425AD01230A9346
:10E4080053E53FF47FAE644214F00F020AD0DDE911
:10E418000401364B03EBC203D3E90023F2F7F2FD04
:10E42800CDE9040124113FF46DAE1F2C37DCDDE982
:10E43800040114F0100318BF6A230A930023DFF8BD
:10E44800B080E20704D5D8E90023F2F7B1FC012334
:10E45800641008F10808F4D10BB1CDE904010A9B56
:10E46800A3B1DDE90401C1F30A52C2F16B03002B29
:10E478000ADD1F2B40F339830020342B049040F32E
:10E488007C834FF05C7305936A230A930022DDE9CD
:10E4980004010023F2F76AF900283FF435AE22237D
:10E4A80000260027CBF8003073E71633FFF6D2AD0D
:10E4B800DDE904010C9B109A9A1A0C4B03EBC2037A
:10E4C800D3E90023F2F79EFD06460F4661E700BF39
:10E4D8000000C0FFFFFFDF410000F03F0000E03F09
:10E4E8000000F07F0000E07F02FCFFFF98DC0108DD
:10E4F80038DA0108AC4B204629460022F2F758FCCE
:10E50800119BCDE91201002B65D101F100430E905A
:10E518000F93A2E651461A46584602F001FA82467F
:10E52800002844D001461A9A584602F047F90028B4
:10E538003DD011901A99584602F00EF8119B002C04
:10E548001A937FF72CAE224658461A9902F042FADF
:10E558001A9000287FF423AEB946054622230026E8
:10E56800924FCBF800302946584601F0F5FF49464E
:10E57800584601F0F1FF5146584601F0EDFF584664
:10E58800149901F0E9FF5846099901F0E5FF00E701
:10E59800159ADDF84090A2EB0308E9E639464246B1
:10E5A800584602F017FA074600287FF400AEB9462D
:10E5B8001A9DD3E739465846159A02F0B1F907462D
:10E5C80000287FF4F0ADF2E7012279491646CB1A0C
:10E5D80002FA03F5CAE5DDE91234CDE90E343CE66A
:10E5E8000023744CCDE90E34CDE9123435E6A9F197
:10E5F80054730593DDE904452046294602F03CFBA7
:10E60800DDE90E23F2F7D4FB2B462246F1F7A2FEF2
:10E61800DFF89891684B01EA09099945CDE90401A9
:10E6280079D9DDE90C0103F15473994202D1064608
:10E638000136BCD04FF0FF33604CCDE9043454E6CA
:10E64800DDE90467A5E600235D4CCDE90E3400231F
:10E65800584CCDE9123400E6DDE912562846314619
:10E668000BF0D4FAF1F7FEFF0B4602463146284676
:10E67800F1F76EFE119D049BC4F313041D432C4354
:10E688008046894626D142A3D3E90023F2F778F8D9
:10E6980000283FF42AAEB946DDE904671A9D62E70F
:10E6A8000293089B584601931AAB0093454A1BAB4B
:10E6B80019A901F03FFB10F00F0504463FF467AEBF
:10E6C800062D40F0B58000227B1C0026002708920A
:10E6D80019935EE630A3D3E90023F2F751F8002836
:10E6E800D9D12FA3D3E9002340464946F2F766F86B
:10E6F80000283FF4FAADCEE7049B012BA3D1B9F172
:10E70800000FA0D1B9461A9C2223254600260027CF
:10E71800CBF8003027E701F154740594DEE50A9F31
:10E728000C9B082D03440C936DDC6546FFF759BB21
:10E7380001223846244900F0F9FD002800F0BB808A
:10E748004FF000094E4648464D46CA46CDF830902F
:10E75800CDF82890FFF7A3BB44F61F639942A8BFE2
:10E768001946109114E40B981849DDE9042301EBCC
:10E77800C001D1E90001F2F71BFB06460F4608E687
:10E788006E2C3FF4A3ABFFF768BB00BFAFF300806C
:10E798009535A094FFFFCF3F9535A094FFFFDF3F4D
:10E7A80035E5AF350000E03F0000E03F0000F07FB6
:10E7B800E2FBFFFF0000F03FFFFF9F7CFFFFEF7FC2
:10E7C8000000F0BF20DA0108BCA4010898DC0108A9
:10E7D800A04919A801F082FD00283FF43EAB199B1F
:10E7E8009D49013B19A8199301F078FD10B9199BAF
:10E7F800013319930026994FCBE522230026974F22
:10E80800CBF80030C5E5BCF1100FD8BF09EB89097A
:10E8180065464FF00000D8BF02EB4909FFF7E6BA9A
:10E82800DDE91234CDE9163441E50020FFF7CCBA12
:10E838001A9A3AB135211CA802F02CFB58461A99AD
:10E8480001F08AFE013D1B9B042D00F2C481DFE824
:10E8580005F0032C291E03001C9A049203F233428C
:10E868001D9B23F4801343EA02530593E10502D567
:10E8780043F000430593794ADDE904671A40002A0A
:10E888007FF487AD01F020F82223036081E54FF083
:10E89800FF326FF00043CDE90423E3057FF5D0AEE6
:10E8A800059BE5E76D4B0593F7E7DDE91C121D9B1A
:10E8B800CDE90412DAE7199A06461346013219928D
:10E8C80081465C78FFF773BAAA460C90FFF791BAB5
:10E8D8000023634CCDE90E340023624CCDE9123499
:10E8E800BBE44B461198B446B946DDE90C67AE4621
:10E8F8005D49C3F31302002845D08A4200F0FD8029
:10E90800ADBB049A1CEA020F34D030463946049352
:10E9180002F0B2F90A9B002B00F03781049BC3F385
:10E928000A53C3F16B03002B40F352811C0504F119
:10E938007F53002203F54013F2F73AFA02460B46DA
:10E9480030463946F1F706FD06460F463046394649
:10E95800464B0022F2F72CFA404B06460B400F4676
:10E96800002B7FF49BAE2223CBF8003096E61EEAFC
:10E97800030FCAD10A9B002BE8D18FE601F154732B
:10E988000593FFF7BFBB002A74D1DDE90445224691
:10E99800002C40F0A2800A9A002A40F0CB8025F093
:10E9A8000044240D2405A4F580146FEA14536FEA7B
:10E9B800035305934FF0FF3304931A9DDDE9046771
:10E9C800D1E5119BDDE904010343B946DDE90C6794
:10E9D800D0D1C1F31303002BCCD121F00044240D76
:10E9E8002405B4F1D66F2546C4D9099A536913B9D9
:10E9F8001369012BBEDD01220999584601F0EAFF8F
:10EA08005146099002F05CF80028B3DD0A9B002B00
:10EA1800C9D0A5F580136FEA13536FEA0353059322
:10EA28004FF0FF330493DDE904678FE7104919A815
:10EA38001CAA01F06DFC05287FF453AA1D9B43F026
:10EA4800FF4343F4E00305931C9B0493DDE904674B
:10EA58009FE400BFC0A40108C4A401080000F07F1F
:10EA68000000E0BF0000E03FFFFF0F00000050394A
:10EA78000CDA0108A5BB049A1CEA020F3FF47AAF2E
:10EA880030463946049302F0F7F80A9B002B62D00F
:10EA9800049BC3F30A53C3F16B03002B40F38C8030
:10EAA8001C0504F17F53002203F54013F2F780F9A7
:10EAB80002460B4630463946F1F74AFC002200234D
:10EAC80006460F46F1F752FE00283FF43FAF1AE61C
:10EAD8004FF00009414AFFF7F8BABEF1000FCBD05A
:10EAE8001EEA030F3FF446AFCAE74FF0FF3202FABF
:10EAF80003F3049A1A400492C6E40A9A0499B2B13C
:10EB0800374A1A40B2F1D46F11D84FF0FF30120DC6
:10EB1800C2F16B0200FA02F2914240D0BEF1000F3E
:10EB28007FF425AF11EA0C0F3FF424AFEDE64FF068
:10EB3800FF32F1E72A4D1D40B5F1D66F3FF669AFB8
:10EB4800B5F15C7F3FF602AF2223002600271A9D0D
:10EB5800CBF8003007E502460B4630463946F1F758
:10EB6800F7FB1A9C0022002306460F462546F1F7BC
:10EB7800FDFD00283FF4F7ACC6E54FF0FF33C2F1C6
:10EB88004B0293400B4005937EE402460B46304609
:10EB98003946F1F7DFFB1A9D06460F46E3E4114AB2
:10EBA80093420CD00E4A1A4002F5801305930023B5
:10EBB8000493DDE90467DDE602460B467AE7013196
:10EBC800F0D1222300261A9D054FCBF80030CAE465
:10EBD80002460B46B4E6002348E600BF70DC010895
:10EBE8000000F07FFFFFEF7F014BFFF735B800BF54
:10EBF8005405002084460A460249034B08686146CA
:10EC0800FFF72AB8C006002054050020024A03492D
:10EC1800034800F0C9B800BF480500203572010854
:10EC2800C80600200C4B416810B59942044601D033
:10EC380008F0FCFAA168094B994202D0204608F076
:10EC4800F5FAE168064B994204D02046BDE8104029
:10EC580008F0ECBA10BD00BF081F0020701F00208C
:10EC6800D81F00202DE9F84300250423304C314AF1
:10EC78003149DFF8C890DFF8C880324F324E116052
:10EC880004F15C0029460822C4E90335C4E90055AB
:10EC9800C4E90555A560656600F0F8FA04F1580066
:10ECA800C4E90749C4E90987E66200F03BFE274B3F
:10ECB8002946082204F1C4006367C4E91A55C4E967
:10ECC8001E552567C4F8CC50C4F8805000F0DEFA11
:10ECD80004F1680304F1C000C4F88430C4E9229840
:10ECE800C4E9247600F01EFE194B294604F59670F7
:10ECF8000822C4F8DC30C4E93455C4E93855C4F8EE
:10ED0800D850C4F83451C4F8E85000F0BFFA04F100
:10ED1800D003C4E93D87C4F8F09004F59470C4F8B2
:10ED2800FC60C4F8EC30BDE8F84300F0FBBD00BF60
:10ED3800081F00204020002015EC000805F10008FD
:10ED48002DF100086DF1000891F10008090001009B
:10ED58001200020010B504460A4800F0E7FD636B94
:10ED680023B9094B094A1B68626323B1BDE8104007
:10ED7800044800F0DDBDFFF775FFBDE8104001480D
:10ED880000F0D6BD50200020402000202DEC0008C7
:10ED9800014800F0CBBD00BF50200020014800F022
:10EDA800C7BD00BF502000202DE9F8434FF00009EF
:10EDB80080460F461646D6E90154013D10D4A38972
:10EDC800012B08D9B4F90E30013304D0214640464E
:10EDD800B84749EA0009013D6B1C04F16804EED10B
:10EDE8003668002EE7D14846BDE8F8830FB400B571
:10EDF800074A83B004AB106853F8042B8168019369
:10EE080005F062FB03B05DF804EB04B0704700BF87
:10EE1800C006002030B5054689B008460C4600F00B
:10EE280097FD01230222204907936B6B06910292FA
:10EE380004A9421C04940191AC6805900392002B2C
:10EE48002ED0626EB4F90C30D20701D4980521D5C2
:10EE5800990406D4626E43F4005322F40052A3814D
:10EE68006266284601AA214608F0FEFA636E002869
:10EE78000CBF0A254FF0FF35DA0702D4A3899B059A
:10EE880002D5284609B030BDA06D00F051FD2846D6
:10EE980009B030BDA06D00F049FDB4F90C30D7E7DA
:10EEA8002846FFF757FFCCE760A30108024B01464D
:10EEB8001868FFF7AFBF00BFC00600202DE9F04378
:10EEC800664C0E46D4F80080174604461D4683B0AB
:10EED800B8F1000F04D0D8F83430002B00F0A68029
:10EEE800022F05D0012F00F2A580002DC0F2A280CC
:10EEF800636EDA0751D52146404608F08BFA216B3C
:10EF080041B104F14003994202D0404600F0C4FDEB
:10EF1800002323630023B4F90CC0A3611CF0800F05
:10EF280063605DD12CF44A6C2CF0030C022FA4F81A
:10EF38000CC063D001AB214640466A4608F078FC15
:10EF4800A3891843A081002D2ED0002E2DD0D8F8EB
:10EF58003430002B37D0009AB4F90C30AA421CBFC9
:10EF680043F40063A381012F04BF43F00103A3818D
:10EF780013F00802C4E90465266028D0D90753D5E0
:10EF88000022A260626E6D42D207A56123D49B0560
:10EF980021D4A06D00F0CCFC1DE0A3899B05AAD468
:10EFA800A06D00F0C3FCA6E7009D2846FEF7D4F943
:10EFB8000646002841D0A38943F08003A381D8F8EE
:10EFC8003430002BC7D14046FFF7C4FEC3E7A26028
:10EFD800626ED207DBD50025284603B0BDE8F08372
:10EFE8004046216900F058FDB4F90CC0022F2CF4FA
:10EFF8004A6C2CF0030CA4F80CC09BD1002500210E
:10F00800012204F1430323602361636E4CF0020084
:10F01800A081D807A1606261DED41CF4007FDBD137
:10F02800A06D00F085FCD7E7A560D1E74046FFF763
:10F0380091FE55E74FF0FF35CEE7DDF80090A94582
:10F0480006D04846FEF788F9064608B14D46B2E7AD
:10F058004FF0FF35B4F90CC0D1E700BFC00600205F
:10F068000EB430B504466FF000459CB00B4A1FAB98
:10F078000B49059253F8042B086802A9CDE901341D
:10F0880004950795069402F00DF80022029B1A7069
:10F098001CB0BDE8304003B0704700BF0802FFFF56
:10F0A800C00600200EB44FF4017270B59DB021ADBA
:10F0B80055F8046BADF814200290069000F048FC57
:10F0C80000234FF6FF7104460E931393094A0A4B27
:10F0D8000A92ADF816103246186802A92B46019517
:10F0E8000394079403F074FD1DB0BDE8704003B0AD
:10F0F800704700BF29F10008C006002010B50C4673
:10F10800B1F90E1000F0A2FB002803DB236D0344C5
:10F11800236510BDA38923F48053A38110BD00BFCC
:10F12800002070472DE9F0410C46B1F90C101F463C
:10F13800CB05054616460BD421F48051A1813B46E8
:10F1480032462846B4F90E10BDE8F04100F0A6BBDF
:10F15800B4F90E100223002200F062FBB4F90C107F
:10F16800EAE700BF10B50C46B1F90E1000F058FBE5
:10F17800B4F90C30421C0EBF23F4805343F480537F
:10F188002065A38110BD00BFB1F90E1000F036BB99
:10F1980088420ED98B1883420BD900EB020C002A47
:10F1A8006DD0624613F801CD994202F801CDF9D12C
:10F1B80070470F2A0FD8034602F1FF3C002A5ED0A1
:10F1C8000CF1010C013B8C4411F8012B614503F84B
:10F1D800012FF9D1704740EA01039B0750D1A2F1F2
:10F1E800100370B501F1200C23F00F0501F1100E8A
:10F1F80000F11004AC441B095EF8105C0EF1100E0F
:10F2080044F8105C5EF81C5C103444F81C5C5EF832
:10F21800185C44F8185C5EF8145CE64544F8145C25
:10F22800EAD1013312F00C0F01EB031102F00F04C5
:10F2380000EB031328D08E46043C24F003064FEA63
:10F24800940C1E441C1F5EF8045B44F8045FB4422F
:10F25800F9D10CF1010402F0030203EB840301EB82
:10F26800840102F1FF3C4AB10CF1010C013B8C44D2
:10F2780011F8012B614503F8012FF9D170BD7047D2
:10F28800034602F1FF3C9BE72246EAE770B5860792
:10F2980047D0541E002A3ED00346CAB201E0013CC2
:10F2A80039D303F8012B9D07F9D1032C2CD9CDB202
:10F2B80005EB05250F2C1A4605EB054534D9A4F1B5
:10F2C800100C2CF00F0603F1100EB6444FEA1C1C6C
:10F2D800C2E90055C2E9025510327245F8D10CF165
:10F2E800010214F00C0F03EB021204F00F0C13D000
:10F2F800ACF1040323F003030433134442F8045B22
:10F308009342FBD10CF003042CB1C9B21C4403F89E
:10F31800011BA342FBD170BD64461346002CF4D1F7
:10F32800F9E703461446C0E7A446E1E7002A3ED0C1
:10F33800844630B50446084380070B462ED1032A7D
:10F3480007D82BE0043A25D01EF0803F22D1032AAB
:10F3580022D919462068A446A0F1013323EA000EF9
:10F368000B4653F8045B0434A842EBD09CF8000029
:10F378000C7884421DD1E64668B11EF8010F11F8D9
:10F38800014FA2EB0E03A04203F1FF3311D11CEB96
:10F398000303F1D1002030BDA44619469CF80000B3
:10F3A8000C78A04205D1012AF4D0E646E4E71046DD
:10F3B8007047001B30BD00BF01292DE9F0415AD923
:10F3C80001274FF0000E4FF0FF34BC463B4607E0E4
:10F3D8009E464FF0010C1F1B0EEB0C0399420ED9F1
:10F3E800051915F80C50C65CAE42F1D333D001278D
:10F3F800BC467446BE440EEB0C039942F0D84FF05D
:10F4080001084FF0000E4FF0FF35C4464346176021
:10F4180008E09E464FF0010CA3EB05080EEB0C0329
:10F4280099420FD9461916F80C60C75CB742F0D854
:10F4380019D04FF00108C4467546C6440EEB0C03BC
:10F448009942EFD80135601C854202D32846C2F89C
:10F458000080BDE8F081BC450ABFE6440CF1010C10
:10F468004FF0010CB8E7C4450ABFE6440CF1010CA3
:10F478004FF0010CD2E74FF001080025E6E700BF86
:10F488002DE9F04F9346ADF21C4D05AA80468A46F9
:10F49800584619461C46FFF78FFF814613460DF262
:10F4A800144243F8044F9342FBD16CB1601E584498
:10F4B8000BF1FF3206AD12F8011FA31A013B5B44A2
:10F4C800824245F82130F6D1059B4A4658460BEB57
:10F4D8000301019308F0FAFA002879D10746054696
:10F4E80044F40063AAEB040E0293661EAE4512D3E1
:10F4F80008EB050C1CF8063006AA52F82330CBB1ED
:10F5080027B1019A9A4284BF1346E31A1D44AE45B7
:10F518004FF00007ECD208EB0A00029908F0A2FBB2
:10F528008244AAEB040EAE45E2D200200DF21C4D37
:10F53800BDE8F08F4F453B4638BF4B469E4218D931
:10F54800591EEA1859444244009502E001339E428C
:10F558000ED012F8010B11F8015F8542F6D09E42D9
:10F56800009D06D9C9F101022A440027D518BDE734
:10F57800009D4F4509F1FF3380F0828005EB0902B9
:10F5880042440BEB09010095CDF80C9002E09F4234
:10F5980013D04B4611F8015D12F8010D03F1FF3944
:10F5A8008542F4D0009DDDF80C90013301379F426D
:10F5B80009D8019B1D44E71A98E701379F42009D2F
:10F5C800DDF80C90F5D960460DF21C4DBDE8F08FC2
:10F5D800A4EB09034B4538BF4B460025013344F4DF
:10F5E8000062AAEB040E0092661E01930593AE45D5
:10F5F80009D308EB0500835D06AA52F823306BB1E6
:10F608001D44AE45F5D208EB0A00009908F02AFB24
:10F618008244AAEB040EAE45EBD286E7B14517D279
:10F6280009F1FF3105EB09024B465944424402E017
:10F638000133B3420CD012F8017B11F801CFBC455D
:10F64800F6D09E4204D9C9F101022A44D518CEE762
:10F65800B9F1000F3FF46AAF05EB090141440BEB28
:10F66800090203E0013B5B453FF460AF134611F824
:10F67800017D12F801CDBC45F4D0019B1D44C0E7C3
:10F688004B4693E72DE9F0410D460978044690B0C2
:10F69800002954D06A78002A00F08280AB78002BC9
:10F6A80051D0E8782E68002800F081802B79002B53
:10F6B80056D0284600F04CF90646204646F400711C
:10F6C80008F0D0FA86425AD8FE2E00F28880801BB5
:10F6D800271840226846711CFFF7D8FD7EB16A1EC4
:10F6E8005FFA86FC901912F8013F03F03F0340339C
:10F6F800A91A6B446144904203F8401CF3D1013CC1
:10F70800A35D03F03F0340336B4413F8403C1C44B3
:10F71800A74203D238E04444A74235D314F806C0C0
:10F7280032460CF03F0C0CF140030DEB030C29465C
:10F7380020461CF8408C08F0C9F90028EBD1204677
:10F7480010B0BDE8F081007842EA0142B8B140EA61
:10F7580003439A42214614F8010FF7D14C1EEEE7F5
:10F76800227862B131BA01E08B421ED0204642EACB
:10F77800032314F8012F002AF6D18B4215D0002458
:10F78800204610B0BDE8F081BB5DB819002BF6D05B
:10F798004FF4006108F066FA0744A742AFD2EEE7DB
:10F7A80010B0BDE8F04108F0BFB9C41EC7E71204A5
:10F7B80042EA0162217842EA03230029DFD00246A7
:10F7C80001E00029DBD041EA0200B3EB002F254617
:10F7D8004FEA002214F8011FF3D1AC1EAFE701462F
:10F7E80033462A46204610B0BDE8F041FFF748BE30
:10F7F800014B93F82801704754050020002238B5C2
:10F80800064D044608462A60F1F7A8FF431C00D0BD
:10F8180038BD2B68002BFBD0236038BD4420002066
:10F8280038B50C46114600228446074D20462A600A
:10F838001A466446F1F79EFF431C00D038BD2B687A
:10F84800002BFBD0236038BD4420002038B50C467F
:10F85800114600228446074D20462A601A4664460F
:10F86800F1F790FF431C00D038BD2B68002BFBD06C
:10F87800236038BD44200020002238B5064D0446D8
:10F8880008462A60F2F77CF9431C00D038BD2B6883
:10F89800002BFBD0236038BD4420002038B50C462F
:10F8A800114600228446074D20462A601A466446BF
:10F8B800F1F73AFF431C00D038BD2B68002BFBD072
:10F8C800236038BD44200020014B1868704700BFF2
:10F8D800C006002070B50F4B0F4DAB42A3EB0506D9
:10F8E80007D00024B61055F8043B01349847A642C7
:10F8F800F9D80AF01BFB094D094B5E1BAB424FEAD6
:10F90800A60606D0002455F8043B01349847A642C1
:10F91800F9D870BD98480208984802089848020823
:10F92800A0480208704700BF704700BF704700BF7B
:10F93800704700BF082802D14FF48050704708B5BF
:10F94800FFF7C2FF162203464FF0FF301A6008BDCA
:10F9580020F0030110F00300C0F1000051F8043B4F
:10F9680000F1040C4FEACC0C6FF000021CBF22FA25
:10F978000CF213434FF0010C4CEA0C2C4CEA0C4CE3
:10F98800A3EB0C0222EA030212EACC1204BF51F8DC
:10F99800043B0430F4D0C2F1000102EA0102B2FAD9
:10F9A80082F2C2F11F0200EBD20070470020014929
:10F9B800704700BF0000F87F004870470000C07F14
:10F9C800024B13B1024800F005B870470000000070
:10F9D800617D0108002301461A46184608F052BA0C
:10F9E8002DE9F843064608208946FFF7A3FF054698
:10F9F800DFF898803046FDF773FFD8F808305F6865
:10FA080027F00307A7F11104A4EB09042C44B4FB65
:10FA1800F5F4013C05FB04F4A54208DC002130465E
:10FA2800FFF72AFFD8F808303B44984205D0304603
:10FA3800FDF75CFF0020BDE8F88330466142FFF720
:10FA48001BFF01300FD0124AD8F808303F1B47F08F
:10FA580001075F60136830461B1B1360FDF746FF04
:10FA68000120BDE8F88300213046FFF705FFD8F8EC
:10FA78000820831A0F2BDADD43F001035360054B8E
:10FA880003491B68C01A0860D1E700BF4001002085
:10FA9800D41E00203801002000297CD0F8B50C467F
:10FAA8000646FDF71DFF54F8043C764FA4F10805FF
:10FAB80023F001016818D7F808C04268844522F08D
:10FAC800030200F08380DB07426000EB020C33D4B2
:10FAD80054F8084CDCF804302D1B2144AC6807F1BD
:10FAE800080C644503F0010364D0D5F80CE0C4F8B1
:10FAF8000CE0CEF80840002B00F0818041F00103B3
:10FB08006B600160B1F5007F22D20122CB08490960
:10FB18008A40796801330A437A6057F8331007EB53
:10FB2800C302083AC5E9021247F83350CD6030469F
:10FB3800BDE8F840FDF7DABEDCF80430DB072BD56A
:10FB480041F00103B1F5007F44F8043C0160DCD3C7
:10FB5800B1F5206F4FEA512353D28B0903F13900D5
:10FB680003F13802C300F818FB580838984203D14B
:10FB780061E09B68984204D05A6822F003028A42E6
:10FB8800F7D8D868C5E9023085603046DD60BDE841
:10FB9800F840FDF7ABBE7047114407F1080C8368C5
:10FBA80063453FD0C268DA60936041F001036B603F
:10FBB8006950A7E7002B5FD10A44D0E90213CB6054
:10FBC800996042F001036B60AA50B0E70A44D90774
:10FBD80007D454F8083CED1A1A44D5E90213CB604F
:10FBE800996042F001036B60274BBD601B6893422C
:10FBF8009DD8264B30461968FFF7F2FE97E7114467
:10FC0800CDE7142B08D9542B1DD80B0B03F16F002B
:10FC180003F16E02C300A6E703F15C0003F15B0287
:10FC2800C300A0E741F00103C7E90455C5E902CCC8
:10FC38006B6069507BE70121921001FA02F2796842
:10FC48000A437A609EE7B3F5AA7F06D8CB0B03F187
:10FC5800780003F17702C30085E740F254529342DB
:10FC680006D88B0C03F17D0003F17C02C3007AE710
:10FC78004FF47E737E2276E741F001036B600160EA
:10FC880055E700BF400100203C010020041F002070
:10FC98002DE9F0410469B4EB611F05DC0023036121
:10FCA80000234361BDE8F08100F114054E1111F005
:10FCB8001F0C05EB840E05EB860321D055F82610A2
:10FCC80004339E4521FA0CF1CCF120082DD92F469A
:10FCD8001A6802FA08F20A4347F8042B53F8041B7F
:10FCE8009E4521FA0CF1F3D8A31B9B00053B9B080A
:10FCF800013305EB830445F8231079B104340DE092
:10FD08009E4588BF00F11002C8D953F8041B9E45D0
:10FD180042F8041FF9D8A41B05EB8404631B9B104D
:10FD2800AC420361BCD0BDE8F08141610029B5D087
:10FD38002C46E3E72DE9F04F1C4685B00090086893
:10FD4800934682780B46302A029440F0F381C11C16
:10FD58000A780C46302A01F10101F9D0A4EB000918
:10FD6800A9F10209DFF8C08218F80220002A00F081
:10FD7800EF80002722783D4618F80220002A00F07C
:10FD88007781264616F8012F18F80220002AF9D1A3
:10FD980001223046A5490193FFF7C8FA019B824624
:10FDA80000284DD03278002D00F0A581A5EB060A79
:10FDB8004FEA8A0A02F0DF02502A35464DD01E600B
:10FDC800002F74D12B1B013B072B394604DD5B1038
:10FDD800072B01F10101FADC009800F097FB0346BC
:10FDE800002800F06A8200F11406A542019640F24C
:10FDF800CA8100270390B9460DE0202F1AD0394652
:10FE080004372A7818F8022002F00F028A4049EADB
:10FE18000209A54254D015F8012D2E2AEDD1A5428C
:10FE2800EBD3012228468149FFF780FA0028F0D059
:10FE3800202FE4D1002146F8049B04278946E0E7F7
:10FE4800002D00F068813278A5EB060A02F0DF0287
:10FE5800502A35464FEA8A0AB1D16A782B2A00F02F
:10FE680048812D2A40F0D5800120AA78AE1C18F8C8
:10FE780002104A1E182A00F2D5807278103918F834
:10FE8800022001365AB90CE001EB810102EB410274
:10FE9800A2F1100116F8012F18F802200AB1192A48
:10FEA800F2DD00B149428A441E60002F8AD0B9F1C0
:10FEB800000F0CBF06250025284605B0BDE8F08FC9
:10FEC800039B019A46F8049BB61AB6101E61484671
:10FED800039300F0F5FB7601DBF80040361AA642E2
:10FEE800039B76DCC0F209810027DBF80820524525
:10FEF800C0F23E81DBF8042052454EDDA2EB0A0A2F
:10FF0800544500F39580DBF80C10022900F0E180DD
:10FF1800032900F05381012940F0DF80544540F067
:10FF2800DC80012C0AD01846611E039300F0E2FF22
:10FF3800039B002800F0D180DBF8042001210298FF
:10FF480062250260019A196111600E9A1360B3E785
:10FF58000122204635490193FFF7E8F9019B07463E
:10FF6800002840F087806278651C18F80210002984
:10FF780000F08280302A2C4640F02B8114F8012FA3
:10FF8800302AFBD018F802204FF00109B2FA82F7A4
:10FF98007F09002A7FF4F5AE6AE0012587B1DBF816
:10FFA8000C20022A6FD0032A71D0012A06D1B90782
:10FFB80004D5019A12681743FA076BD445F0100567
:10FFC80028460E9A1360029BC3F800A005B0BDE84E
:10FFD800F08F361B1846314600F08CFF039B07460E
:10FFE80078B10127711E01984A1150F8220001F0DA
:08FFF8001F0207FA02F20242A7
:020000040801F1
:1000000003D0B94200F3CF8002271846314603934C
:10001000B244FFF741FE039B6BE718F80210002083
:100020004A1E182A05F101067FF62BAF2E46CAE6B6
:1000300064DB0108BCA401080AF1FF35002F40F081
:10004000A480002D40F0A78001220198691150F88A
:10005000211005F01F05AA400A4218465146039395
:1000600018BF47F00207A4EB0A04FFF715FE0225AC
:10007000DBF804A0039B95E726468DE6254622780B
:1000800002F0DF02502A00F099801D6013E70F9AFA
:10009000C2F101020F920F9A002A93D001991E69B2
:1000A00088460A4600274FEA860901EB860003E0EE
:1000B000904242F8047C45D9944652F8041BB1F1B1
:1000C000FF3FF5D00131022DCCF800107ED014F0A6
:1000D0001F0440F0AE80212576E70F9900293FF4F8
:1000E00031AF50251946009800F03AFA002328460F
:1000F0000E9A136005B0BDE8F08F0020B9E6AA465D
:100100005CE6A61B19463246009800F067FC00F139
:10011000140203460027AAEB060A0192E9E6727868
:10012000751C18F802102E4600293FF447AE16F849
:10013000012F18F802100029F9D13BE64FF0000911
:10014000841C13E69A6896424ADA0121022D06EBD6
:10015000010003EB86061861DDF80480716135D07B
:10016000002874DC00221A6100225A61DBF80820A2
:100170000AF1010A5245AEDA1946009800F0F0F98A
:1001800000230E9AA32513609AE601275CE74FF03F
:100190000009019E99E618462946039300F0AEFE39
:1001A000039B074650E71846B11E039300F0A6FED6
:1001B000039B00283FF428AF032726E74FF0000AEF
:1001C00001274EE60F9900298BD0BBE6DBF8002013
:1001D000013AA24262D02225F6E64FF00109D4E5A9
:1001E000596800980131019300F094F9019B07468A
:1001F00000286CD01A6903F10C01023292000C3015
:100200000193F0F763FD019B0098194600F0A8F9EF
:1002100001213B69022D03EB010007EB83033861E9
:1002200007F1140859613B46D0D08642BFF64FAF64
:1002300096E7C14459F8040C019300F045FAC4F163
:100240002004A042019BBFF646AF186988E75A69AF
:1002500008EB800003F11804A0424FEA520229D9AA
:100260004546216842EAC17245F8042B54F8042B34
:10027000A0424FEA5202F4D8C11A19398908013153
:1002800048F8212008EB810102B10431A1EB0802FA
:10029000921041451A617FF469AF65E7012261114F
:1002A00058F8211004F01F04A2400A4214BF21256F
:1002B000222589E6C8F800200AB14146E5E71A611F
:1002C00052E70246E421054B054807F01FFE0246AF
:1002D0008421024B024807F019FE00BF14A5010853
:1002E00028A5010810B504688646013409E014F811
:1002F000013BA3F1410CBCF1190F98BF203393428D
:1003000007D111F8012B002AF1D10120CEF80040CD
:1003100010BD002010BD00BF0B682DE9F04F591132
:1003200002EB810113F01F0306464FF000050DBFDD
:100330000846081D8E46A1F1040E316840F8045CA1
:100340004C1C497885B0002900F0AF807746F44610
:100350000093AA460B46A9467146AB469646DFF87F
:1003600084810246019610E0202B00F296804D45D4
:1003700008DD674502D9BAF1070F67DDE6455CD3B2
:100380004FF0080A14F8013FB3B118F80360002ECB
:10039000EAD00AF1010ABAF1080F05F1010542DCC1
:1003A000DCF800301B0106F00F061E43CCF800609D
:1003B00014F8013F002BE8D1104672468E46009B90
:1003C000002D72D0BC4502D2BAF1070F74DD624530
:1003D00055D26346111F53F8044B734541F8044F3F
:1003E000F9D9AEEB0C0323F003030EF10101043342
:1003F0000CF1010C8C4588BF04230021134443F801
:10040000041B7345FBD950F8041C19B107E05EF8D2
:10041000043D23B97245FAD10123CEF800300520FE
:1004200005B0BDE8F08FE645ACD24CF804BC002323
:100430004FF0010AACF1040CB5E7ACF104074CF83D
:1004400004BCA946BC464FF0000A9BE7CAF108006D
:1004500080006646CDE902C2DCF800308446C0F177
:10046000200A706800FA0AF21A4320FA0CF332608C
:1004700046F8043FB742F4D8DDE902C27EE750F8FF
:10048000041C002BC1D04FF0FF34C3F1200324FA29
:1004900003F3194040F8041CB7E7104672468E4635
:1004A00019462929019E009B03D0042005B0BDE810
:1004B000F08F0134346083E7DCF80040CAF10801B2
:1004C0008900664688462546C1F12009716801FA0F
:1004D00009F42C4321FA08F5346046F8045FB7426A
:1004E000F4D874E764DB010882B049B15AB16BB14A
:1004F00013780B601278101E18BF012002B07047ED
:1005000001A9002AF3D1104602B070476FF0010034
:10051000F4E700BF38B5436C05460C464BB153F8C1
:10052000240080B1026843F824200023C0E903338B
:1005300038BD2122042107F009FD03466864002824
:10054000EDD1002038BD0121284601FA04F56A1DCD
:10055000920007F0FBFC0028F3D0C0E90145E4E776
:1005600031B1436C4A6853F82200086043F8221006
:10057000704700BF2DE9F0414FF0000E0E461C46BB
:100580000D69074601F1140001680EF1010E8BB2EE
:1005900002FB0343090C4FEA134C02FB01CC9BB254
:1005A00003EB0C43754540F8043B4FEA1C44EBDC7D
:1005B0003CB1B368AB4207DD06EB850301355C61F6
:1005C00035613046BDE8F081716838460131FFF78A
:1005D000A1FF8046A8B1326906F10C0102329200F7
:1005E0000C30F0F773FB7B6C726853F822103160AB
:1005F00043F82260464606EB850301355C613561B0
:10060000DFE70246BA21024B024807F07FFC00BF39
:1006100014A501088CA501082DE9F8431E460C46D7
:1006200026490833174681FB032C092E4FEAE37352
:100630000546C3EB6C0339DD4FF0010C00214FEA96
:100640004C0C634501F10101F9DC2846FFF762FF1C
:10065000014668B3089B092F43614FF00103036112
:1006600012DC09270A34BE420BDDF61B264414F8BF
:10067000013B0A222846303BFFF77CFFB44201468B
:10068000F5D10846BDE8F88304F10909C8463C44A1
:1006900018F8013B0A222846303BFFF76BFFA045C4
:1006A0000146F5D1A7F108044C44DCE70021CCE772
:1006B0000246D321024B034807F028FC398EE33869
:1006C00014A501088CA50108B0F5803F03463ABF88
:1006D000102083400020B3F1807F3CBF1B02083014
:1006E000B3F1805F3CBF1B010430B3F1804F03D3F3
:1006F000002B06DB013070479B0003D45B0003D462
:10070000202070470230704703307047036801466D
:1007100013F0070209D0DA0721D498074BBF5B0812
:100720009B08012002200B60704798B2A0B11046D0
:10073000DAB20AB908301B0A1A0704BF1B090430D1
:100740009A0704BF9B080230DA0703D45B0800F164
:10075000010006D00B6070471020C340E8E700207E
:1007600070472020704700BF38B5436C04460D46E3
:100770004BB15868B0B102685A600022012345614C
:10078000C0E9032338BD2122042107F0DFFB034623
:1007900060640028EDD1002240F24511074B084863
:1007A00007F0B4FB1C220121204607F0CFFB0028F4
:1007B000F1D001220223C0E90123DEE714A50108DC
:1007C0008CA501082DE9F04FD1F8108015690E466F
:1007D000A845924685B005DB2A46534645468A46DB
:1007E00090461E46DAF80830DAF8041005EB0804E3
:1007F000A342B8BF0131FFF78DFE002800F08980C9
:1008000000F1140707EB840E774505D23B46002222
:1008100043F8042B9E45FBD8143606EB88080AF1F2
:100820001409464509EB850566D2A5EB0A03153B7D
:1008300023F003030AF1150A043355452CBF9B46E8
:100840004FF0040BCDF808E08246AE46039405E075
:10085000090C2AD1B04507F104074AD956F8041B00
:100860008DB2002DF4D0CC463C46002301965CF8B6
:10087000040B216886B28AB205FB0622000C090C23
:1008800005FB00111A4401EB124192B242EA014207
:10089000E64544F8042B4FEA1143E8D8019E47F897
:1008A0000B3056F8041C090CD4D000223B68484693
:1008B0001D463C46944602889BB201FB02C202EBF5
:1008C000154243EA024344F8043B50F8043B2568D0
:1008D0004FEA134CABB201FB0C33704503EB1243F0
:1008E0004FEA134CE7D3B04547F80B3007F1040744
:1008F000B4D8DDE902E45046002C02DC05E0013CFE
:1009000003D05EF8043D002BF9D0046105B0BDE8CA
:10091000F08F02464FF4B171014B024807F0F6FA2E
:1009200014A501088CA5010812F003032DE9F0417C
:10093000144607462CD10E46A4101CD03D6C85B33E
:10094000E3074FF0000806D4641014D02868A8B15B
:100950000546E307F8D52A4631463846FFF732FF09
:1009600036B17B6C716853F82120326043F8216006
:1009700064100646EAD13046BDE8F0812A46294691
:100980003846FFF71FFF28600546C0F80080E0E703
:100990000F4A013B52F823200023FFF7EBFD0646E8
:1009A000CAE701213846FFF7B5FD054640B140F2E0
:1009B00071230122C0E90423002338640360BFE7E8
:1009C000024640F24511034B034807F09FFA00BF6F
:1009D00064DC010814A501088CA501082DE9F04785
:1009E0000C462769A36807EB62177D1C9D42904661
:1009F000064649684FEA621904DD5B009D4201F139
:100A00000101FADC3046FFF785FD002851D0B9F12D
:100A1000000F00F114010FDD0B464FF0000C09F13F
:100A200005024FEA820E00EB820243F804CB9342A8
:100A3000FBD1AEF114031944226904F1140318F038
:100A40001F0803EB820C2CD08E464FF0000AC8F131
:100A500020091A6802FA08F242EA0A024EF8042B48
:100A600053F8042B9C4522FA09FAF2D8ACEB0403A4
:100A7000153B23F00303043304F11502944538BFFA
:100A8000042341F803A0BAF1000F00D13D46736C76
:100A90006268056153F82210216043F82240BDE8E6
:100AA000F087043953F8042B9C4541F8042FF9D8FA
:100AB000ECE702464FF4EF71014B024807F026FACB
:100AC00014A501088CA5010884460B690069C01AA9
:100AD00015D10CF1140C14310CEB830210B401EBA2
:100AE000830301E0944508D252F8044D53F8041DE5
:100AF0008C42F7D004D24FF0FF3010BC70477047E3
:100B0000012010BC704700BF2DE9F04F14460A6960
:100B100023698846D21A002A83B040F0888001F108
:100B2000140604F1140202EB830206EB830301E0D6
:100B30009E427FD253F8045D52F8041D8D42F7D0D7
:100B400076D323460025444698466168FFF7E2FCC9
:100B5000002800F0898000F1140949464FF0000C8C
:100B60002769D8F8106004F1140B08F1140EC56061
:100B700004F110020EEB86060BEB870ACDF804B0E9
:100B80005EF8044B52F8045F1FFA84FBABB2A3EB90
:100B90000B03240C6344C4EB154404EB23449BB2C5
:100BA00043EA0443764541F8043B4FEA244CE7D836
:100BB00008F115018E4234BF00210121A6EB080681
:100BC000153EB608002906F101024FEA820208BF6D
:100BD0000422DDF804B00BEB0204A2454A4434D9E8
:100BE00015462146E04651F8046BB3B263444FEA20
:100BF000164E0EEB234E06EB08039BB243EA0E4360
:100C00008A454FEA2E4C45F8043BEBD80AF1FF3AEF
:100C1000AAEB040A2AF0030A524423B952F8043D0D
:100C2000013F002BFAD0076103B0BDE8F08F88DAEE
:100C300001258AE70021FFF76DFC70B10122002336
:100C4000C0E9042303B0BDE8F08F00294FEA86060F
:100C500008BF002609EB0602DFE7024640F2372113
:100C6000054B064807F052F9024640F24521024B77
:100C7000024807F04BF900BF14A501088CA5010834
:100C8000124B0A460B40A3F15073002B03DD0022E8
:100C90001946104670475B42B3F1A07F4FEA2351DB
:100CA00006DA4FF4002300220B4119461046704724
:100CB00014391E29D4BF4FF0004201224FF0000327
:100CC000D8BFCA4010461946704700BF0000F07FE9
:100CD000F8B5046900F1140202EB840454F8045CD2
:100CE000261F2846FFF7F0FC0346C0F120000A2B20
:100CF000086030DDB242A3F10B071AD254F8083C69
:100D00001FB3C7F1200C23FA0CF1BD4045EA0106E0
:100D1000A4F1080546F07F51AA4203FA07F341F413
:100D2000401116D254F80C2C22FA0CF21343184638
:100D3000F8BD0B2B08D0002305FA07F747F07F51C9
:100D4000184641F44011F8BD002345F07F5141F4AD
:100D500040111846F8BDB2422CBF002254F8082CAE
:100D6000C3F10B0703F1150325FA07FC38BFFA405E
:100D700005FA03F34CF07F511343184641F4401138
:100D8000F8BD00BFF0B5012183B016461F46FFF73E
:100D9000C1FB0546002847D0C7F30A54C7F3130325
:100DA0000CB143F48013002E019314D101A8FFF776
:100DB000ADFC0122019B20306B612A6114B3089BBA
:100DC000A4F2334404441C60099BC0F13500186050
:100DD000284603B0F0BD68460096FFF797FC019BDC
:100DE00000B30099C0F1200203FA02F2C34001935C
:100DF0000A43002B6A610CBF01220222AB612A6107
:100E0000002CDCD105EB8201A0F23243086908997D
:100E10000B60FFF759FC099BC0EB42101860284695
:100E200003B0F0BD009AE4E7024640F20F31024BF6
:100E3000024807F06BF800BF14A501088CA5010853
:100E40002DE9F04383B0884669468146FFF740FFAD
:100E500004460D46404601A9FFF73AFFD9F8103085
:100E6000D8F81020A3EB020CDDE900329B1A03EB4B
:100E70004C13002B0BDD05EB03573D4602460B469A
:100E800020462946F0F7C2F803B0BDE8F083C3EB73
:100E9000033301EB03594946F0E700BF01F1FF3C82
:100EA000116902F114034FEA6C1C03EB81010CF190
:100EB000010C8B4200EB8C0C16D210B5A0F1040E85
:100EC00053F8044B99424EF8044FF9D88B1A153B4E
:100ED00023F0030304331844844504D9002340F865
:100EE000043B8445FBD810BD844505D9002340F858
:100EF000043B8445FBD87047704700BF03694A1123
:100F0000934200F1140009DA00EB830302E053F886
:100F1000042DA2B98342FAD80020704700EB820367
:100F2000F8DD11F01F01F5D010B450F8224024FA7A
:100F300001F28A40944208D0012010BC7047012081
:100F4000704753F8042D002AF6D18342F9D80020C7
:100F500010BC7047242B2DE9F84F42D8012B40D00C
:100F60001F468E468046484875461EF801BB10F85D
:100F70000B4014F00804F7D1BBF12D0F6FD06FF0C8
:100F80000049BBF12B0F04BF9EF800B005F1020E23
:100F90007BBBBBF1300F4CD00A273B460025B9FB89
:100FA000F7F6284607FB169A05E03BD0012507FB1C
:100FB00000C01EF801BBABF1300CBCF1090F06D923
:100FC000ABF1410CBCF1190F1AD8ABF1370C6345EA
:100FD0001FDDB5F1FF3FECD08642E6D24FF0FF3582
:100FE000E7E7FEF775FC1622034600201A60BDE80D
:100FF000F88F102BD2D1BBF1300F23D01F46CDE795
:10100000ABF1610CBCF1190F03D8ABF1570C634580
:10101000DFDC6B1C2BD054B9002AE8D085BB1160F3
:10102000BDE8F88FE245C1DA4FF0FF35C1E7404235
:10103000F2E79EF8003003F0DF03582B08D00827B2
:101040003B46ABE79EF8000000F0DF005828D5D102
:1010500010279EF801B03B460EF1020E9EE79EF867
:1010600000B04FF00049012405F1020E90E7222361
:10107000C8F8003032B10EF1FF3148461160CFE7B9
:101080008146F8E74846B2E761DA0108FFF762BF38
:10109000034649B1FF2A02D801200A7070478A220C
:1010A0004FF0FF301A607047084670472DE9F04F47
:1010B000DDB00C4691460D910F93834606F026FE57
:1010C000036818461A93FEF747FC0822189000217F
:1010D0002CA8FEF7DFF8A389180603D52369002B97
:1010E00000F01587002300249E46CDE9313300230C
:1010F00033AACDE91634DA4614464D46CDE91BEE47
:101100003092CDF864E0CDF880E0CDF874E0CDF811
:1011100028E0CDF848E02F466E4BD3F8E460FEF7A8
:101120006BFB0DF1B00C03463A46504628A9CDF8AA
:1011300000C0B047002800F09F80C0F29580289B37
:10114000252B01D00744E7E7B7EB0508064640F03A
:10115000978000224FF0FF33934609937B787E1CE3
:101160008DF897200B9299460136A9F120035A2B4E
:1011700000F2B280DFE813F0F302B000B000EF023B
:10118000B000B000B000FD02B000B0006A0035024F
:10119000B0002702D202B000CE025B005B005B0011
:1011A0005B005B005B005B005B005B00B000B000BD
:1011B000B000B000B000B000B0002801B000AA013B
:1011C0003E02280128012801B000B000B000B000A4
:1011D0003A02B000B000A802B000B000B000D001E8
:1011E000B000BC02B000B0008A06B000B000B00091
:1011F000B000B000B000B000B0002801B000AA01FB
:1012000001022801280128012B0201027400B0000C
:101210006402B0005502AF066E027400B000D00147
:101220007200AC06B000B000B206B000720000223E
:10123000A9F1300316F8019B02EB820203EB420294
:10124000A9F13003092BF5D90B928EE70F9B53F8C8
:10125000042B002A0B920F93C0F2B281337882E7FD
:1012600033784BF0200B7EE7082200212CA8FEF7F4
:1012700011F8012007444FE7B7EB0508064610D0E8
:10128000329BC4E9005843443293319B0133072B0E
:10129000319315DC08340A9B43440A93002E7FF4F3
:1012A00058AF329B002B41F05E810D9B9B8903F070
:1012B0004003002B41F080830A985DB0BDE8F08FB9
:1012C00050460D9930AA08F0D7F90028EDD133AC7B
:1012D000E1E700BF540500201096B9F1000FE0D0FF
:1012E000012300228DF80C91069343AD8DF89720D1
:1012F0000C93CDE913220E92099211921BF0020376
:1013000002D00699023106911BF08408329E05D165
:101310000B9906980F1A002F00F39B806AB10122E7
:101320006260319A013601320DF19701072A329637
:101330003192216000F3D883083463B102236360E3
:10134000319B0236013326AA072B32963193226055
:1013500000F3BF830834B8F1800F00F0BF82099B0F
:101360000C9A9F1A002F00F3F9821BF4807F40F043
:101370001E820C9B25601E446360319B32960133B4
:10138000072B319300F33F8308341BF0040F05D083
:101390000B9B069A9D1A002D00F3B383DDE90A32F8
:1013A00006998A42ACBF9B185B180A93002E40F046
:1013B0000883002331930E9B1BB150460E99FEF714
:1013C0006FFB33AC109DA6E60F9B1096073323F0FE
:1013D0000703F3E802670F9327F000431F931E965D
:1013E0004FF0FF32DDE91E01B24BCDE91667EFF792
:1013F000F3F9002840F0F484DDE91E014FF0FF32DC
:10140000AC4BEFF7CBF9002840F0EA840022002330
:1014100030463946EFF7B8F9002840F0B2879DF81A
:10142000972000210320A44DA44B2BF0800B0E919C
:101430000690B9F1470FD8BF1D46CDE913110991A8
:101440000C901191002A3FF459AF069B013306938B
:1014500054E7102F319A41F30D82DFF864C2214620
:1014600030460D9C2E46CDF854C06546219304E0CD
:10147000103F102F01F1080116DD1023013210304A
:10148000072ACDE931200D604B60F1DD2146504641
:1014900030AA08F0F1F8002840F09B82DDE9312005
:1014A000103F102F33A9E8DC35460C460646219B39
:1014B000013215993E44072ACDE931262160676043
:1014C00000F381869DF89720083427E70F9BB9F138
:1014D000430F109603F1040603D01BF0100F00F029
:1014E0000185082200212EA8FDF7D4FE0F9A43ADF6
:1014F0002EAB29465046126807F09AFF0346013387
:101500000C9001F054820C9B23EAE37306930022B3
:101510000F968DF89720ECE600230F9F109657F852
:10152000045B8DF89730002D00F00085B9F1530F62
:1015300000F094861BF01003119340F08F86099BF6
:10154000002BC1F21B801A462846119906F01CFC9C
:101550000E90002801F081820E9B11995B1B0C9369
:1015600023EAE3734FF07309CDE913119DF8972037
:101570000F97099106930E9164E71BF0200F1096C8
:101580003ED00F9B073323F007031846596850F8E5
:10159000083B0A460F900029C0F2CA830999002926
:1015A000C0F2888253EA02012BF0800740F0838268
:1015B000099A002A40F08482BB460C925CAD64E13B
:1015C0000B9B5B420B9333784BF0040BCBE53378EA
:1015D000682B03BF73784BF4007B01364BF0400B54
:1015E000C1E52B238DF897303378BCE533784BF089
:1015F000080BB8E54BF0100B1BF0200F1096C0D174
:101600000F9A1BF0100F52F8043B0F9240F0C28368
:101610001BF0400F00F0BA8343F3C03211461BB2F7
:10162000B9E71BF0200F109600F0C5830F9B0A9AB4
:101630001B681A60D2175A600F9B04330F93C1E6E0
:1016400033786C2B03BF73784BF0200B01364BF0D3
:10165000100B88E547F630030F9AADF8983052F832
:10166000043B02210F924FF0780900221548109692
:101670004BF0020719900020099D8DF89700002D6E
:10168000C0F2EC8053EA020027F0800B40F0E580C6
:10169000002D40F0D285002940F0538317F001035C
:1016A0000C9300F0718330230DF26F158DF86F31BC
:1016B000EBE000BFFFFFEF7FECA50108E8A5010804
:1016C00070DD0108F8A5010810964BF0100B1BF017
:1016D000200200F012830F9B073323F00703194603
:1016E0005A6851F8083B0F9100212BF48067C2E73C
:1016F00010964BF0100717F0200200F00B830F9BA1
:101700000121073323F0070318465A6850F8083BB5
:101710000F90B0E733784BF0800B24E5314611F899
:10172000019BB9F12A0F01F02882A9F13003092B9E
:1017300098BF002201F2A28011F8019B02EB820205
:1017400003EB4202A9F13003092BF5D942EAE27317
:101750000E46099309E533784BF0010B03E59DF83C
:1017600097203378002A7FF4FEAC20228DF8972052
:10177000F9E4504606F0CAFA436818461D93FEF78E
:10178000EBF820900746504606F0C0FA83681B939A
:10179000002F3FF463AD1B9A3378002A3FF4E3AC8B
:1017A0001278002A3FF4DFAC4BF4806BDBE4B9F134
:1017B000650F40F33781DDE9160100220023EEF7C3
:1017C000D9FF002800F0D88101236360319B934A40
:1017D00001330136072B32963193226000F33285B4
:1017E0000834279B129A934280F2C982189B1A9A56
:1017F0001E44C4E90023319B32960133072B3193F9
:1018000000F37A830834129B5D1E002D7FF7BDAD77
:10181000102D319B40F3EB80DFF804921027DDF8A8
:101820003480CDF8549004E00834103D102D40F37E
:10183000E08001331036072BC4E90097CDE931363B
:10184000F2DD4146504630AA07F016FF002840F06E
:10185000C080DDE9313633ACE7E75F46012900F0AF
:101860002A8102295CAD1ED1199803F00F01415C59
:101870001B0943EA0273120905F8011D53EA02012C
:10188000F3D1BB465CAB5B1B0C93099A0C9900230C
:101890008A42B8BF0A46CDE9133306920E939DF8EB
:1018A00097201193CEE503F00701DB0843EA42736A
:1018B000D208303153EA0206284605F8011DF2D15C
:1018C000FB07DED53029DCD03023023805F8013C97
:1018D0005CAB1B1ABB4605460C93D6E70B9B069ADE
:1018E0009F1A002F7FF73BAD102F319B41F35B8098
:1018F0004B48224631464FF0100806460D9C159085
:1019000004E0103F102F02F1080214DD0133103102
:10191000072BC2E90068CDE93131F2DD214650469E
:1019200030AA07F0A9FE002853D1DDE93131103F7C
:10193000102F33AAEADC14460E460133159A3E44B2
:10194000072BCDE931362260676000F3C084099B24
:101950000C9A08349F1A002F7FF707AD304A102FDA
:10196000319B159221DD32464FF010082E460D9D19
:1019700004E0103F102F04F1080414DD013328495E
:101980001032072BC4E90018CDE93132F1DD2946C8
:10199000504630AA07F070FED8B9DDE93132103F69
:1019A000102F33ACEADC354616460133159A3E4417
:1019B000072BCDE931362260676000F3928108344D
:1019C000D3E450460D9930AA07F056FE00283FF4A4
:1019D000F0ACD3460E9B002B3FF467AC58460E99F3
:1019E000FEF75EF80D9B9B8903F0400361E40C4A0F
:1019F0001592159A01332E44072B22606560CDE9BC
:101A000031367FF7C1AC50460D9930AA07F034FE4D
:101A10000028DED1329E33ACB7E400BF28A601080F
:101A200060DD0108129B319F012B06F1010607F1D1
:101A3000010704F1080940F310810123072FCDE9C4
:101A400031762560636000F38081189B01371A9A14
:101A50001E44072FC9E90023CDE9317600F38281C6
:101A600009F10809129B0022DDE916015C1E002322
:101A7000EEF780FE002840F0098101370135264449
:101A8000072FCDE93176C9F80050C9F8044000F3BA
:101A9000F08009F108091C9B01371E44C9F8043085
:101AA000072F2AABCDE93176C9F80030ABDC09F15C
:101AB00008046AE45F460A2B72F1000180F0258376
:101AC00030338DF86F310123BB460C930DF26F1547
:101AD000DBE650460D9930AA07F0CEFD00287FF4D2
:101AE00078AF329E33AC36E450460D9930AA159348
:101AF00007F0C2FD00287FF46CAF329E159B33AC1B
:101B00001BE4102D319B40F33187DFF8CC82102786
:101B1000DDF83490CDF8548004E0103D102D04F130
:101B2000080415DD01331036072BC4E90087CDE921
:101B30003136F2DD4946504630AA07F09DFD0028B7
:101B40007FF447AFDDE93136103D102D33ACE9DCD1
:101B50000133159A2E44072BC4E90025CDE931360F
:101B60007FF71CAC50460D9930AA07F085FD002880
:101B70007FF42FAF329E11E42799002940F333837D
:101B8000DDE911839845A8BF9846B8F1000F0ADD3A
:101B9000319B46440133072BC4E9005832963193F8
:101BA00000F33E860834119FB8F1000FA8BFA7EBE1
:101BB0000807002F00F3CB81DDF844901BF4806F01
:101BC000A94440F0EA81279B129A9342C0F27182A5
:101BD0001BF0010F40F06D82129AAF18A7EB0907B6
:101BE000D51AAF42A8BF2F46002F0BDD319B3E44D4
:101BF0000133072BC4F8009067603296319300F3ED
